:020000040800F2
:10000000000002203F130208CD020008CD020008C4
:10001000CD020008CD020008CD020008000000005B
:10002000000000000000000000000000D1020008F5
:10003000CF0200080000000001030008F32F0108B0
:10004000CD020008CD020008CD020008CD02000854
:10005000CD020008CD020008CD020008CD02000844
:10006000CD020008CD020008CD0200080F6501088E
:100070001F6501082F6501083F6501084F650108EC
:10008000CD020008CD020008CD020008CD02000814
:10009000CD020008CD020008CD0200085F6501080E
:1000A000CD020008CD020008CD020008CD020008F4
:1000B000CD0200086B650108CD020008CD020008E2
:1000C000CD020008CD020008CD020008CD020008D4
:1000D0007B650108CD0200088B650108A365010856
:1000E000CD020008CD02000800000000CD0200088B
:1000F000CD020008CD020008B3650108CD0200085A
:10010000CD020008C3650108CD020008CD02000839
:10011000CD020008CD020008CD020008D365010819
:10012000CD020008CD020008CD020008CD02000873
:10013000CD020008CD020008CD020008CD02000863
:1001400000000000000000000000000000000000AF
:10015000CD020008CD020008CD020008CD02000843
:10016000CD020008CD020008CD020008CD02000833
:10017000CD020008CD020008CD02000800000000FA
:10018000CD020008CD020008CD020008CD02000813
:10019000E3650108CD020008CD020008CD02000889
:1001A000CD020008CD020008CD02000800000000CA
:1001B000CD020008CD020008CD020008CD020008E3
:1001C000CD020008CD020008000000000000000081
:1001D0000000000000000000CD0200080000000048
:1001E000000000000000000000000000000000000F
:1001F0000000000000000000CD020008CD02000851
:10020000CD020008CD02000800000000CD02000869
:10021000CD020008CD020008CD020008CD02000882
:10022000CD02000800000000F36501080000000096
:10023000CD020008CD02000800000000CD02000839
:10024000CD020008CD020008CD020008CD02000852
:10025000CD020008CD020008CD020008CD02000842
:10026000CD020008CD020008CD020008CD02000832
:10027000CD020008CD020008CD02000800000000F9
:10028000CD020008CD020008CD020008CD02000812
:1002900000000000CD020008CD02000800000000B0
:1002A00000000000CD020008CD020008CD020008C9
:1002B00003660108CD020008CD020008CD02000847
:0C02C000CD020008CD020008CD020008AD
:0202CC00FEE74B
:0202CE00704777
:1002D000074B19680868B0E8F04F80F30988BFF34E
:1002E0006F8F4FF0000080F31188704700BF00BF90
:0402F000AC24002416
:0C02F400241F0208B041000890410008DF
:10030000EFF30980BFF36F8F154B1A681EF0100FC3
:1003100008BF20ED108A20E9F04F10602DE9090098
:100320004FF0500080F31188BFF34F8FBFF36F8FF2
:1003300014F01FFC4FF0000080F31188BDE80900A5
:1003400019680868B0E8F04F1EF0100F08BFB0EC55
:10035000108A80F30988BFF36F8F704700BF00BF1A
:04036000AC240024A5
:0403640072B6FEE788
:100368002DE9F84F2DED068B84B0B5EE401BF1EE6C
:1003780010FA00F09180B4EE411BF1EE10FA80F112
:100388008B80B0EE408B50EC101B420042EAD171DA
:1003980011F5001F9FED429B77D2B0EEC89BB0EEDF
:1003A800C1ABB4EE4A9BF1EE10FA02D5B0EE489B11
:1003B8006BE0B4EE4A9BF1EE10FA05D100F0004074
:1003C800002140EC191B60E002A8B0EE4A0B20F0B7
:1003D800CCFFB4EE4A9BF1EE10FA4FDB59EC1A0B46
:1003E8000190029F09F0004A4AF0E04040F07F6B1C
:1003F800C9F30A556FF31E5940F2FF78B0EE490B66
:1004080003A820F0B2FF0398C01B691EB0EE4A0B88
:1004180012D34545B0EE4A0B0ED0431940F2FE7296
:10042800002693425A4605DC012B5246A4BF49EAEE
:100438000352019E42EC106BB4EE490BF1EE10FA38
:1004480015DDB0EE4A0B95B14545B0EE4A0B0ED01E
:10045800014440F2FE7000228142584605DC012921
:100468005046A4BF49EA0150019A40EC102B39EEDE
:10047800409BB4EE4A9BF1EE10FABFDAB5EE408B22
:10048800F1EE10FA48BFB1EE499BB0EE490B04B04B
:10049800BDEC068BBDE8F88F9FED019BF5E700BF2B
:0804A800000000000000F87FD5
:1004B00050EC10CBC0F30A52531E40F2FE718B4237
:1004C00051D240F2FE318A4208D8BFEE000B9FEDB8
:1004D0002A1BB0F1FF3F31FE000B704740F2324162
:1004E0008A4288BF7047F0B5A2F2FF33B3F1200112
:1004F0004FF48017C3F1200407FA04F540F2000618
:10050000CFF6F07606FA04F25CBF27FA01F546FA58
:1005100001F202EA0C0E27FA03F24EBF1E4100223E
:100520004FF0FF36064015EB0E0572412CFA04F42D
:1005300000FA03F73C43002958BF0CFA01F46FF3AB
:100540001F540CFA03F148BF0C43B4FA84F1490973
:100550000028A8BF41F0010100291CBF32467546A2
:1005600042EC105BF0BD002A04BF00F0004094464E
:1005700040EC10CB704700BF0000000000000000FE
:10058000000000000000244000000000000059406E
:10059000000000000088C3400000000084D797419D
:1005A0000080E03779C34143176E05B5B5B893466F
:1005B000F5F93FE9034F384D321D30F94877825A3B
:0805C0003CBF737FDD4F157590
:1005C80001000000000000000A0000000000000018
:1005D8006400000000000000E803000000000000C4
:1005E8001027000000000000A086010000000000A5
:1005F80040420F00000000008096980000000000B4
:1006080000E1F5050000000000CA9A3B0000000068
:1006180000E40B540200000000E8764817000000D0
:100628000010A5D4E800000000A0724E18090000D0
:1006380000407A10F35A00000080C6A47E8D0300A3
:100648000000C16FF286230000008A5D78456301CF
:10065800000064A7B3B6E00D0000E8890423C78A48
:100668002DE9F84F2DED0A8B8EB00692894680460B
:100678000020C8F800000DF11D0003909FEDC6ABE7
:10068800B2EE048BB7EE00BB9FEDC5CB19F8011B8A
:10069800252906D0002900F0DA85404620F09DFE85
:1006A800F4E70026494619F8012BA2F12003102B84
:1006B8000DD88020DFE803F0091B1B191B1B1B1535
:1006C8001B1B30181B101B1B120040200DE05E2A5C
:1006D8000DD14FF4805008E0102006E04FF4007070
:1006E80003E04FF4004000E020200643DAE701F180
:1006F8000109A2F1300009284FF000001BD819F8B1
:10070800011B00EB800002EB40003038A1F1300201
:100718000A2A0A46F3D30EE0069850F8042B0690EE
:10072800002A104648BF5042102303EAD2621643FB
:100738004A7801F102092E2A0DD1494611F8012BF8
:100748002A2A0BD1069999F8012051F804AB069191
:1007580009F1020916E04FF0000A1CE0A2F130038B
:10076800092B4FF0000A13D811F8013B0AEB8A094C
:1007780002EB4902A2F1300AA3F130020A2A1A4612
:10078800F2D38946BAF1000F58BF46F4807602E0EA
:1007980046F4807689466B2A0ADC4C2A03D0682AFC
:1007A80018D06A2A28D119F8012B46F0020623E04E
:1007B8006C2A05D07A2A14BF742A19F8012B1BE079
:1007C800494611F8012B6C2A10D199F8012009F13A
:1007D8000209EAE7494611F8012B682A09D199F874
:1007E800012009F1020946F0080605E046F0010675
:1007F80001E046F00406894620EAE077462A1FDD34
:10080800A2F1630015282FD8DFE810F06000170068
:1008180045002300A4011600170016001600160054
:100828001600700084004E00160016007F001600A7
:10083800480016001600360028E746F4804631E0E6
:10084800442A09DD452A24D0462A7FF41FAF46F4FE
:10085800005646F4006B7FE1252A40F06582404649
:10086800252120F0BAFD11E7472A00F07181582AA6
:100878007FF40CAF46F40056F0054FEA066048BF17
:1008880026F4007643F25801782A08BF43F278012B
:1008980047E046F4005646F4806B5DE1F00548BF3A
:1008A80026F4007600213EE03006232101EAE070BC
:1008B800CDE9047046F48076069A002152F8040BBC
:1008C80006924FF0080A0DF11E04DEE00698A7F123
:1008D800010A10F8044B069040463146524615F07E
:1008E800B7F84046214620F078FDAEE1069951F868
:1008F800040B06913107D8F8001000F11982B207ED
:1009080052BF0160002206C0C0E6069850F8044BAA
:10091800069079E1F0054FEA066048BF26F40076B4
:10092800302101EAE07170044FEA8670069DCDE936
:10093800047104D4002808D42B1D00210BE00028E2
:1009480015D455F8040BC11717E0E81D20F007056A
:1009580005F1080369680DF11E04286875070693F8
:1009680015D416F008051CBFC0B2002132E0E81DFE
:1009780020F00705696855F8080B0DF11E04730788
:1009880012D4330744BF40F3C01140B20FE080B225
:1009980000211FE000BF00BFA0C8EB85F3CCE17FBA
:1009A800000000000000594040F3C03100B20029A7
:1009B800069507DBB3060BD47306059D48BF2025B3
:1009C800059507E00023404263EB01012D2300E079
:1009D8002B230593F30548BF26F40076F30558BF8B
:1009E8004FF0010A00276E2A21DD6F3A092A00F22A
:1009F8006D80DFE802F0054A6B6B6B6B226B6B4A0C
:100A080050EA010262D0C20842EA41720625134642
:100A180065F3DF00E055013752EAD1004FEAD10112
:100A28004FEAD20040EA41721846F0D14EE0582A07
:100A38002BD0642A18BF692A48D150EA010245D050
:100A48000C46054630040AD507F00300032806D1F2
:100A58000DF11E0B2C200BF80700013701E00DF1FA
:100A68001E0B28460A22002303F07CFA00EB8002C2
:100A7800A5EB420242F030020BF807200137D5F10E
:100A880009020022A241DBD320E0002750EA01023C
:100A98001CD0B20442F24042C0F602025CBF42F2ED
:100AA8005042C0F60202030943EA017500F00F0044
:100AB8002B46105CE055013755EA11104FEA111129
:100AC8004FEA151040EA01751846EFD105994FF025
:100AD800FF30FF2988BF0138AAEB070222EAE27A31
:100AE80007EB0A03049AD41A002918BF0444B00576
:100AF80006D440463146224614F0AAFF0599002440
:100B0800FF29039D05D9090A404620F066FC05998E
:100B180000E011B1404620F060FC404631462246D4
:100B280014F096FF40463021524620F0A6FC012FD3
:100B380005DBE95D404620F050FC013FF9D8F0069E
:100B48007FF5A4AD40462021224620F096FC9DE585
:100B580046F4005646F4406B5FEACB5058BF4FF05E
:100B6800060A0BF4406006990731A0F5406021F0B1
:100B78000701B0FA80F0BAF1000F08BF4FEA501A27
:100B8800D1E9005646EC195B01F108000690B0EE79
:100B9800490B14F01EFF80B1B5EE409BF1EE10FA40
:100BA8001DD55FEA8B4042F2B804C0F602045CBF70
:100BB80042F2BD04C0F6020424E0B0EE490B20F076
:100BC800C6FB00284AD05FEA8B4042F26044C0F678
:100BD80002045CBF42F26444C0F6020412E01BF453
:100BE800005042F2C202C0F6020242F2C701C0F649
:100BF8000201104612BF541C08464C1C5FEA8B6168
:100C080048BF04462BF48076002C04BF41F612340A
:100C1800C0F60204F005204602D420F0C0FC02E031
:100C2800514620F0D2FC054626F40076A7EB000AD0
:100C380040463146524614F00BFF35B114F8011BFB
:100C4800404620F0CAFB013DF8D1F0067FF51EAD05
:100C580040462021524620F010FC17E5B0EE490B23
:100C680014F0C4FE002804BF0646054646EC195B8E
:100C7800B0EE490B20F073FB044686F0004040ECD0
:100C8800105B002C09FE009BB0EE490B0DA820F06C
:100C98006AFB0D9800EB400046F26761C6F2666198
:100CA80050FB01F0002C18BF4BF0600B811001EBDA
:100CB800D0700D90B5EE409BF1EE10FA16D00130D1
:100CC80020F06DFBB4EE490BF1EE10FA0D9806D545
:100CD800411C0D910230F3E70D9801380D9020F07A
:100CE8005EFBB4EE490BF1EE10FAF5DC0D990BF44E
:100CF8004064B4F5806F07D0B4F5406F0AD18A45D7
:100D0800C8BF11F1050F05DCB1F59A7F13D189EE43
:100D18000A9B15E05FEA4B5040F1E7800E2940F34B
:100D2800C1804FF0000AE0E0002A7FF4AFACA1E2F6
:100D38000170FFF7ABBC484220F031FB20EE099B65
:100D4800B5EE409BF1EE10FA23D0B0EE490B14F04B
:100D580040FE00287FF420AF0D98B4EE489BF1EEDA
:100D680010FA08DB89EE089B0130B4EE489BF1EEDF
:100D780010FAF7DA0D90B4EE4B9BF1EE10FA08D5A5
:100D880029EE089B0138B4EE4B9BF1EE10FAF7D42C
:100D98000D90B4F5406F544608BF013CBAF1000FFE
:100DA80018BFA246CAF1000020F0F9FA4FF0FF3050
:100DB80014F02DFE30EE090BB4EE480BF1EE10FAEC
:100DC800A1BF0D9880EE080B01300D9050EC106B10
:100DD8000290BAF1000F35D005940BF40860B0F515
:100DE800006F31D1BAF1100FA8BF4FF0100A029866
:100DF80040EC196B504620F0D2FA20EE090B51EC6A
:100E0800100B03F061F80446084300F007820D4612
:100E18004CF6CD42CCF6CC42A4FB0201531E04FB97
:100E2800031105FB0211C20742EA5102C90741EA50
:100E38005000D0F1993049F69910C1F699109041B7
:100E480080F0EE81CDF814A0059A0BF080001043D5
:100E5800A7EB02000D9D0CBF471F871F01245FEA07
:100E6800CB4002D404950299BDE045F25650C5F234
:100E7800555055FB00F000EBD07000EB4000281AED
:100E880002300299DFE800F003A1AB03A10041ECB6
:100E9800106B20EE080B51EC106B013D0D95013FD6
:100EA80002249CE0C84350444FF0100A1028B8BFF1
:100EB80082465FEA0B6218D4B8B1504620F06FFA48
:100EC800B6EE001B00EE091BB0EE410BFFF7ECFA83
:100ED800B0EE481BFFF744FAB5EE400BF1EE10FAFE
:100EE80002D1BAF1010AE8D10D99CDF814A0CAF1DE
:100EF800000010398142C8BF084620F050FA4FF070
:100F0800FF3014F084FD30EE099B0D98013020F07D
:100F180046FAB4EE490BF1EE10FA0D9898BF01307D
:100F2800002814D411281AD3A0F110010D91C0F192
:100F3800100020F034FA20EE090B51EC100B02F0EF
:100F4800C3FF05460E460020CDE9010019E050EC2C
:100F5800191BCDE9011000250D95002611E051EC73
:100F6800190B02F0B1FF05460E4602F0CDFF41EC29
:100F7800100B39EE400B50EC101BCDE9011000208E
:100F88000D902BF4806A40F2C850C0F6000008307B
:100F9800002400F10801013405C8281A76EB020084
:100FA8000846F6D2059AB81A0BF0800111434FF0A3
:100FB800FF321CBF1146013A1BF0600F08BF0A46FA
:100FC8000D99511A0844071B2AE041EC106B20EEDA
:100FD8000C0B51EC106B023D0D95023F032422EAE5
:100FE800E272CDE904522BF4006A41EC196B3046E9
:100FF80002F06AFF05460E4602F086FF41EC100B30
:1010080039EE400B50EC101BCDE901101BF0600FBE
:1010180018BF013F049820F0BEF96328C8BF013FFC
:1010280027EAE77B1AF4047F0DD1012F0BDB40F28E
:10103800C857C0F600074046202120F0CEF9BBF182
:10104800010BF8D103E040F2C857C0F600075FEA89
:101058008A604FEA4A6003D4002808D5202103E0BB
:101068002D21002858BF2B21404620F0B6F95FEA11
:10107800CA6009D4BBF1000F06D04046302120F0E9
:10108800ACF9BBF1010BF8D1013C07EBC40006C871
:10109800681A76EB0200302006D36D1A96410130AB
:1010A8006B1A76EB0203F8D2C1B2404620F095F9EC
:1010B800002CE9D15FEA0A540BD50D98012808DB0A
:1010C80001380D904046302120F087F90D9800280E
:1010D800F6DC0AF08000059D284343D040462E21C7
:1010E80020F07BF91020102DB8BF2846002C0D9950
:1010F80020EAE077384648BF401A20F050F9012D21
:1011080026DBDDE9011040EC111B20EE010B51EC50
:10111800100B02F0D9FE04460D463E46013E40F251
:10112800C850C0F6000000EBC60006C8601A75EB90
:101138000200302006D3641A95410130631A75EB1A
:101148000203F8D2C1B2404620F047F9002EE5D19B
:101158000599C81B06D07C1A4046302120F03DF97D
:101168000134F9D35FEA4A504BD545215FEA8A40FA
:1011780058BF6521404620F030F90D9800284046B8
:1011880004DB2B2120F029F90D9805E02D2120F012
:1011980024F90D9840420D90642815DB48F21F543D
:1011A800C5F2EB14A0FB0401302000EB51114046BE
:1011B80020F013F90D9850FB04F14A1102EBD1719C
:1011C800642201FB12000D9046F26764C6F2666461
:1011D80050FB04F0811001EBD07000F13001404663
:1011E80020F0FBF80D9850FB04F18A1002EBD17146
:1011F80001EB8101A0EB410000F13001404620F0F5
:10120800ECF8BBF1000F3FF441AA4046202120F042
:10121800E4F8BBF1010BF8D1FFF738BA059013E6F3
:10122800CDF814A0204629460A22002302F09AFE8F
:1012380004460D460A22002302F094FE0598013860
:1012480005903FF401AE52EA0300EBD0FCE5D8F874
:101258000C0028B1D8E9001291423CBF0022425448
:10126800404620F0FCF8D8F800000EB0BDEC0A8B20
:10127800BDE8F88F404620F0F2F84FF0FF30F4E771
:1012880085B0049000208DF80F0004988069E8B9B3
:101298000498806A0290032817D80299DFE801F0C1
:1012A800020B0214049890F82F00C00710B1012017
:1012B8008DF80F0009E00498C06AB0F1C07F02D130
:1012C80001208DF80F0000E0FFE73BE004988069FB
:1012D800B0F5005F20D10498806A019003281AD8DD
:1012E8000199DFE801F00206020F01208DF80F00D6
:1012F80011E0049890F82F00C00710B101208DF874
:101308000F0008E00498C06AB0F1C07F02D1012044
:101318008DF80F00FFE715E00498806A0090032815
:1013280003D30098032804D00CE001208DF80F00A7
:1013380008E0049890F82F00C00710B101208DF83C
:0C1348000F00FFE79DF80F0005B0704794
:101354008AB044F21040C5F60200006800F038007C
:1013640001460191182800F25A810199DFE811F031
:1013740019005701570157015701570157015701E8
:1013840035005701570157015701570157015701BC
:101394003B005701570157015701570157015701A6
:1013A400410044F20040C5F602000068C0F340105A
:1013B40068B144F20040C5F602000068C0F3C10100
:1013C40049F20000C0F2D030C840029004E049F273
:1013D4000000C0F2D030029026E140F60010C0F2C6
:1013E4003D00029020E147F64000C0F27D100290DB
:1013F4001AE144F22840C5F60200016801F0030135
:1014040008910068C0F30510079044F22C40C5F61B
:101414000200006800F001000690069844F234418E
:10142400C5F60201096889B2C908484300EE100AEA
:10143400B8EE400A8DED040A0798002800F0EC800D
:101444000898009038B10098012863D000980228C9
:1014540000F08480A6E044F20040C5F60200006873
:10146400C0F3401090B344F20040C5F60200006897
:10147400C0F3C10149F20000C0F2D030C840059069
:101484009DED050AB8EE400A9DED071AB8EE411A23
:1014940080EE010A44F23040C5F6020000686FF3A2
:1014A4005F2001EE100AB8EE411A9DED042A9FED6B
:1014B400613A82EE032A31EE021AB7EE002A31EEC7
:1014C400021A20EE010A8DED030A22E09DED070ABF
:1014D400B8EE401A9FED590A80EE010A44F23040FA
:1014E400C5F6020000686FF35F2001EE100AB8EE43
:1014F400411A9DED042A9FED4F3A82EE032A31EE04
:10150400021AB7EE002A31EE021A20EE010A8DED1E
:10151400030A6AE09DED070AB8EE401A9FED460AF9
:1015240080EE010A44F23040C5F6020000686FF311
:101534005F2001EE100AB8EE411A9DED042A9FEDDA
:101544003D3A82EE032A31EE021AB7EE002A31EE5A
:10155400021A20EE010A8DED030A46E09DED070A0A
:10156400B8EE401A9FED320A80EE010A44F2304090
:10157400C5F6020000686FF35F2001EE100AB8EEB2
:10158400411A9DED042A9FED2B3A82EE032A31EE97
:10159400021AB7EE002A31EE021A20EE010A8DED8E
:1015A400030A22E09DED070AB8EE401A9FED220AD5
:1015B40080EE010A44F23040C5F6020000686FF381
:1015C4005F2001EE100AB8EE411A9DED042A9FED4A
:1015D400193A82EE032A31EE021AB7EE002A31EEEE
:1015E400021A20EE010A8DED030A44F23040C5F6DA
:1015F4000200006881B2012000EB512009909DEDAA
:10160400030A9DED091AB8EE411A80EE010ABCEEF8
:10161400C00A8DED020A01E00020029004E040F6C9
:101624000010C0F23D00029002980AB0704700BF5B
:1016340020BCBE4B000000460024744A0024744CB5
:1016440080B59AB0189000208DF857008DF8560098
:101654001898C0780007002840D51898406E149058
:1016640060B11498B0F5801F11D01498B0F5001F24
:1016740015D01498B0F5401F19D019E044F22C414C
:10168400C5F60201086840F40030086013E01898B9
:101694000830022108F0E8FB8DF857000BE0189899
:1016A4002830022108F037FD8DF8570003E002E0EE
:1016B40001208DF857009DF8570058B944F2504165
:1016C400C5F60201086820F44010189A526E1043BF
:1016D400086003E09DF857008DF85600189840788C
:1016E400C00700283BD01898806D1390042820D898
:1016F4001399DFE801F0030C141C1D0044F22C4183
:10170400C5F60201086840F40030086014E0189837
:101714000830002108F0A8FB8DF857000CE0189859
:101724002830002108F0F7FC8DF8570004E003E0AE
:1017340002E001208DF857009DF8570058B944F293
:101744005041C5F60201086820F00700189A926D0E
:101754001043086003E09DF857008DF85600189870
:101764004078400700284CD51898D0F8A40012906F
:10177400A0B11298B0F5001F19D01298B0F5800FDF
:101784001DD01298B0F5C00F21D01298B0F5000FFB
:101794001ED01298B0F5200F1BD01BE044F22C4150
:1017A400C5F60201086840F40030086015E0189896
:1017B4000830002108F058FB8DF857000DE0189808
:1017C4002830002108F0A7FC8DF8570005E004E05C
:1017D40003E002E001208DF857009DF8570060B93E
:1017E40044F25841C5F60201086820F46000189AD2
:1017F400D2F8A4201043086003E09DF857008DF848
:10180400560018984078000700284CD51898D0F84E
:10181400A8001190A0B11198B0F1807F19D011984F
:10182400B0F1007F1DD01198B0F1407F21D0119804
:10183400B0F1806F1ED01198B0F1A06F1BD01BE0E7
:1018440044F22C41C5F60201086840F400300860F7
:1018540015E018980830002108F006FB8DF85700B1
:101864000DE018982830002108F055FC8DF8570039
:1018740005E004E003E002E001208DF857009DF844
:10188400570060B944F25841C5F60201086820F0D7
:10189400E060189AD2F8A8201043086003E09DF88D
:1018A40057008DF856001898C0788007002836D560
:1018B4001898C06C1090D8B11098102806D01098C1
:1018C40020280CD01098302811D012E044F22C417A
:1018D400C5F60201086840F4003008600CE018986E
:1018E4000830022108F0C0FA8DF8570004E003E044
:1018F40002E001208DF857009DF8570058B944F2D2
:101904004C41C5F60201086820F03000189AD26CE8
:101914001043086003E09DF857008DF856001898AE
:101924004078C006002845D51898C06D0F9080B146
:101934000F98B0F5805F15D00F98B0F5005F19D0FF
:101944000F98B0F5405F1DD00F98B0F5804F1AD0B6
:101954001AE044F22C41C5F60201086840F4003054
:10196400086014E018980830002108F07DFA8DF81A
:1019740057000CE018982830002108F0CCFB8DF8B3
:10198400570004E003E002E001208DF857009DF8C1
:10199400570058B944F25041C5F60201086820F4D2
:1019A400E040189AD26D1043086003E09DF8570098
:1019B4008DF85600189840788006002842D518986B
:1019C400006E0E90A0B10E98B0F5803F11D00E9825
:1019D400B0F5003F15D00E98B0F5403F19D00E98E1
:1019E400B0F5802F16D00E98B0F5A02F13D013E0C9
:1019F40015E018980830012108F036FA8DF85700E0
:101A04000DE018982830012108F085FB8DF8570067
:101A140005E004E003E002E001208DF857009DF8A2
:101A2400570058B944F25041C5F60201086820F441
:101A3400E020189A126E1043086003E09DF85700E6
:101A44008DF85600189840784006002844D5189818
:101A5400D0F8AC000D90A0B10D98B0F1805F11D01A
:101A64000D98B0F1005F15D00D98B0F1405F19D01A
:101A74000D98B0F1804F16D00D98B0F1A04F13D04F
:101A840013E015E018980830012108F0EDF98DF8FD
:101A940057000DE018982830012108F03CFB8DF820
:101AA400570005E004E003E002E001208DF8570050
:101AB4009DF8570060B944F25841C5F60201086820
:101AC40020F0E040189AD2F8AC201043086003E0FC
:101AD4009DF857008DF856001898407800060028A5
:101AE40034D51898C06E0C90C8B10C98B0F1805FD2
:101AF40004D00C98B0F1005F09D011E044F22C41FD
:101B0400C5F60201086840F4003008600BE018983C
:101B14000830012108F0A8F98DF8570003E002E02D
:101B240001208DF857009DF8570058B944F25041F0
:101B3400C5F60201086820F04050189AD26E10438E
:101B4400086003E09DF857008DF856001898C07897
:101B5400C00790B31898806C0B90032817D80B9982
:101B6400DFE801F014020B1344F22C41C5F6020124
:101B7400086840F4003008600CE01898083002212E
:101B840008F072F98DF8570004E003E002E0012048
:101B94008DF857009DF8570058B944F24C41C5F6EA
:101BA4000201086820F00300189A926C1043086040
:101BB40003E09DF857008DF8560018988078400689
:101BC400002840F1E6821898D0F8B000B0F5807F84
:101BD40000F03A821898D0F8B000B0F5007F00F019
:101BE40033821898D0F8B000B0F50C5F00F02C8266
:101BF4001898D0F8B000B0F54C5F00F02582189822
:101C0400D0F8B000B0F5864F00F01E821898D0F8D6
:101C1400B000B0F5A64F00F017821898D0F8B000C5
:101C2400B0F5C64F00F010821898D0F8B000B0F5A7
:101C3400E64F00F009821898D0F8B000B0F5034FD1
:101C440000F002821898D0F8B000B0F5134F00F0FD
:101C5400FB811898D0F8B000B0F5234F00F0F48160
:101C64001898D0F8B000B0F5334F00F0ED81189813
:101C7400D0F8B000B0F5434F00F0E6811898D0F8E2
:101C8400B000B0F5534F00F0DF811898D0F8B000E1
:101C9400B0F5634F00F0D8811898D0F8B000B0F5D3
:101CA400734F00F0D1811898D0F8B00040F20031A1
:101CB400C0F20101884200F0C7811898D0F8B00042
:101CC40041F20031C0F20101884200F0BD81189850
:101CD400D0F8B00042F20031C0F20101884200F0B5
:101CE400B3811898D0F8B00043F20031C0F201017A
:101CF400884200F0A9811898D0F8B00044F200316D
:101D0400C0F20101884200F09F811898D0F8B00019
:101D140045F20031C0F20101884200F09581189823
:101D2400D0F8B00046F20031C0F20101884200F060
:101D34008B811898D0F8B00047F20031C0F201014D
:101D4400884200F081811898D0F8B00048F2003140
:101D5400C0F20101884200F077811898D0F8B000F1
:101D640049F20031C0F20101884200F06D811898F7
:101D7400D0F8B0004AF20031C0F20101884200F00C
:101D840063811898D0F8B0004BF20031C0F2010121
:101D9400884200F059811898D0F8B0004CF2003114
:101DA400C0F20101884200F04F811898D0F8B000C9
:101DB4004DF20031C0F20101884200F045811898CB
:101DC400D0F8B0004EF20031C0F20101884200F0B8
:101DD4003B811898D0F8B0004FF20031C0F20101F5
:101DE400884200F031811898D0F8B00040F20031F8
:101DF400C0F20201884200F027811898D0F8B000A0
:101E040041F20031C0F20201884200F01D811898AD
:101E1400D0F8B00042F20031C0F20201884200F072
:101E240013811898D0F8B00043F20031C0F20201D7
:101E3400884200F009811898D0F8B00044F20031CB
:101E4400C0F20201884200F0FF801898D0F8B00078
:101E540045F20031C0F20201884200F0F580189882
:101E6400D0F8B00046F20031C0F20201884200F01E
:101E7400EB801898D0F8B00047F20031C0F20201AC
:101E8400884200F0E1801898D0F8B00048F20031A0
:101E9400C0F20201884200F0D7801898D0F8B00050
:101EA40049F20031C0F20201884200F0CD80189856
:101EB400D0F8B0004AF20031C0F20201884200F0CA
:101EC400C3801898D0F8B0004BF20031C0F2020180
:101ED400884200F0B9801898D0F8B0004CF2003174
:101EE400C0F20201884200F0AF801898D0F8B00028
:101EF4004DF20031C0F20201884200F0A58018982A
:101F0400D0F8B0004EF20031C0F20201884200F075
:101F14009B801898D0F8B0004FF20031C0F2020153
:101F2400884200F091801898D0F8B00040F2003157
:101F3400C0F20301884200F087801898D0F8B000FE
:101F440041F20031C0F2030188427DD01898D0F8E4
:101F5400B00042F20031C0F20301884274D01898F4
:101F6400D0F8B00043F20031C0F2030188426BD0D4
:101F74001898D0F8B00044F20031C0F2030188424E
:101F840062D01898D0F8B00045F20031C0F20301D5
:101F9400884259D01898D0F8B00046F20031C0F207
:101FA4000301884250D01898D0F8B00047F20031AD
:101FB400C0F20301884247D01898D0F8B00048F224
:101FC4000031C0F2030188423ED01898D0F8B00026
:101FD40049F20031C0F20301884235D01898D0F894
:101FE400B0004AF20031C0F2030188422CD01898A4
:101FF400D0F8B0004BF20031C0F20301884223D084
:102004001898D0F8B0004CF20031C0F203018842B5
:102014001AD01898D0F8B0004DF20031C0F2030184
:10202400884211D01898D0F8B0004EF20031C0F2B6
:102034000301884208D01898D0F8B0004FF200315C
:10204400C0F20301884200D107E041F67640C0F6B1
:10205400020040F27D3102F09EFD44F60001C5F617
:102064000201086840F48070086014F038FD16908E
:1020740044F60000C5F602000068C00500280AD432
:1020840014F02DFD1699401A652803D303208DF80A
:10209400570000E0ECE79DF85700002875D144F2A2
:1020A4007040C5F60200006800F440701899D1F839
:1020B400B01001F44071884211D044F27041C5F669
:1020C4000201086820F440701790086840F48030DA
:1020D4000860086820F48030086017980860189831
:1020E400D0F8B000B0F5807F17D114F0F8FC16904A
:1020F40044F27040C5F602000068C0F3400060B9C5
:1021040014F0EDFC1699401A41F28931884203D348
:1021140003208DF8570000E0EAE79DF8570078BBEC
:102124001898D0F8B00000F44070B0F5407F12D198
:1021340044F21041C5F60201086820F47C50189A54
:10214400D2F8B0204FF6F043C0F6FF731A4040EACD
:102154001210086007E044F21041C5F60201086855
:1021640020F47C5008601898D0F8B0206FF31F3228
:1021740044F27041C5F6020108681043086003E0A8
:102184009DF857008DF8560003E09DF857008DF830
:10219400560018980068C007002800F04780189877
:1021A400806F0A9028282BD80A99DFE801F01529B6
:1021B40029292929292916292929292929291E29A9
:1021C4002929292929292629292929292929272980
:1021D400292929292929280015E0189808300121DE
:1021E40007F042FE8DF857000DE0189828300121C1
:1021F40007F091FF8DF8570005E004E003E002E0EA
:1022040001208DF857009DF8570058B944F2544105
:10221400C5F60201086820F03800189A926F10433E
:10222400086003E09DF857008DF856001898007870
:102234008007002834D51898406F0990052819D8CC
:102244000999DFE801F003040C14151615E0189839
:102254000830012107F008FE8DF857000DE01898AA
:102264002830012107F057FF8DF8570005E004E0FE
:1022740003E002E001208DF857009DF8570058B99B
:1022840044F25441C5F60201086820F00700189A88
:10229400526F1043086003E09DF857008DF8560014
:1022A400189800784007002836D51898D0F8900080
:1022B4000890052819D80899DFE801F003040C14E4
:1022C400151615E018980830012107F0CDFD8DF89A
:1022D40057000DE018982830012107F01CFF8DF8F5
:1022E400570005E004E003E002E001208DF8570008
:1022F4009DF8570060B944F25841C5F602010868D8
:1023040020F00700189AD2F890201043086003E0E8
:102314009DF857008DF8560018980078800600281C
:1023240044D51898D0F88C000790A0B10798B0F164
:10233400805F11D00798B0F1005F15D00798B0F115
:10234400405F19D00798B0F1804F16D00798B0F1CC
:10235400A04F13D013E015E018980830002107F0BF
:1023640083FD8DF857000DE018982830022107F0FE
:10237400D2FE8DF8570005E004E003E002E00120FE
:102384008DF857009DF8570060B944F25441C5F6E2
:102394000201086820F0E040189AD2F88C2010431B
:1023A400086003E09DF857008DF8560018980078EF
:1023B4004006002844D51898D0F898000690A0B19B
:1023C4000698B0F5806F11D00698B0F5006F15D05F
:1023D4000698B0F5406F19D00698B0F5805F16D016
:1023E4000698B0F5A05F13D013E015E018980830F4
:1023F400002107F039FD8DF857000DE018982830BA
:10240400022107F088FE8DF8570005E004E003E0A0
:1024140002E001208DF857009DF8570060B944F29E
:102424005841C5F60201086820F4E050189AD2F821
:1024340098201043086003E09DF857008DF856007B
:10244400189800780006002844D51898D0F89C0005
:102454000590A0B10598B0F5005F11D00598B0F5CE
:10246400804F15D00598B0F5C04F19D00598B0F538
:10247400004F16D00598B0F5204F13D013E015E0A7
:1024840018980830002107F0EFFC8DF857000DE094
:1024940018982830022107F03EFE8DF8570005E019
:1024A40004E003E002E001208DF857009DF8570096
:1024B40060B944F25841C5F60201086820F460404E
:1024C400189AD2F89C201043086003E09DF8570046
:1024D4008DF85600189800780007002839D5189808
:1024E400D0F88000B0F5805F0FD01898D0F8800045
:1024F400B0F5005F09D01898D0F8800028B118987A
:10250400D0F88000B0F5405F00D107E041F6764096
:10251400C0F6020040F2FC4102F03DFB1898D0F8EE
:102524008000B0F5805F08D118982830022107F0A8
:10253400F2FD10B101208DF8560044F25441C5F665
:102544000201086820F44050189AD2F88020104301
:10255400086018980078C006002839D51898D0F873
:102564009400B0F5807F0FD01898D0F89400B0F59F
:10257400007F09D01898D0F8940028B11898D0F8A2
:102584009400B0F5407F00D107E041F67640C0F6F4
:1025940002004FF4A46102F0FEFA1898D0F89400F7
:1025A400B0F5807F08D118982830022107F0B3FDD8
:1025B40010B101208DF8560044F25841C5F60201CD
:1025C400086820F44070189AD2F8942010430860E8
:1025D400189880780007002835D51898D0F8A000FE
:1025E400049040B10498B0F5803F0CD00498B0F545
:1025F400003F10D010E018980830002107F034FC98
:102604008DF857000BE018982830022107F083FD5D
:102614008DF8570003E002E001208DF857009DF883
:10262400570060B944F25841C5F60201086820F425
:102634004030189AD2F8A0201043086003E09DF8B7
:1026440057008DF85600189880784007002838D530
:102654001898D0F884000390B0F5801F08D0039830
:10266400B0F5001F0DD00398B0F5401F11D011E054
:1026740044F22C41C5F60201086840F400300860B9
:102684000BE018982830012107F045FD8DF857001C
:1026940003E002E001208DF857009DF8570060B96F
:1026A40044F25441C5F60201086820F44010189A17
:1026B400D2F884201043086003E09DF857008DF899
:1026C400560018988078C007002840D01898006DEC
:1026D40020B11898006DB0F5803F00D107E041F6B5
:1026E4007640C0F6020040F2865102F054FA18987F
:1026F400006D029020B10298B0F5803F09D010E03F
:1027040044F22C41C5F60201086840F40030086028
:102714000AE018980830022107F0A6FB8DF857004C
:1027240002E001208DF857009DF8570058B944F293
:102734004C41C5F60201086820F48030189A126DE5
:102744001043086003E09DF857008DF85600189870
:10275400C0788006002808D518982830022107F090
:10276400DAFC10B101208DF85600189880788007A3
:10277400002832D51898C06F0190B8B10198B0F50F
:10278400807F08D00198B0F5007F0DD00198B0F596
:10279400407F0AD00BE044F22C41C5F602010868E0
:1027A40040F40030086005E004E003E002E00120AA
:1027B4008DF857009DF8570058B944F25441C5F6B6
:1027C4000201086820F44070189AD26F1043086020
:1027D40003E09DF857008DF8560018988078C006DD
:1027E40000281BD51898006F20B11898006FB0F11D
:1027F400004F00D107E041F67640C0F6020040F2F7
:10280400E55102F0C8F944F25041C5F602010868E6
:1028140020F00040189A126F1043086018988078CE
:10282400800600281BD51898806E20B11898806EF9
:10283400B0F1807F00D107E041F67640C0F6020097
:1028440040F2F95102F0A7F944F25041C5F60201F1
:10285400086820F08070189A926E104308601898E7
:10286400C0784006002820D51898D0F8B40028B1C4
:102874001898D0F8B400B0F5004F00D107E041F645
:102884007640C0F6020040F20F6102F084F944F28F
:102894001041C5F60201086820F400400860189849
:1028A400D0F8B4200868104308601898C07800066F
:1028B400002820D51898406D48B11898406DB0F1A3
:1028C400805F04D01898406DB0F1005F00D107E03C
:1028D40041F67640C0F6020040F2196102F05BF95D
:1028E40044F24C41C5F60201086820F04050189AA1
:1028F400526D10430860189880780006002824D58B
:102904001898D0F8880058B11898D0F88800B0F515
:10291400800F05D01898D0F88800B0F5000F00D1CA
:1029240007E041F67640C0F6020040F2236102F06F
:1029340032F944F25441C5F60201086820F440001B
:10294400189AD2F888201043086018980079C007B4
:1029540070B118980830002107F086FA8DF85700F6
:102964009DF8570000B903E09DF857008DF8560014
:1029740018980079800700280ED51898083001218E
:1029840007F072FA8DF857009DF8570000B903E07C
:102994009DF857008DF856001898007940070028D4
:1029A4000ED518980830022107F05EFA8DF857000A
:1029B4009DF8570000B903E09DF857008DF85600C4
:1029C40018980079000700280ED51898283000219F
:1029D40007F0A1FB8DF857009DF8570000B903E0FC
:1029E4009DF857008DF8560018980079C006002805
:1029F4000ED518982830012107F08DFB8DF857006B
:102A04009DF8570000B903E09DF857008DF8560073
:102A140018980079800600280ED5189828300221CD
:102A240007F079FB8DF857009DF8570000B903E0D3
:102A34009DF857008DF856009DF8560018B90020EF
:102A44008DF8670002E001208DF867009DF86700AB
:042A54001AB080BD77
:102A580088B0079044F22840C5F60200016801F0EA
:102A6800030106910068C0F30510059044F22C405C
:102A7800C5F60200006800F001000490049844F2D2
:102A88003441C5F60201096889B2C908484300EE15
:102A9800100AB8EE400A8DED020A0598002800F0E9
:102AA80012810698009038B10098012863D00098E8
:102AB800022800F08480A6E044F20040C5F6020037
:102AC8000068C0F3401090B344F20040C5F602001D
:102AD8000068C0F3C10149F20000C0F2D030C8401C
:102AE80003909DED030AB8EE400A9DED051AB8EE75
:102AF800411A80EE010A44F23040C5F6020000682F
:102B08006FF35F2001EE100AB8EE411A9DED022A1C
:102B18009FED723A82EE032A31EE021AB7EE002ACE
:102B280031EE021A20EE010A8DED010A22E09DED38
:102B3800050AB8EE401A9FED6B0A80EE010A44F2CE
:102B48003040C5F6020000686FF35F2001EE100AFE
:102B5800B8EE411A9DED022A9FED603A82EE032AF3
:102B680031EE021AB7EE002A31EE021A20EE010AFF
:102B78008DED010A6AE09DED050AB8EE401A9FED59
:102B8800580A80EE010A44F23040C5F60200006897
:102B98006FF35F2001EE100AB8EE411A9DED022A8C
:102BA8009FED4E3A82EE032A31EE021AB7EE002A62
:102BB80031EE021A20EE010A8DED010A46E09DED84
:102BC800050AB8EE401A9FED440A80EE010A44F265
:102BD8003040C5F6020000686FF35F2001EE100A6E
:102BE800B8EE411A9DED022A9FED3C3A82EE032A87
:102BF80031EE021AB7EE002A31EE021A20EE010A6F
:102C08008DED010A22E09DED050AB8EE401A9FED10
:102C1800350A80EE010A44F23040C5F60200006829
:102C28006FF35F2001EE100AB8EE411A9DED022AFB
:102C38009FED2A3A82EE032A31EE021AB7EE002AF5
:102C480031EE021A20EE010A8DED010A9DED010A0E
:102C580044F23040C5F60200016889B2490A01EE23
:102C6800101AB8EE411AB7EE002A31EE021A80EEB9
:102C7800010A0799BCEEC00A81ED000A9DED010A20
:102C88000168C1F3064101EE101AB8EE411A31EE9F
:102C9800021A80EE010A0799BCEEC00A81ED010A0A
:102CA8009DED010A0068C0F3066001EE100AB8EE57
:102CB800411A31EE021A80EE010A0798BCEEC00AEA
:102CC80080ED020A06E0079900200860079948602D
:102CD8000799886008B0704720BCBE4B00000046CA
:082CE8000024744A0024744C1E
:102CF00088B0079044F22840C5F60200016801F050
:102D0000030106910068C0F30530059044F22C40A1
:102D1000C5F602000068C0F300100490049844F265
:102D20003C41C5F60201096889B2C908484300EE72
:102D3000100AB8EE400A8DED020A0598002800F04E
:102D400012810698009038B10098012863D000984D
:102D5000022800F08480A6E044F20040C5F602009C
:102D60000068C0F3401090B344F20040C5F6020082
:102D70000068C0F3C10149F20000C0F2D030C84081
:102D800003909DED030AB8EE400A9DED051AB8EEDA
:102D9000411A80EE010A44F23840C5F6020000688C
:102DA0006FF35F2001EE100AB8EE411A9DED022A82
:102DB0009FED723A82EE032A31EE021AB7EE002A34
:102DC00031EE021A20EE010A8DED010A22E09DED9E
:102DD000050AB8EE401A9FED6B0A80EE010A44F234
:102DE0003840C5F6020000686FF35F2001EE100A5C
:102DF000B8EE411A9DED022A9FED603A82EE032A59
:102E000031EE021AB7EE002A31EE021A20EE010A64
:102E10008DED010A6AE09DED050AB8EE401A9FEDBE
:102E2000580A80EE010A44F23840C5F602000068F4
:102E30006FF35F2001EE100AB8EE411A9DED022AF1
:102E40009FED4E3A82EE032A31EE021AB7EE002AC7
:102E500031EE021A20EE010A8DED010A46E09DEDE9
:102E6000050AB8EE401A9FED440A80EE010A44F2CA
:102E70003840C5F6020000686FF35F2001EE100ACB
:102E8000B8EE411A9DED022A9FED3C3A82EE032AEC
:102E900031EE021AB7EE002A31EE021A20EE010AD4
:102EA0008DED010A22E09DED050AB8EE401A9FED76
:102EB000340A80EE010A44F23840C5F60200006888
:102EC0006FF35F2001EE100AB8EE411A9DED022A61
:102ED0009FED2A3A82EE032A31EE021AB7EE002A5B
:102EE00031EE021A20EE010A8DED010A9DED010A74
:102EF00044F23840C5F60200016889B2490A01EE81
:102F0000101AB8EE411AB7EE002A31EE021A80EE1E
:102F1000010A0799BCEEC00A81ED000A9DED010A85
:102F20000168C1F3064101EE101AB8EE411A31EE04
:102F3000021A80EE010A0799BCEEC00A81ED010A6F
:102F40009DED010A0068C0F3066001EE100AB8EEBC
:102F5000411A31EE021A80EE010A0798BCEEC00A4F
:102F600080ED020A06E00799002008600799486092
:102F70000799886008B0704720BCBE4B000000462F
:082F80000024744A0024744C83
:102F880088B0079044F22840C5F60200016801F0B5
:102F9800030106910068C0F30550059044F22C40E7
:102FA800C5F602000068C0F300200490049844F2BB
:102FB8004441C5F60201096889B2C908484300EED0
:102FC800100AB8EE400A8DED020A0598002800F0B4
:102FD80012810698009038B10098012863D00098B3
:102FE800022800F08480A6E044F20040C5F6020002
:102FF8000068C0F3401090B344F20040C5F60200E8
:103008000068C0F3C10149F20000C0F2D030C840E6
:1030180003909DED030AB8EE400A9DED051AB8EE3F
:10302800411A80EE010A44F24040C5F602000068E9
:103038006FF35F2001EE100AB8EE411A9DED022AE7
:103048009FED723A82EE032A31EE021AB7EE002A99
:1030580031EE021A20EE010A8DED010A22E09DED03
:10306800050AB8EE401A9FED6B0A80EE010A44F299
:103078004040C5F6020000686FF35F2001EE100AB9
:10308800B8EE411A9DED022A9FED603A82EE032ABE
:1030980031EE021AB7EE002A31EE021A20EE010ACA
:1030A8008DED010A6AE09DED050AB8EE401A9FED24
:1030B800580A80EE010A44F24040C5F60200006852
:1030C8006FF35F2001EE100AB8EE411A9DED022A57
:1030D8009FED4E3A82EE032A31EE021AB7EE002A2D
:1030E80031EE021A20EE010A8DED010A46E09DED4F
:1030F800050AB8EE401A9FED440A80EE010A44F230
:103108004040C5F6020000686FF35F2001EE100A28
:10311800B8EE411A9DED022A9FED3C3A82EE032A51
:1031280031EE021AB7EE002A31EE021A20EE010A39
:103138008DED010A22E09DED050AB8EE401A9FEDDB
:10314800340A80EE010A44F24040C5F602000068E5
:103158006FF35F2001EE100AB8EE411A9DED022AC6
:103168009FED2A3A82EE032A31EE021AB7EE002AC0
:1031780031EE021A20EE010A8DED010A9DED010AD9
:1031880044F24040C5F60200016889B2490A01EEDE
:10319800101AB8EE411AB7EE002A31EE021A80EE84
:1031A800010A0799BCEEC00A81ED000A9DED010AEB
:1031B8000168C1F3064101EE101AB8EE411A31EE6A
:1031C800021A80EE010A0799BCEEC00A81ED010AD5
:1031D8009DED010A0068C0F3066001EE100AB8EE22
:1031E800411A31EE021A80EE010A0798BCEEC00AB5
:1031F80080ED020A06E007990020086007994860F8
:103208000799886008B0704720BCBE4B0000004694
:083218000024744A0024744CE8
:1032200080B586B004900391029200208DF80700CB
:10323000029888B1029804280ED0029808280BD072
:1032400002980C2808D00298102805D0029814285B
:1032500002D002983C2800D107E041F67000C0F689
:10326000020041F2B30101F098FC03980068602865
:103270001FD00398006870281BD003980068402175
:10328000C0F20101884214D0039800685021C0F2B6
:10329000010188420DD0039800686021C0F201014D
:1032A000884206D0039800687021C0F2010188426C
:1032B00000D107E041F67000C0F6020041F2B4010F
:1032C00001F06BFC0398806818B1039880680228AD
:1032D00000D107E041F67000C0F6020041F2B501EE
:1032E00001F05BFC0398006918B103980069042899
:1032F00000D107E041F67000C0F6020041F2B601CD
:1033000001F04BFC049890F83C00012803D1022006
:103310008DF8170048E20499012081F83C000298DA
:103320000090142800F235820099DFE811F01500B2
:10333000320232023202A30032023202320212019F
:103340003202320232027001320232023202CF0104
:103350003202320232020002049800680021C4F2F4
:103360000101884264D004980068B0F1804F5FD0BA
:103370000498006840F20041C4F20001884257D02E
:103380000498006840F60001C4F2000188424FD062
:103390000498006840F60041C4F20001884247D01A
:1033A0000498006840F20041C4F2010188423FD015
:1033B0000498006841F60001C4F20001884237D049
:1033C0000498006841F60041C4F2000188422FD001
:1033D0000498006842F20001C4F20001884227D03C
:1033E0000498006844F20001C4F2010188421FD031
:1033F0000498006844F20041C4F20101884217D0E9
:103400000498006844F60001C4F2010188420FD01C
:10341000049800684EF20001C4F20001884207D00F
:10342000049800684EF20041C4F20001884200D1C5
:1034300007E041F67000C0F602004FF4865101F03B
:10344000ACFB04980068039909F034FB0498016808
:10345000886940F00800886104980168886920F054
:103460000400886103980269049801688869104320
:10347000886191E1049800680021C4F2010188424A
:1034800044D004980068B0F1804F3FD004980068A1
:1034900040F20041C4F20001884237D0049800682D
:1034A00040F60001C4F2000188422FD00498006861
:1034B00040F60041C4F20001884227D00498006819
:1034C00040F20041C4F2010188421FD00498006814
:1034D00041F60001C4F20001884217D00498006848
:1034E00044F20001C4F2010188420FD00498006840
:1034F0004EF20001C4F20001884207D0049800682F
:103500004EF20041C4F20001884200D107E041F6CA
:103510007000C0F6020041F2D10101F03EFB0498B8
:103520000068039916F057FF04980168886940F411
:103530000060886104980168886920F4806088616F
:103540000398026904980168886940EA022088614A
:1035500022E1049800680021C4F20101884234D0BD
:1035600004980068B0F1804F2FD00498006840F2B2
:103570000041C4F20001884227D00498006840F658
:103580000001C4F2000188421FD00498006840F690
:103590000041C4F20001884217D00498006840F24C
:1035A0000041C4F2010188420FD0049800684EF235
:1035B0000001C4F20001884207D0049800684EF26E
:1035C0000041C4F20001884200D107E041F67000DA
:1035D000C0F6020041F2E20101F0DFFA049800684F
:1035E000039909F036FB04980168C86940F00800A7
:1035F000C86104980168C86920F00400C861039894
:10360000026904980168C8691043C861C4E004985D
:1036100000680021C4F20101884234D00498006897
:10362000B0F1804F2FD00498006840F20041C4F2FE
:103630000001884227D00498006840F60001C4F2D7
:10364000000188421FD00498006840F60041C4F28F
:103650000001884217D00498006840F20041C4F28B
:10366000010188420FD0049800684EF20001C4F2B4
:103670000001884207D0049800684EF20041C4F26D
:103680000001884200D107E041F67000C0F6020058
:1036900041F2F30101F081FA04980068039909F0FE
:1036A000B1FB04980168C86940F40060C8610498DF
:1036B0000168C86920F48060C861039802690498B1
:1036C0000168C86940EA0220C86165E004980068A2
:1036D0000021C4F20101884207D00498006840F23A
:1036E0000041C4F20101884200D107E041F67000B8
:1036F000C0F6020041F2041101F04FFA049800688C
:10370000039916F042FF04980168486D40F00800E4
:10371000486504980168486D20F0040048650398E6
:10372000026904980168486D1043486534E00498C4
:1037300000680021C4F20101884207D004980068A3
:1037400040F20041C4F20101884200D107E041F695
:103750007000C0F6020041F2151101F01EFA049843
:103760000068039909F0C7FB04980168486D40F4AC
:103770000060486504980168486D20F480604865E1
:103780000398026904980168486D40EA0220486580
:1037900002E001208DF807000499002081F83C0028
:1037A0009DF807008DF817009DF8170006B080BD42
:1037B00080B584B08DF80E0002919DF80E00014690
:1037C0000191052821D80199DFE801F003070B12C8
:1037D000171B029818F021FF1BE0029818F053FF06
:1037E00017E00298007818F084FF8DF80F0013E0BE
:1037F0000EF0F1FA029908700BE0029818F0A3FF9E
:1038000007E0029818F0B3FF03E0FF208DF80F00E7
:1038100002E000208DF80F009DF90F0004B080BD7C
:1038200080B582B046F6DC60C2F2004090F900003C
:10383000062803D105208DF8070069E146F6DF6010
:10384000C2F20040017840F2034000EB01200EF08C
:1038500022F8222809D046F6DF60C2F20040007844
:103860000221442200230DF00DF901208DF80500FE
:1038700019F0B3FE8DF8060046F6DC60C2F2004097
:1038800090F9000001460091042800F23D81009962
:10389000DFE801F003154184C60046F6C661C2F2B6
:1038A00000410020087048708870C87019F081F8D5
:1038B00046F6DC61C2F200410120087024E19DF867
:1038C0000600022822D141F6F610C0F6020012F0DE
:1038D000D1F842F2B440C2F2004001680A7C46F6D8
:1038E000C661C2F200410A700268527C4A700268E6
:1038F000927C8A700068C07CC87019F05EFA46F647
:10390000DC61C2F200410220087003E00EF0BEFA52
:103910008DF80500F8E09DF80600052826D141F64F
:103920009F70C0F6020012F0A5F81AF090F870B17E
:1039300046F64470C2F20040006880471AF0D5F89D
:1039400046F6DC61C2F20041032008700DE01AF077
:10395000CCF846F64070C2F200400068804746F658
:10396000DC61C2F200410020087016E09DF80600FC
:1039700006280ED141F6C650C0F6020012F07AF8C1
:103980001AF0B3F846F6DC61C2F20041012008707B
:1039900003E00EF07BFA8DF80500B5E004208DF809
:1039A000050046F63870C2F2004000680130B0B33E
:1039B00046F63870C2F20040016842F2D040C2F2CE
:1039C00000400068B0EB510F29D941F6DC50C0F639
:1039D000020012F04FF800208DF8060046F6C6608F
:1039E000C2F20040027846F6BE61C2F200410A709F
:1039F00042784A7082788A70C078C87042F2E44196
:103A0000C2F2004108680130086019F0D6F91AF0D6
:103A10006CF846F6DC61C2F200410420087073E0E5
:103A200004208DF805009DF80600052854D146F6BF
:103A3000DD61C2F200410020087046F6BE60C2F2AD
:103A40000040007846F6C661C2F20041097888421B
:103A500023D146F6BE60C2F20040407846F6C66109
:103A6000C2F200414978884217D146F6BE60C2F2E0
:103A70000040807846F6C661C2F2004189788842EB
:103A80000BD146F6BE60C2F20040C07846F6C66171
:103A9000C2F20041C97888420FD003208DF805009A
:103AA00046F63C70C2F200400068804741F60D20A7
:103AB000C0F6020011F0DEFF05E042F25430C0F61D
:103AC000020011F0D7FF1AF010F846F6DC61C2F2DE
:103AD00000410320087016E09DF8060006280ED16C
:103AE00041F6B470C0F6020011F0C4FF19F0FDFFFA
:103AF00046F6DC61C2F200410120087003E00EF0DE
:103B0000C5F98DF80500FFE79DF805008DF8070061
:083B10009DF8070002B080BD22
:103B180085B0ADF81200BDF8122045F2BA71C0F6B2
:103B2800010141F28220C0F60200B2F5805FB8BF01
:103B3800084603900398811C03910088ADF80A0099
:103B4800BDF80A0028B1BDF81200BDF80A10884275
:103B580000DA6FE00398811C03910088ADF8080033
:103B68009DF80900ADF806009DF80800ADF80800BA
:103B7800BDF81200BDF80A10BDF8082011448842AB
:103B88004EDABDF8060001460091082847D800998A
:103B9800DFE801F005101B21272D33393F0003987A
:103BA800BDF81210BDF80A20891A30F81100ADF8D6
:103BB800120034E0BDF81200BDF80A10411A01F0F5
:103BC8000101401AADF8120029E0BDF812001038C2
:103BD800ADF8120023E0BDF812002038ADF812004D
:103BE8001DE0BDF812003038ADF8120017E0BDF83E
:103BF80012001A38ADF8120011E0BDF812000830B2
:103C0800ADF812000BE0BDF812005038ADF8120004
:103C180005E0BDF81200A0F5E350ADF8120009E088
:103C2800BDF8060028B9BDF80810039800EB41005C
:0C3C380003907FE7BDF8120005B0704754
:103C440080B58EB08DF836008DF835100C920120B9
:103C54008DF82F0046F67470C2F200400078C00759
:103C640018B103208DF8370034E09DF83500014683
:103C74000191032827D80199DFE801F00206101A00
:103C840000208DF82F0021E002A81AF03CF80898D3
:103C94000C99086000208DF82F0017E002A81AF094
:103CA40032F809980C99088000208DF82F000DE057
:103CB40002A81AF028F80998400A0C990860002014
:103CC4008DF82F0002E004208DF82F009DF82F00BE
:0C3CD4008DF837009DF837000EB080BD61
:103CE000DFF80C00016841F47001016070470000CA
:043CF00088ED00E07B
:103CF40008480068006880F308884FF0000080F3EB
:103D0400148862B661B6BFF34F8FBFF36F8F00DFC5
:083D140000BF000008ED00E013
:103D1C0080B58EB042F24040C2F20040006807A964
:103D2C00002210F017FB002800F0A4800798B0F1D7
:103D3C00FF3F14DC07A804300290029848B94FF0FA
:103D4C00500080F31188BFF36F8FBFF34F8F0D902E
:103D5C00FEE702990A68486889689047FFE7079868
:103D6C00002800F18680099806900698406920B1D9
:103D7C00069804301BF00BFCFFE705A81CF057FB62
:103D8C00039007980190092800F273800199DFE8ED
:103D9C0001F0050505373F5E0505373F069991F89B
:103DAC00280040F0010081F828000698089B8169E2
:103DBC001944039A1CF05BFB08B30698016A884708
:103DCC00069890F828004007002817D506980899FF
:103DDC0082690A44694600230B6019461CF083FB78
:103DEC000490049848B94FF0500080F31188BFF349
:103DFC006F8FBFF34F8F0C90FEE7FFE7FFE738E0C4
:103E0C00069991F8280000F0FE0081F8280030E0B7
:103E1C00069991F8280040F0010081F828000898D4
:103E2C00069988610698806948B94FF0500080F374
:103E3C001188BFF36F8FBFF34F8F0B90FEE706987F
:103E4C00039B816919441A461CF011FB11E006987A
:103E5C0090F828008007002803D406980FF0BAFBCE
:103E6C0006E0069991F8280000F0FE0081F8280081
:083E7C00FFE74FE70EB080BD27
:103E8400281F020800000000342100246000000004
:103E940000000024000800001800000000000000DA
:043EA400000000001A
:103EA800AFEE01083BEF01084FEF0108EBEF010807
:043EB800453C00087D
:103EBC00034C206804348047FBE712F07CF8FEE7E3
:043ECC00E8240208DC
:103ED0000A15C90241EA5051C00241F0004140F2C6
:103EE0001E439A1A08DA20320DD4D141D0404840FE
:103EF0009140D14048407047202A28BF202231FA03
:103F000002F0002170476FF000010846704700BFC3
:103F1000F9B140F23D42B1FA81F3D21AC3F1200C5B
:103F200030FA0CFC9840994051EA0C0183054FEAA5
:103F3000D02040EA41504FEAD12101EB025138BF75
:103F40007047013041F100011B4208BF20F0010021
:103F5000704748B140F21D42B0FA80F3D21A98403F
:0C3F6000C10A400501EB0251704700BF90
:103F6C00002B35D129B9B0FBF2FC0CFB12026046D8
:103F7C007047914215D22DE9F041B2FA82F39A4082
:103F8C009940D3F1200C30FA0CFC51EA0C0198400A
:103F9C0000F04EF8280036FA03F200210023BDE8A9
:103FAC00F081F0B5B1FBF2FC0CFB1211B2FA82F30A
:103FBC009A409940D3F1200630FA06F631439840E6
:103FCC0000F036F8614628003200DA400023F0BDDC
:103FDC00F3B5B3FA83FC49085FEA300013FA0CF32B
:103FEC00DCF1200432FA04F423430CB41A0000F080
:103FFC001FF80CBC33FA0CF3DCF11F0C35FA0CF582
:10400C0018BF013D03BCA5FB026705FB0377801BB2
:10401C00B941904271EB030C05D3821A71EB030387
:10402C00681C0021F0BD02000B0028000021F0BD2F
:10403C00940D4FF6C2752D02B5FBF4F4D60A013679
:10404C0004FB04F5A5FB0656F64306EB04165508CF
:10405C0032BF00277708013505FB1677A6FB07470B
:10406C007F0807EBC63714001500E7FB02457F1BE2
:10407C004D1C0400E7FB014505FB1206A64284BF5C
:10408C00013DB618964224BF0135B61A704700BFE1
:10409C000246F0B44FF00137FB0151F8044BE51B1D
:1040AC00A5431D4002D142F8044BF6E70439F0BC9D
:1040BC0011F8013B02F8013B002BF9D1704700BF0E
:1040CC005AB3844690EA01039B071FD1830707D09C
:1040DC0011F8013B00F8013B013AF7D11CE0844692
:1040EC00203A09D32DE9F007B1E8F807A0E8F80762
:1040FC00203AF9D2BDE8F0071C3205D451F8043B44
:10410C0040F8043B043AF9D2043205D011F8013BD3
:0C411C0000F8013B013AF9D16046704701
:1041280000220B0011001A0084465AB3830704D0FA
:1041380000F8011B013AF9D124E0C9B241EA012192
:1041480041EA0141202A11D3203A2DE9F0030B4618
:104158000C460D460E460F4688468946A0E8FA03E7
:10416800203AFBD2BDE8F00320320BD0042A05D355
:1041780040F8041B043A05D0042AF9D200F8011BC0
:08418800013AFBD160467047CB
:104190006B1602088B160208155C010897160208B8
:1041A0008B160208155C0108075C01083716020827
:1041B000261F02084621020846210208462102085D
:1041C000462102084621020846210208462102082B
:1041D0004621020846210208FFFFFFFFFFFFFFFF05
:1041E000FFFFFFFFFFFF0000EA1E0208F8200208A1
:1041F000191B020815210208701B0208E62002089C
:08420000EF200208771B020801
:1042080080B598B0179116901698179980F4807019
:104218000843002840F0978044F25040C5F6020059
:10422800006800F007000B900B980890042800F233
:1042380086800899DFE801F00314257D360044F2F2
:104248000040C5F6020000688001002805D513A8C3
:10425800FEF7FEFB14980C9001E000200C9070E033
:1042680044F20040C5F6020000680001002805D5A8
:1042780010A8FEF739FD10980C9001E000200C9072
:104288005FE044F20040C5F60200006880000028A4
:1042980005D50DA8FEF774FE0D980C9001E00020DE
:1042A8000C904EE044F24C40C5F60200006800F065
:1042B80040500A9044F20040C5F6020000684007EA
:1042C80000280FD50A9868B944F20040C5F60200E4
:1042D8000068C0F3C10149F20000C0F2D030C84004
:1042E8000C9025E044F20040C5F602000068C005C5
:1042F800002809D50A98B0F1805F05D140F6001072
:10430800C0F23D000C9013E044F20040C5F60200F4
:1043180000688003002809D50A98B0F1005F05D12C
:1043280047F64000C0F27D100C9001E000200C9090
:1043380007E048F20000C0F2BB000C9001E000204A
:104348000C9000F023BC1698179980F480600843FD
:10435800002840F09F8044F25840C5F602000068EB
:1043680000F460000B900B98079080B10798B0F5A7
:10437800001F1DD00798B0F5800F2AD00798B0F518
:10438800C00F7ED00798B0F5000F33D07FE044F21D
:104398000040C5F6020000688001002805D513A872
:1043A800FEF756FB14980C9001E000200C9070E08A
:1043B80044F20040C5F6020000680001002805D557
:1043C80010A8FEF791FC10980C9001E000200C90CA
:1043D8005FE044F20040C5F6020000688000002853
:1043E80005D50DA8FEF7CCFD0D980C9001E0002036
:1043F8000C904EE044F24C40C5F60200006800F014
:1044080040500A9044F20040C5F602000068400798
:1044180000280FD50A9868B944F20040C5F6020092
:104428000068C0F3C10149F20000C0F2D030C840B2
:104438000C9025E044F20040C5F602000068C00573
:10444800002809D50A98B0F1805F05D140F6001020
:10445800C0F23D000C9013E044F20040C5F60200A3
:1044680000688003002809D50A98B0F1005F05D1DB
:1044780047F64000C0F27D100C9001E000200C903F
:1044880007E048F20000C0F2BB000C9001E00020F9
:104498000C907BE31698179980F400600843002875
:1044A80040F09F8044F25840C5F60200006800F0D2
:1044B800E0600B900B98069080B10698B0F1807F71
:1044C8001DD00698B0F1007F2AD00698B0F1407F41
:1044D8007ED00698B0F1806F33D07FE044F2004080
:1044E800C5F6020000688001002805D513A8FEF76C
:1044F800AFFA14980C9001E000200C9070E044F2A0
:104508000040C5F6020000680001002805D510A883
:10451800FEF7EAFB10980C9001E000200C905FE099
:1045280044F20040C5F6020000688000002805D566
:104538000DA8FEF725FD0D980C9001E000200C90C9
:104548004EE044F24C40C5F60200006800F04050CE
:104558000A9044F20040C5F60200006840070028AF
:104568000FD50A9868B944F20040C5F60200006801
:10457800C0F3C10149F20000C0F2D030C8400C902D
:1045880025E044F20040C5F602000068C005002896
:1045980009D50A98B0F1805F05D140F60010C0F245
:1045A8003D000C9013E044F20040C5F6020000689C
:1045B8008003002809D50A98B0F1005F05D147F6B5
:1045C8004000C0F27D100C9001E000200C9007E044
:1045D80048F20000C0F2BB000C9001E000200C90F3
:1045E800D4E21698179980F480500843002840F0C8
:1045F8009F8044F25040C5F60200006800F4E04095
:1046080009900998059080B10598B0F5805F1DD094
:104618000598B0F5005F2AD00598B0F5405F7ED0C8
:104628000598B0F5804F33D07FE044F20040C5F6DE
:10463800020000688001002805D513A8FEF708FAD3
:1046480014980C9001E000200C9070E044F20040B7
:10465800C5F6020000680001002805D510A8FEF77D
:1046680043FB10980C9001E000200C905FE044F2AE
:104678000040C5F6020000688000002805D50DA896
:10468800FEF77EFC0D980C9001E000200C904EE0A7
:1046980044F24C40C5F60200006800F040500A9011
:1046A80044F20040C5F602000068400700280FD514
:1046B8000A9868B944F20040C5F602000068C0F3E1
:1046C800C10149F20000C0F2D030C8400C9025E08A
:1046D80044F20040C5F602000068C005002809D56C
:1046E8000A98B0F1805F05D140F60010C0F23D0095
:1046F8000C9013E044F20040C5F602000068800305
:10470800002809D50A98B0F1005F05D147F64000A6
:10471800C0F27D100C9001E000200C9007E048F2F8
:104728000000C0F2BB000C9001E000200C902DE2CC
:104738001698179980F400500843002840F08480A8
:1047480044F25040C5F60200006800F4E0200990E9
:1047580009980490A0B10498B0F5803F14D004984B
:10476800B0F5003F21D00498B0F5403F2ED0049812
:10477800B0F5802F43D00498B0F5A02F50D060E05A
:1047880005F04AFB0C905EE044F20040C5F60200DA
:1047980000680001002805D510A8FEF7A5FA1198B1
:1047A8000C9001E000200C904DE044F20040C5F66A
:1047B800020000688000002805D50DA8FEF7E0FB80
:1047C8000E980C9001E000200C903CE044F2004070
:1047D800C5F602000068400700280DD544F20040E5
:1047E800C5F602000068C0F3C10149F20000C0F23A
:1047F800D030C8400C9001E000200C9023E044F237
:104808000040C5F602000068C005002805D540F63E
:104818000010C0F23D000C9001E000200C9012E066
:1048280044F20040C5F6020000688003002805D560
:1048380047F64000C0F27D100C9001E000200C907B
:1048480001E000200C90A1E11698179980F400204F
:104858000843002840F0808044F25840C5F6020022
:10486800006800F4403009900998039040B103981B
:10487800B0F5803F15D00398B0F5003F22D068E02E
:1048880044F20040C5F6020000680001002805D582
:1048980010A8FEF729FA10980C9001E000200C905F
:1048A80059E044F20040C5F6020000688000002884
:1048B80005D50DA8FEF764FB0F980C9001E00020C9
:1048C8000C9048E044F24C40C5F60200006800F045
:1048D80040500A9044F20040C5F6020000684007C4
:1048E80000280FD50A9868B944F20040C5F60200BE
:1048F8000068C0F3C10149F20000C0F2D030C840DE
:104908000C9025E044F20040C5F602000068C0059E
:10491800002809D50A98B0F1805F05D140F600104B
:10492800C0F23D000C9013E044F20040C5F60200CE
:1049380000688003002809D50A98B0F1005F05D106
:1049480047F64000C0F27D100C9001E000200C906A
:1049580001E000200C9019E11698179980F4803036
:104968000843A0BB44F24C40C5F60200006800F4BE
:10497800803009900998029020B10298B0F5803FE4
:1049880011D021E044F20040C5F602000068800121
:10499800002805D513A8FEF75BF814980C9001E0E1
:1049A80000200C9012E044F20040C5F602000068B6
:1049B8000001002805D510A8FEF796F912980C906A
:1049C80001E000200C9001E000200C90DEE0169839
:1049D800179980F480400843002840F0848044F20E
:1049E8005840C5F60200006800F0E04009900998B8
:1049F8000190A0B10198B0F1805F14D00198B0F196
:104A0800005F21D00198B0F1405F2ED00198B0F13D
:104A1800804F43D00198B0F1A04F50D060E005F02E
:104A2800D3FC0C905EE044F20040C5F6020000683A
:104A38000001002805D510A8FEF756F911980C902A
:104A480001E000200C904DE044F20040C5F6020061
:104A580000688000002805D50DA8FEF791FA0E9889
:104A68000C9001E000200C903CE044F20040C5F6B8
:104A780002000068400700280DD544F20040C5F642
:104A880002000068C0F3C10149F20000C0F2D03052
:104A9800C8400C9001E000200C9023E044F2004054
:104AA800C5F602000068C005002805D540F60010CC
:104AB800C0F23D000C9001E000200C9012E044F29E
:104AC8000040C5F6020000688003002805D547F6B7
:104AD8004000C0F27D100C9001E000200C9001E035
:104AE80000200C9052E01698179980F40040084373
:104AF800002849D144F25040C5F60200006800F091
:104B0800405009900998009040B10098B0F1805F3A
:104B180015D00098B0F1005F22D032E044F2004096
:104B2800C5F6020000688003002805D547F6400056
:104B3800C0F27D100C9001E000200C9023E044F2BC
:104B48000040C5F6020000688001002805D513A8BA
:104B5800FDF77EFF14980C9001E000200C9012E005
:104B680044F20040C5F6020000680001002805D59F
:104B780010A8FEF7B9F811980C9001E000200C90ED
:104B880001E000200C9001E000200C900C9818B077
:024B980080BDDE
:0A4B9A0082B00190009102B0704754
:104BA40080B59EB01D9000208DF867001D98406868
:104BB4004BF62041C0F2BE01884200D807E042F221
:104BC4005C20C0F6020040F6E231FFF7E4FF1D98D6
:104BD4008068B0F1805F07D01D98806820B11D986F
:104BE4008068B0F5805F00D107E042F25C20C0F637
:104BF400020040F6E331FFF7CEFF1D98006840F64F
:104C04000041C5F60001884211D11D98C06820B149
:104C14001D98C068B0F5005F00D107E042F25C2047
:104C2400C0F6020040F6E631FFF7B5FF2BE01D9811
:104C3400C068B0F5805F0CD01D98C06848B11D985D
:104C4400C068B0F5405F04D01D98C068B0F5005F3F
:104C540000D107E042F25C20C0F6020040F6EA31DF
:104C6400FFF799FF1D98006A20B11D98006AB0F5FE
:104C7400006F00D107E042F25C20C0F6020040F66B
:104C8400EB31FFF788FF1D98006948B11D98006952
:104C9400B0F5806F04D01D980069B0F5C06F00D1E5
:104CA40007E042F25C20C0F6020040F6EE31FFF766
:104CB40072FF1D9840696FF00C01084203D11D98E2
:104CC400406900B107E042F25C20C0F6020040F601
:104CD400EF31FFF760FF1D98806970B11D988069FE
:104CE400B0F5807F09D01D988069B0F5007F04D0AD
:104CF4001D988069B0F5407F00D107E042F25C2046
:104D0400C0F602004FF43F61FFF745FF1D98C069EC
:104D140020B11D98C069B0F5004F00D107E042F200
:104D24005C20C0F6020040F6F131FFF734FF1D9815
:104D3400406A58B31D98406A012827D01D98406ADC
:104D4400022823D01D98406A03281FD01D98406A6A
:104D540004281BD01D98406A052817D01D98406A66
:104D6400062813D01D98406A07280FD01D98406A62
:104D740008280BD01D98406A092807D01D98406A5E
:104D84000A2803D01D98406A0B2800D107E042F29C
:104D94005C20C0F6020040F6F231FFF7FCFE1D99DC
:104DA40088680B694A69C9691843104308431C9011
:104DB4001D980068006846F6F311CCF6FF710840B0
:104DC4001C9908431D99096808601D98006840688B
:104DD40020F440501D9A1168D268104348601D9811
:104DE40080691C901D98006840F60041C5F60001DA
:104DF400884204D01D98016A1C9808431C901D9891
:104E0400006880684FF2FF41C1F2FF1108401C990D
:104E140008431D99096888601D980068C06A20F0DD
:104E24000F001D9A1168526A1043C8621D980068E9
:104E340041F20001C4F20101884240F03F8044F293
:104E44005440C5F60200006800F038000146109195
:104E540028282FD81099DFE801F0152D2D2D2D2DA0
:104E64002D2D192D2D2D2D2D2D2D1D2D2D2D2D2D92
:104E74002D2D212D2D2D2D2D2D2D252D2D2D2D2D72
:104E84002D2D290001208DF86D0016E004208DF8E9
:104E94006D0012E008208DF86D000EE010208DF8F2
:104EA4006D000AE020208DF86D0006E040208DF8AA
:104EB4006D0002E080208DF86D004DE21D980068C1
:104EC40044F20041C4F2000188422CD144F254401F
:104ED400C5F60200006800F0070001460F9105289E
:104EE4001DD80F99DFE801F003070B0F13170020FB
:104EF4008DF86D0016E004208DF86D0012E0082096
:104F04008DF86D000EE010208DF86D000AE0202071
:104F14008DF86D0006E040208DF86D0002E08020E1
:104F24008DF86D0018E21D98006844F60001C4F283
:104F3400000188422CD144F25440C5F602000068B6
:104F440000F0070001460E9105281DD80E99DFE8F0
:104F540001F003070B0F131700208DF86D0016E006
:104F640004208DF86D0012E008208DF86D000EE02D
:104F740010208DF86D000AE020208DF86D0006E009
:104F840040208DF86D0002E080208DF86D00E3E193
:104F94001D98006844F60041C4F2000188422CD1F7
:104FA40044F25440C5F60200006800F007000146D0
:104FB4000D9105281DD80D99DFE801F003070B0FAB
:104FC400131700208DF86D0016E004208DF86D0095
:104FD40012E008208DF86D000EE010208DF86D00B1
:104FE4000AE020208DF86D0006E040208DF86D0069
:104FF40002E080208DF86D00AEE11D98006845F256
:105004000001C4F2000188422CD144F25440C5F698
:105014000200006800F0070001460C9105281DD825
:105024000C99DFE801F003070B0F131700208DF82C
:105034006D0016E004208DF86D0012E008208DF854
:105044006D000EE010208DF86D000AE020208DF830
:105054006D0006E040208DF86D0002E080208DF8A0
:105064006D0079E11D98006841F20041C4F201012C
:10507400884240F03F8044F25440C5F60200006884
:1050840000F0380001460B9128282FD80B99DFE84F
:1050940001F0152D2D2D2D2D2D2D192D2D2D2D2DD1
:1050A4002D2D1D2D2D2D2D2D2D2D212D2D2D2D2D48
:1050B4002D2D252D2D2D2D2D2D2D290001208DF863
:1050C4006D0016E004208DF86D0012E008208DF8C4
:1050D4006D000EE010208DF86D000AE020208DF8A0
:1050E4006D0006E040208DF86D0002E080208DF810
:1050F4006D0031E11D98006847F60001C4F200011B
:1051040088422CD144F25440C5F60200006800F0F5
:10511400070001460A9105281DD80A99DFE801F025
:1051240003070B0F131700208DF86D0016E0042001
:105134008DF86D0012E008208DF86D000EE010204F
:105144008DF86D000AE020208DF86D0006E0402007
:105154008DF86D0002E080208DF86D00FCE01D9854
:10516400006847F60041C4F2000188422CD144F2A1
:105174005440C5F60200006800F00700014609919A
:1051840005281DD80999DFE801F003070B0F131751
:1051940000208DF86D0016E004208DF86D0012E0FB
:1051A40008208DF86D000EE010208DF86D000AE0E7
:1051B40020208DF86D0006E040208DF86D0002E09F
:1051C40080208DF86D00C7E01D98006841F600014D
:1051D400C4F20101884240F03F8044F25440C5F6D5
:1051E4000200006800F038000146089128282FD8F2
:1051F4000899DFE801F0152D2D2D2D2D2D2D192DBC
:105204002D2D2D2D2D2D1D2D2D2D2D2D2D2D212DE6
:105214002D2D2D2D2D2D252D2D2D2D2D2D2D2900F3
:1052240001208DF86D0016E004208DF86D0012E069
:1052340008208DF86D000EE010208DF86D000AE056
:1052440020208DF86D0006E040208DF86D0002E00E
:1052540080208DF86D007FE01D98006841F60041C4
:10526400C4F20101884240F03F8044F25440C5F644
:105274000200006800F038000146079128282FD862
:105284000799DFE801F0152D2D2D2D2D2D2D192D2C
:105294002D2D2D2D2D2D1D2D2D2D2D2D2D2D212D56
:1052A4002D2D2D2D2D2D252D2D2D2D2D2D2D290063
:1052B40001208DF86D0016E004208DF86D0012E0D9
:1052C40008208DF86D000EE010208DF86D000AE0C6
:1052D40020208DF86D0006E040208DF86D0002E07E
:1052E40080208DF86D0037E01D98006840F600417D
:1052F400C5F6000188422CD144F25840C5F602009C
:10530400006800F007000146069105281DD806999B
:10531400DFE801F003070B0F131702208DF86D006F
:1053240016E004208DF86D0012E008208DF86D0061
:105334000EE010208DF86D000AE020208DF86D003D
:1053440006E040208DF86D0002E080208DF86D00AD
:1053540002E080208DF86D001D98006840F6004141
:10536400C5F60001884240F09E809DF86D0001461C
:10537400059102280FD00598042810D00598082814
:1053840013D00598102816D0059820282FD00598FA
:10539400402832D035E005F019F8119036E015A810
:1053A400FDF7A4FC1698119030E012A8FDF7EAFD71
:1053B400139811902AE044F20040C5F602000068F8
:1053C400C0F3401068B144F20040C5F60200006822
:1053D400C0F3C10149F20000C0F2D030C8401190BE
:1053E40004E049F20000C0F2D03011900EE040F623
:1053F4000010C0F23D00119008E04FF400401190FD
:1054040004E00020119001208DF867001198002815
:1054140048D011981D994A6A41F26A11C0F60201F6
:1054240031F81210B0FBF1F0189018981D994968E2
:1054340001EB4101884205D318981D994968B0EBE6
:10544400013F03D901208DF867002BE011981D99C5
:105454004A6803924A6A41F26A11C0F6020131F8BD
:105464001220002304931946FEF77EFD039A049B41
:10547400090241EA1061000210EB520041F10001FF
:10548400FEF772FD1A901A98B0F5407F07D31A9868
:10549400000D20B91A981D990968C86002E001201E
:1054A4008DF867002DE11D98C069B0F5004F40F0FC
:1054B4009C809DF86D0001460291402800F25E80B8
:1054C4000299DFE801F021255B5B295B5B5B2F5BC5
:1054D4005B5B5B5B5B5B355B5B5B5B5B5B5B5B5B3E
:1054E4005B5B5B5B5B5B515B5B5B5B5B5B5B5B5B12
:1054F4005B5B5B5B5B5B5B5B5B5B5B5B5B5B5B5BF8
:105504005B5B5B5B5B5B570004F088FC11903AE0EB
:1055140004F097FC119036E015A8FDF7E7FB169808
:10552400119030E012A8FDF72DFD139811902AE098
:1055340044F20040C5F602000068C0F3401068B1B0
:1055440044F20040C5F602000068C0F3C10149F20C
:105554000000C0F2D030C840119004E049F20000CD
:10556400C0F2D03011900EE040F60010C0F23D00C1
:10557400119008E04FF40040119004E000201190D5
:1055840001208DF86700119870B311981D9A516825
:10559400536A41F26A12C0F6020232F81320B0FBD9
:1055A400F2F0400000EB5100B0FBF1F01A901A98B1
:1055B400102816D3BDF86A0098B91A9820F00F0085
:1055C400ADF86E001A9800F00E01BDF86E0040EAC6
:1055D4005100ADF86E00BDF86E001D990968C860F1
:1055E40002E001208DF867008BE09DF86D00014614
:1055F4000191402800F25E800199DFE801F0212545
:105604005B5B295B5B5B2F5B5B5B5B5B5B5B355B6A
:105614005B5B5B5B5B5B5B5B5B5B5B5B5B5B515BE0
:105624005B5B5B5B5B5B5B5B5B5B5B5B5B5B5B5BC6
:105634005B5B5B5B5B5B5B5B5B5B5B5B5B5B570015
:1056440004F0ECFB11903AE004F0FBFB119036E01F
:1056540015A8FDF74BFB1698119030E012A8FDF742
:1056640091FC139811902AE044F20040C5F6020020
:105674000068C0F3401068B144F20040C5F602006F
:105684000068C0F3C10149F20000C0F2D030C84044
:10569400119004E049F20000C0F2D03011900EE005
:1056A40040F60010C0F23D00119008E04FF40040B5
:1056B400119004E00020119001208DF867001198EA
:1056C400F8B111981D9A5168536A41F26A12C0F6F2
:1056D400020232F81320B0FBF2F000EB5100B0FBF1
:1056E400F1F01A901A98102808D3BDF86A0028B966
:1056F400BDF868001D990968C86002E001208DF8B2
:1057040067001D990120A1F86A001D99A1F868009D
:105714001D99002048671D9988679DF867001EB091
:0257240080BD46
:1057260080B586B069460020086040F20002C2F2E9
:10573600000240F23C03C2F200030A2006210EF0EA
:1057460054FA014642F2D440C2F2004001600068B9
:1057560028B941F63170C0F6020010F088F96946A2
:105766000020086040F28C02C2F2000240F2B4034C
:10577600C2F200030A2004210EF037FA014642F273
:10578600B840C2F200400160006828B941F64E7088
:10579600C0F6020010F06BF941F29B00C0F6020061
:1057A60043F68462C0F600020021049119F0F8FC69
:1057B600049B42F2BC41C2F20041086040F2043050
:1057C600C2F200006946886040F20410C2F200008E
:1057D60048601920086041F21B00C0F6020041F63D
:1057E6006B71C0F6020180221AF094F905900598B3
:1057F60048B941F2B660C0F6020041F66B71C0F6D8
:10580600020110F034F942F26430C2F20000694637
:10581600886040F26430C2F20000486019200860D7
:1058260040F6E760C0F6020042F25411C0F60201EB
:105836004FF4006200231AF06DF90590059848B9F7
:1058460041F2B660C0F6020042F25411C0F60201FF
:1058560010F00DF943F2C430C2F2000069468860C8
:1058660042F2C430C2F2000048601920086041F2DA
:10587600FF00C0F6020042F25C11C0F602014FF4CE
:10588600806200231AF046F90590059848B941F25E
:10589600B660C0F6020042F25C11C0F6020110F0DA
:1058A600E6F843F22460C2F200006946886043F2DB
:1058B6002440C2F2000048601920086045F2E54025
:1058C600C0F6010041F2C961C0F602018022002340
:1058D6001AF020F90590059848B941F2B660C0F66D
:1058E600020041F2C961C0F6020110F0C0F843F6A9
:1058F6008400C2F200006946886043F28460C2F206
:10590600000048601920086045F23370C0F60100B7
:1059160041F68631C0F60201802200231AF0FAF819
:105926000590059848B941F2B660C0F6020041F606
:0E5936008631C0F6020110F09AF806B080BD6E
:1059440080B586B08DF81600049100208DF80F0004
:10595400029001909DF81600014600910F2800F274
:105964007F800099DFE801F0080B1E1923287C7C56
:105974002D474A4E52535A6B0CF039F974E004988F
:1059840020B1049801900198043002900198029982
:1059940016F087FC8DF8170069E00498008816F06B
:1059A40056FD61E016F07BFD049908805CE00498E4
:1059B400008816F09EFD57E016F0C1FD049908809A
:1059C40052E046F6E060C2F200408178049A117019
:1059D400C178049A51700179049A91704179049ABA
:1059E400D1708179049A1171C0790499487104992C
:1059F4000020887138E00CF039F935E0049816F08D
:105A0400C8FD31E004980CF04EF92DE02CE0049828
:105A140000780CF07BF98DF8170028E00CF0BDF944
:105A24008DF80F009DF90F00013018B9FF208DF893
:105A340017001CE09DF80F000499087014E00CF0A6
:105A4400B7F98DF80F009DF90F00013018B9FF2048
:105A54008DF817000BE09DF80F000499087003E01F
:105A6400FF208DF8170002E000208DF817009DF943
:065A7400170006B080BD22
:105A7A0080B588B0002002900790069005900490A7
:105A8A0000F061FE0298012101918DF810108DF845
:105A9A00110005901F228DF8182087228DF81920F1
:105AAA008DF81A008DF81B008DF81C108DF81D104A
:105ABA008DF81E008DF81F0004A8039011F0AEF8AF
:105ACA00019A029903988DF811204FF0105305930B
:105ADA0010238DF818308DF819108DF81A2003222A
:105AEA008DF81B208DF81D1011F098F8042011F084
:065AFA007DF808B080BD3C
:105B000010B58EB08DF833000B91ADF82A2000202F
:105B1000ADF82200ADF820009DF8331040F20340AC
:105B200000EB01200BF0B7FE014605911C2800F2A6
:105B3000F1800599DFE811F0DD00EE00EE00EE00E7
:105B4000EE00EE00EE00EE00EE00EE00EE00EE00E5
:105B5000EE00EE00EE00EE00EE00EE00EE00C800FB
:105B6000EE00EE00EE001D00EE00EE00EE00EE0096
:105B7000B5009DF8331040F2024000EB01200BF01D
:105B80008AFEC007002841D09DF8331040F20C4037
:105B900000EB012007A904220BF041FF9DF8331010
:105BA0004FF4826000EB01200BF075FE04909DF82D
:105BB000331040F2114000EB01200BF06CFE049911
:105BC00040EA0120ADF81A009DF833109DF81C2022
:105BD0009DF81D309DF81E009DF81FE0BDF81A408D
:105BE000EC46CCF80840CCF804E0CCF8000041F6D4
:105BF0000C60C0F602000FF03DFF9DF8331040F23C
:105C0000024000EB012001210BF0F8FD9DF833006C
:105C100016F093F8ADF82200012841DBBDF8220010
:105C2000B0F5006F03DD4FF40060ADF822009DF881
:105C300033000B99BDF822200BF089F909900998DF
:105C4000002802DC09980D9066E00998ADF8220062
:105C50000020ADF82000BDF82200BDF820108842D9
:105C60001ED09DF833000B99BDF820301944BDF8C3
:105C70002220D21A92B20BF069F809900998B0F17B
:105C8000FF3F06DC9DF8330015F057FF09980D9093
:105C900042E00999BDF820000844ADF82000DAE799
:105CA00038E09DF833000AF0E4FF0990012802D0A3
:105CB00009980D9030E09DF8331041F63720C0F67A
:105CC00002000FF0D7FE25E09DF83310BDF82A2022
:105CD00042F26830C0F602000FF0CCFE9DF83300AF
:105CE00015F08BFF0990012802D009980D9013E060
:105CF00010E09DF83300BDF82A20012100230AF0AE
:105D0000C1FE09909DF83310884202D009980D9089
:0E5D100002E0FFE701200D900D980EB010BDCF
:105D1E0080B59EB00BA84C21FEF7FFF90020019034
:105D2E000A900990089007900690059004900390B1
:105D3E00022012F039FE0020029044F61800C5F63B
:105D4E0002000168022262F38F310160006800F4E4
:105D5E0040400290029844F61800C5F60200006812
:105D6E0000F40050B0F5005F00D0F4E702F079FEC9
:105D7E0044F27041C5F60201086820F01800086070
:105D8E0005210B914FF480300C9001200D900220D4
:105D9E0014901590169128211791189019901A9019
:105DAE0008201B9000201C901D900BA802F062FE94
:105DBE0008B1FAF7D0FA3F20039003200490002098
:105DCE00059006900790089009900A9003A801216B
:0E5DDE0003F01FFC08B1FAF7BEFA1EB080BD3C
:105DEC0080B584B044F2D440C5F60200016841F09D
:105DFC0001010160006800F001000390039842F279
:105E0C000800C2F2004002904021C5F2002101605E
:105E1C001D214160002181608022C260016140F23D
:105E2C000223436140F6080383612023C3610262AD
:105E3C004FF0007242624FF4006282624FF40052E3
:105E4C00C2624FF4803202634163816302F016FB3D
:105E5C0008B1FAF781FA42F20800C2F200400022BF
:105E6C00114612F02EFC08B1FAF776FA7A2001905E
:105E7C000521002200F01AFC019810F08AFE04B0F3
:025E8C0080BDD7
:105E8E0080B5B0B02F906846B821FEF746F92F982E
:105E9E00006844F20001C5F60001884215D10020C9
:105EAE0001904FF4800000904FF480702C90684663
:105EBE00FBF7C1FB08B1FAF74EFA44F27041C5F692
:0E5ECE000201086840F40040086030B080BD5A
:105EDC0041F63451C2F2004147F20000C5F20020F5
:105EEC000860002048604FF4805088604FF4804078
:0E5EFC00C8604FF40030086102204861704712
:105F0A0080B5BEB03D9000203C903B903A903990CD
:105F1A0038900AA8B821FEF702F93D98006847F2BE
:105F2A000001C5F20021884267D100200B904FF48E
:105F3A0080310A911E900AA8FBF77FFB08B1FAF795
:105F4A000CFA44F2D440C5F60200016841F48031EB
:105F5A000160006800F480300990099844F2E0403A
:105F6A00C5F60200016841F004010160006800F012
:105F7A0004000890089844F2E040C5F6020001685F
:105F8A0041F008010160006800F0080007900798D6
:105F9A004FF4F85038900220019039900020059073
:105FAA003A90032002903B900C2003903C9040F6DC
:105FBA000000C5F6020038A9049101F097FFDDF848
:105FCA0004C0029A03980499059B4FF0040ECDF879
:105FDA00E0E0CDF8E4C03A933B923C9040F60040B2
:105FEA00C5F6020001F082FF059A312006900521CC
:0E5FFA0000F05DFB069810F0CDFD3EB080BDBE
:1060080080B582B041F62440C2F20040009043F2CD
:106018000041C4F2010101604FF4800141604FF476
:10602800C02181600821C1600021019101614161A5
:106038004FF0005282614FF08052C26101624162AA
:106048008162C1624FF0804242638163C16301642F
:1060580041648164C16401654165816505F0DBFBCC
:0A60680008B1FAF77BF902B080BD21
:1060720080B582B044F2F440C5F60200016841F0F6
:1060820002010160006800F00200019001986FF0C7
:0E60920001000F21002200F00EFB02B080BDC5
:1060A00080B590B00E900E980F280FD80E9937201B
:1060B0000090002200F000FB009810F070FD0E9898
:1060C00046F62471C2F20041086003E001208DF819
:1060D0003F0048E044F2E840C5F60200016841F0A4
:1060E00020010160006800F020000190019806A8DE
:1060F00002A912F0B4FC0B980490049818B903F0AC
:106100008FFE059003E003F08BFE4000059005989C
:106110004DF68361C4F21B31A0FB01014FF0FF304B
:1061200000EB9140039042F23020C2F2004041F275
:106130000041C4F20001016040F2E731C1600399FF
:10614000416000210161816005F0FDFE40B942F22D
:106150003020C2F2004014F034F88DF83F0002E025
:0E61600001208DF83F009DF83F0010B080BD7B
:10616E004EF68851CEF20001086840F470000860C7
:10617E0042F20000C5F20020006800F00F00062871
:10618E0008D842F20001C5F200210868072262F326
:10619E000300086044F20041C5F60201086840F0B1
:1061AE000100086044F21042C5F6020200201060A1
:1061BE0008684EF67F52CEF6F6221040086042F284
:1061CE000000C5F20020006800F00F00082808D378
:1061DE0042F20001C5F200210868072262F30300B3
:1061EE00086044F21841C5F602010020086044F22E
:1061FE001C41C5F60201086044F22041C5F60201B9
:10620E00086044F22842C5F6020240F20021C0F2B4
:10621E000221116044F22C42C5F602020021C0F2A6
:10622E00FF11116044F23042C5F6020240F28021A5
:10623E00C0F20111116044F23442C5F60202106040
:10624E0044F23842C5F60202116044F23C42C5F6F1
:10625E000202106044F24042C5F60202116044F29E
:10626E004441C5F60201086044F20042C5F602023E
:10627E00116821F48021116044F26041C5F60201DB
:10628E00086044F20001C5F2002143F2D20008601A
:02629E00704747
:1062A00080B590B0002101910F910E910D910C914C
:1062B0000B910A910991089107910691059104911A
:1062C0000391029142F2C820C2F2004040F2004223
:1062D000C4F2000202600322426081604FF47A72CD
:1062E000C26001618021816105F02DFE08B1FAF7DD
:1062F00039F84FF480500C9042F2C820C2F20040AE
:106300000CA907F04EF908B1FAF72CF842F2C820B0
:10631000C2F2004006F031F808B1FAF723F8002085
:1063200009900B9042F2C820C2F2004009A914F073
:1063300054FA08B1FAF716F860200290C8200390CA
:10634000022004900020069042F2C820C2F20040D1
:1063500002A90422FCF764FF08B1FAF703F842F23D
:0E636000C820C2F2004000F002F810B080BD6C
:10636E0080B588B0079000200690059004900390A9
:10637E0002900798006840F20041C4F20001884282
:10638E001BD144F2E040C5F60200016841F0040161
:10639E000160006800F004000190019880200290D6
:1063AE0002200390002104910591069040F6000012
:0E63BE00C5F6020002A901F097FD08B080BDEF
:1063CC0080B584B0002103910291019142F27C20AE
:1063DC00C2F2004041F20002C4F2000202606322E9
:1063EC00426081604FF6FF71C1608021816105F0D0
:1063FC00A4FD08B1F9F7B0FF00200190039042F220
:10640C007C20C2F2004001A914F0E1F908B1F9F7BF
:06641C00A3FF04B080BDE7
:1064220080B582B041F6FC20C2F20040009044F2F6
:106432000041C4F2000101604FF4E13141600023E8
:1064420001938360C36003610C2141618361C36175
:1064520003624362836219461A4609F057FA08B189
:10646200F9F77FFF41F6FC20C2F20040002109F05B
:106472000CFC08B1F9F775FF41F6FC20C2F20040AE
:10648200002109F0C1FC08B1F9F76BFF41F6FC20CD
:10649200C2F2004009F060FB08B1F9F762FF02B0F6
:0264A20080BDBB
:1064A40080B582B041F66820C2F20040019044F603
:1064B4000001C4F2000101604FF4E13141600021A8
:1064C4008160C16001610C2242618161C16101622C
:1064D4004162282181624FF4004181634FF40051ED
:1064E400016408F058F908B1F9F73AFF41F6682059
:1064F400C2F20040002109F0C7FB08B1F9F730FFF0
:1065040041F66820C2F20040002109F07CFC08B189
:10651400F9F726FF41F66820C2F2004009F01BFBA0
:0A65240008B1F9F71DFF02B080BDB9
:10652E0080B582B041F69030C2F20040009041F644
:10653E000041C4F2010101604FF4E13141600023DA
:10654E0001938360C36003610C2141618361C36168
:10655E0003624362836219461A4609F0D1F908B103
:10656E00F9F7F9FE41F69030C2F20040002109F031
:10657E0086FB08B1F9F7EFFE41F69030C2F200400B
:10658E00002109F03BFC08B1F9F7E5FE41F6903029
:10659E00C2F2004009F0DAFA08B1F9F7DCFE02B0F7
:0265AE0080BDAE
:1065B00080B582B0032000F060F8FAF7CBFE44F219
:1065C0001842C5F602021168C1F3032342F24C21BE
:1065D000C0F60201CB5C03F01F03D8400090009886
:1065E000126802F00F02895C01F01F01C84046F6F4
:1065F0004871C2F200410860009846F64C71C2F240
:10660000004108600F20FFF74BFD18B101208DF805
:10661000070004E0FFF72DFD00208DF807009DF82E
:06662000070002B080BD7E
:1066260046F67370C2F20040027842F28841C2F226
:0A6636000041086810440860704736
:1066400080B584B0039010F04CFA0290039801904A
:106650000198013038B146F67370C2F200400178FB
:1066600001980844019010F03CFA0299401A0199EF
:0A667000884200D2F7E704B080BDB5
:10667A0080B582B00190019807280BD001980628AE
:10668A0008D00198052805D00198042802D001985D
:10669A00032800D106E041F6A230C0F6020091219B
:0E66AA00FEF776FA019810F01DFA02B080BDDE
:1066B80080B586B0ADF816000491039203980F28B0
:1066C80000D806E041F6A230C0F60200A921FEF784
:1066D80060FA04980F2800D806E041F6A230C0F608
:1066E8000200AA21FEF755FA10F01BFA0290BDF934
:1066F8001600019002980499039A10F01AFA0146BC
:0A670800019800F002F806B080BD11
:1067120082B0ADF806000091BDF90600002809D448
:1067220000980001BDF906104EF20042CEF20002BE
:1067320088540AE000980001BDF8061001F00F012C
:0E6742004EF61452CEF20002885402B0704798
:10675000BFF35F8F4EF62451CEF20001086820F49B
:10676000803008604EF69451CEF20001002008609F
:02677000704770
:1067720010B58EB00C9010F0B3F90A900C9820B9B5
:1067820001208DF8370000F0F6BD0C98006810214A
:10679200C4F20201884200F0B8800C9800682821F7
:1067A200C4F20201884200F0B0800C9800684021D7
:1067B200C4F20201884200F0A8800C9800685821B7
:1067C200C4F20201884200F0A0800C980068702197
:1067D200C4F20201884200F098800C980068882177
:1067E200C4F20201884200F090800C980068A02157
:1067F200C4F20201884200F088800C980068B82137
:10680200C4F20201884200F080800C98006840F2D5
:106812001041C4F20201884277D00C98006840F21D
:106822002841C4F2020188426FD00C98006840F2FD
:106832004041C4F20201884267D00C98006840F2DD
:106842005841C4F2020188425FD00C98006840F2BD
:106852007041C4F20201884257D00C98006840F29D
:106862008841C4F2020188424FD00C98006840F27D
:10687200A041C4F20201884247D00C98006840F25D
:10688200B841C4F2020188423FD00C98006845F238
:106892000841C5F60201884237D00C98006845F2DB
:1068A2001C41C5F6020188422FD00C98006845F2BF
:1068B2003041C5F60201884227D00C98006845F2A3
:1068C2004441C5F6020188421FD00C98006845F287
:1068D2005841C5F60201884217D00C98006845F26B
:1068E2006C41C5F6020188420FD00C98006845F24F
:1068F2008041C5F60201884207D00C98006845F233
:106902009441C5F60201884200D106E041F2D4600A
:10691200C0F60200E621FEF73FF90C98806838B114
:106922000C988068402803D00C988068802800D199
:1069320006E041F2D460C0F60200E721FEF72CF92E
:106942000C98C068B0F5007F02D00C98C06800B9FE
:1069520006E041F2D460C0F60200E821FEF71CF91D
:106962000C980069B0F5806F02D00C98006900B9EC
:1069720006E041F2D460C0F60200E921FEF70CF90C
:106982000C98406948B10C984069B0F5006F04D08A
:106992000C984069B0F5805F00D106E041F2D46006
:1069A200C0F60200EA21FEF7F7F80C98806948B1B8
:1069B2000C988069B0F5005F04D00C988069B0F53E
:1069C200804F00D106E041F2D460C0F60200EB2114
:1069D200FEF7E2F80C98C06990B10C98C069B0F566
:1069E200807F0DD00C98C069202809D00C98C0690E
:1069F200B0F5802F04D00C98C069B0F5402F00D1BB
:106A020006E041F2D460C0F60200EC21FEF7C4F8C1
:106A12000C98006A70B10C98006AB0F5803F09D0FA
:106A22000C98006AB0F5003F04D00C98006AB0F5EB
:106A3200403F00D106E041F2D460C0F60200ED21F1
:106A4200FEF7AAF80C98016801201022C4F2020293
:106A52009142079000F091800C9801680120282251
:106A6200C4F202029142079000F087800C980168FC
:106A720001204022C4F20202914207907DD00C987C
:106A8200016801205822C4F202029142079074D098
:106A92000C98016801207022C4F202029142079010
:106AA2006BD00C98016801208822C4F20202914244
:106AB200079062D00C9801680120A022C4F2020261
:106AC2009142079059D00C9801680120B822C4F273
:106AD20002029142079050D00C980168012040F2C6
:106AE2001042C4F202029142079046D00C9801680B
:106AF200012040F22842C4F20202914207903CD0A7
:106B02000C980168012040F24042C4F20202914214
:106B1200079032D00C980168012040F25842C4F22A
:106B220002029142079028D00C980168012040F29D
:106B32007042C4F20202914207901ED00C98016882
:106B4200012040F28842C4F202029142079014D01E
:106B52000C980168012040F2A042C4F20202914264
:106B620007900AD00C9800684FF64831CBF6FD71B9
:106B72000844B0FA80F0400907900798C00700283F
:106B820000F0B1810C984068892800D806E041F2F3
:106B9200D460C0F60200F121FDF7FEFF0C98406AB6
:106BA20018B10C98406A042800D106E041F2D46082
:106BB200C0F60200F221FDF7EFFF0C98406A0028B0
:106BC2004AD00C98806A58B10C98806A012807D084
:106BD2000C98806A022803D00C98806A032800D19E
:106BE20006E041F2D460C0F60200F721FDF7D4FFBF
:106BF2000C98C06A70B10C98C06AB0F5000F09D049
:106C02000C98C06AB0F1807F04D00C98C06AB0F1D1
:106C1200C07F00D106E041F2D460C0F60200F82144
:106C2200FDF7BAFF0C98006B70B10C98006BB0F5D1
:106C3200001F09D00C98006BB0F5800F04D00C989F
:106C4200006BB0F5C00F00D106E041F2D460C0F68F
:106C52000200F921FDF7A0FF0C99022081F835000E
:106C62000C99002081F834000C9800681021C4F2BD
:106C72000201884270D00C9800682821C4F20201F7
:106C8200884269D00C9800684021C4F2020188420F
:106C920062D00C9800685821C4F2020188425BD08D
:106CA2000C9800687021C4F20201884254D00C98FA
:106CB20000688821C4F2020188424DD00C98006815
:106CC200A021C4F20201884246D00C980068B82183
:106CD200C4F2020188423FD00C98006840F2104191
:106CE200C4F20201884237D00C98006840F2284171
:106CF200C4F2020188422FD00C98006840F2404151
:106D0200C4F20201884227D00C98006840F2584130
:106D1200C4F2020188421FD00C98006840F2704110
:106D2200C4F20201884217D00C98006840F28841F0
:106D3200C4F2020188420FD00C98006840F2A041D0
:106D4200C4F20201884207D00C98006840F2B841B0
:106D5200C4F20201884206D10C980168086820F04A
:106D62000100086005E00C980168086820F0010045
:106D720008600C9800680068C00788B10FF0B0FE88
:106D82000A99401A06280AD30C99202048650C99C2
:106D9200032081F8350001208DF83700EBE2E8E7A7
:106DA2000C98006800680B900B9848F23F01CFF6F0
:106DB200106108400B900C998868D1F80CC00B69DF
:106DC2004A6940EA0C00184310438A691043CA69B1
:106DD2001043096A01430B9808430B900C98406AD0
:106DE200042806D10C99C86A096B01430B98084321
:106DF2000B900C984068292805D30C984168012013
:106E02002F2906902CD30C9840683F2805D30C9864
:106E1200416801204329069022D30C9840684728F4
:106E220005D30C98416801204929069018D30C9883
:106E320040684F2805D30C984168012053290690D9
:106E42000ED30C98416800207429059006D30C9843
:106E520041680020782938BF0120059005980690E6
:106E62000698C00718B10B9840F480100B900B984D
:106E72000C99096808600C98006840690B900B989F
:106E820020F007000B900C98416A0B9808430B9076
:106E92000C98406A042815D10C98816A0B98084313
:106EA2000B900C98C06A68B10C98FAF7ECF948B1EB
:106EB2000C99402048650C99012081F835008DF825
:106EC200370058E20B980C99096848610C9800F059
:106ED20056FA09900C98C06D00F01F013F208840BF
:106EE200099988601BE10C980168012045F208426B
:106EF200C5F602029142049046D00C980168012026
:106F020045F21C42C5F60202914204903CD00C9814
:106F12000168012045F23042C5F602029142049016
:106F220032D00C980168012045F24442C5F60202B3
:106F32009142049028D00C980168012045F25842F1
:106F4200C5F60202914204901ED00C9801680120FD
:106F520045F26C42C5F602029142049014D00C989C
:106F62000168012045F28042C5F602029142049076
:106F72000AD00C9800684AF66C31CAF2FD710844D6
:106F8200B0FA80F0400904900498C007002800F08D
:106F9200BB800C980168012045F20842C5F6020246
:106FA2009142039046D00C980168012045F21C42A0
:106FB200C5F60202914203903CD00C980168012070
:106FC20045F23042C5F602029142039032D00C984B
:106FD2000168012045F24442C5F602029142039043
:106FE20028D00C980168012045F25842C5F60202E9
:106FF200914203901ED00C980168012045F26C4228
:10700200C5F602029142039014D00C980168012047
:1070120045F28042C5F60202914203900AD00C98D2
:1070220000684AF66C31CAF2FD710844B0FA80F089
:10703200400903900398C00760B10C98406811287A
:1070420000D807E041F2D460C0F6020040F26B11B2
:10705200FDF7A2FD0C99022081F835000C99002061
:1070620081F834000C98006800680B900B986FF35D
:1070720010100B900C988068402802D110200290CA
:1070820007E00C9880688038B0FA80F040098003ED
:10709200029002980C99CA680B69D1F814C0D1F811
:1070A20018E0CC694EEA040E4CEA0E0C43EA0C03DB
:1070B2001A4340EAD200096A40EA11110B980843C8
:1070C2000B900B980C99096808600C9908684AF6AD
:1070D200F832CAF2FD7210444CF6CD42CCF6CC42E4
:1070E200A0FB02026FF0030000EA9200C8650C9850
:1070F20000F045F908900C98C06D00F01F010120C6
:107102008840089948600AE00C99402048650C992B
:10711200032081F8350001208DF837002BE10C980F
:10712200016801201022C4F202029142019000F093
:10713200EA800C98016801202822C4F202029142DE
:10714200019000F0E0800C98016801204022C4F216
:1071520002029142019000F0D6800C980168012051
:107162005822C4F202029142019000F0CC800C98A5
:10717200016801207022C4F202029142019000F0E3
:10718200C2800C98016801208822C4F20202914256
:10719200019000F0B8800C9801680120A022C4F28E
:1071A20002029142019000F0AE800C980168012029
:1071B200B822C4F202029142019000F0A4800C981D
:1071C2000168012040F21042C4F202029142019091
:1071D20000F099800C980168012040F22842C4F224
:1071E20002029142019000F08E800C980168012009
:1071F20040F24042C4F202029142019000F08380C8
:107202000C980168012040F25842C4F202029142F5
:10721200019078D00C980168012040F27042C4F2CB
:107222000202914201906ED00C980168012040F256
:107232008842C4F202029142019064D00C98016823
:10724200012040F2A042C4F20202914201905AD0BF
:107252000C980168012040F2B842C4F20202914245
:10726200019050D00C980168012045F20842C5F601
:1072720002029142019046D00C980168012045F229
:107282001C42C5F60202914201903CD00C98016862
:10729200012045F23042C5F602029142019032D0FD
:1072A2000C980168012045F24442C5F6020291425F
:1072B200019028D00C980168012045F25842C5F689
:1072C2000202914201901ED00C980168012045F201
:1072D2006C42C5F602029142019014D00C980168EA
:1072E200012045F28042C5F60202914201900AD085
:1072F2000C9800684AF66C31CAF2FD710844B0FA83
:1073020080F0400901900198C00758B30C9800F032
:1073120005F90C988068802802D10C9900204860F9
:107322000C990879096E08600C98416E806E48606D
:107332000C98406878B10C98406808280BD80C98D3
:107342000FF002FE0C98C16E002008600C98016FCD
:10735200406F486006E00C990020C8660C990867E7
:107362000C9948670C99002048650C9A012182F813
:0E73720035108DF837009DF837000EB010BDB5
:1073800083B002900298016801201022C4F2020228
:107390009142009000F0918002980168012028221B
:1073A000C4F202029142009000F0878002980168C6
:1073B00001204022C4F20202914200907DD0029846
:1073C000016801205822C4F202029142009074D058
:1073D0000298016801207022C4F2020291420090DA
:1073E0006BD00298016801208822C4F20202914207
:1073F000009062D0029801680120A022C4F202022B
:107400009142009059D0029801680120B822C4F23C
:1074100002029142009050D002980168012040F28F
:107420001042C4F202029142009046D002980168D4
:10743000012040F22842C4F20202914200903CD066
:1074400002980168012040F24042C4F202029142D7
:10745000009032D002980168012040F25842C4F2F4
:1074600002029142009028D002980168012040F267
:107470007042C4F20202914200901ED0029801684C
:10748000012040F28842C4F202029142009014D0DE
:1074900002980168012040F2A042C4F20202914227
:1074A00000900AD0029800684FF64831CBF6FD7183
:1074B0000844B0FA80F0400900900098C00728B353
:1074C0000298007810384AF6AB21CAF6AA21A0FB30
:1074D000011000090190019800F0070142F27410B8
:1074E000C0F60200405C0299C8650198042806D3E2
:1074F00002990868042262F30900886505E0029990
:10750000086840F2FF329043886504E002990868F9
:0E75100020F0FF0088650298806D03B0704780
:10751E0084B00390039800680190039801680120DD
:10752E0045F20842C5F602029142009046D00398F9
:10753E000168012045F21C42C5F6020291420090FC
:10754E003CD003980168012045F23042C5F6020294
:10755E009142009032D003980168012045F24442D6
:10756E00C5F602029142009028D0039801680120CE
:10757E0045F25842C5F60202914200901ED0039881
:10758E000168012045F26C42C5F60202914200905C
:10759E0014D003980168012045F28042C5F602021C
:1075AE00914200900AD0039800684AF66C31CAF2F4
:1075BE00FD710844B0FA80F0400900900098C007B1
:1075CE0008B30398007808384CF6CD41CCF6CC4180
:1075DE00A0FB011000090290029945F60000C5F6C5
:1075EE00020000EB810003990866039945F68000BE
:1075FE00C5F602004866029800F01F01012088407F
:10760E000399886631E00398007810384AF6AB216A
:10761E00CAF6AA21A0FB011000090290019840F2BF
:10762E00B841C4F20201884209D8019840F21041D3
:10763E00C4F20201884202D30298083002900299E5
:10764E0040F60000C4F2020000EB810003990866C8
:10765E00039940F68000C4F202004866029800F0DA
:0E766E001F01012088400399886604B0704710
:10767C0080B58AB008900FF02EFA0490089820B9C3
:10768C0001208DF8270000F02CBC089890F83500EC
:10769C0002280BD00899802048650899002081F8B1
:1076AC00340001208DF8270000F01BBC08980168FD
:1076BC0001201022C4F202029142039000F091804A
:1076CC000898016801202822C4F20202914203901A
:1076DC0000F087800898016801204022C4F2020261
:1076EC00914203907DD00898016801205822C4F281
:1076FC0002029142039074D0089801680120702214
:10770C00C4F20202914203906BD0089801680120E8
:10771C008822C4F202029142039062D00898016858
:10772C000120A022C4F202029142039059D0089881
:10773C0001680120B822C4F202029142039050D099
:10774C0008980168012040F21042C4F202029142F2
:10775C00039046D008980168012040F22842C4F2F8
:10776C000202914203903CD008980168012040F23B
:10777C004042C4F202029142039032D00898016850
:10778C00012040F25842C4F202029142039028D0E8
:10779C0008980168012040F27042C4F20202914242
:1077AC0003901ED008980168012040F28842C4F270
:1077BC0002029142039014D008980168012040F213
:1077CC00A042C4F20202914203900AD008980068C9
:1077DC004FF64831CBF6FD710844B0FA80F0400901
:1077EC0003900398C00778B108980168086820F0E6
:1077FC001E00086008980168486920F08000486104
:10780C0008980068059008E008980168086820F05E
:10781C000E0008600898006805900898016801201F
:10782C001022C4F202029142029000F0EA80089801
:10783C00016801202822C4F202029142029000F059
:10784C00E0800898016801204022C4F202029142B3
:10785C00029000F0D6800898016801205822C4F2EA
:10786C0002029142029000F0CC800898016801203D
:10787C007022C4F202029142029000F0C280089879
:10788C00016801208822C4F202029142029000F0A9
:10789C00B880089801680120A022C4F2020291422B
:1078AC00029000F0AE80089801680120B822C4F262
:1078BC0002029142029000F0A48008980168012015
:1078CC0040F21042C4F202029142029000F0998000
:1078DC0008980168012040F22842C4F20202914249
:1078EC00029000F08E8008980168012040F240421E
:1078FC00C4F202029142029000F083800898016861
:10790C00012040F25842C4F202029142029078D017
:10791C0008980168012040F27042C4F202029142C0
:10792C0002906ED008980168012040F28842C4F29F
:10793C0002029142029064D008980168012040F242
:10794C00A042C4F20202914202905AD008980168F7
:10795C00012040F2B842C4F202029142029050D08F
:10796C0008980168012045F20842C5F602029142CE
:10797C00029046D008980168012045F21C42C5F6D9
:10798C000202914202903CD008980168012045F215
:10799C003042C5F602029142029032D0089801683A
:1079AC00012045F24442C5F602029142029028D0D1
:1079BC0008980168012045F25842C5F6020291422E
:1079CC0002901ED008980168012045F26C42C5F661
:1079DC0002029142029014D008980168012045F2ED
:1079EC008042C5F60202914202900AD008980068C3
:1079FC004AF66C31CAF2FD710844B0FA80F04009C5
:107A0C0002900298C00728B10898016E086820F40B
:107A1C0080700860089800681021C4F20201884246
:107A2C0070D0089800682821C4F20201884269D0FD
:107A3C00089800684021C4F20201884262D008987C
:107A4C0000685821C4F2020188425BD00898006893
:107A5C007021C4F20201884254D008980068882131
:107A6C00C4F2020188424DD008980068A021C4F2EB
:107A7C000201884246D008980068B821C4F202017D
:107A8C0088423FD00898006840F21041C4F20201CD
:107A9C00884237D00898006840F22841C4F20201AD
:107AAC0088422FD00898006840F24041C4F202018D
:107ABC00884227D00898006840F25841C4F202016D
:107ACC0088421FD00898006840F27041C4F202014D
:107ADC00884217D00898006840F28841C4F202012D
:107AEC0088420FD00898006840F2A041C4F202010D
:107AFC00884207D00898006840F2B841C4F20201ED
:107B0C00884206D108980168086820F001000860D6
:107B1C0005E008980168086820F0010008600598E5
:107B2C000068C007A8B10EF0D6FF0499401A0628C9
:107B3C000ED30899202048650899032081F8350058
:107B4C000899002081F8340001208DF82700C8E145
:107B5C00E5E70898016801201022C4F20202914264
:107B6C00019000F091800898016801202822C4F24D
:107B7C0002029142019000F0878008980168012070
:107B8C004022C4F20202914201907DD00898016813
:107B9C0001205822C4F202029142019074D008983C
:107BAC00016801207022C4F20202914201906BD054
:107BBC000898016801208822C4F2020291420190C7
:107BCC0062D0089801680120A022C4F202029142FE
:107BDC00019059D0089801680120B822C4F2020221
:107BEC009142019050D008980168012040F2104257
:107BFC00C4F202029142019046D00898016801201B
:107C0C0040F22842C4F20202914201903CD0089802
:107C1C000168012040F24042C4F2020291420190FC
:107C2C0032D008980168012040F25842C4F2020296
:107C3C009142019028D008980168012040F27042CE
:107C4C00C4F20202914201901ED0089801680120F2
:107C5C0040F28842C4F202029142019014D008987A
:107C6C000168012040F2A042C4F20202914201904C
:107C7C000AD0089800684FF64831CBF6FD710844DD
:107C8C00B0FA80F0400901900198C00758B10898EB
:107C9C00806D07900898C06D00F01F013F20884050
:107CAC00079988600AE00898806D06900898C06D66
:107CBC0000F01F010120884006994860089801686F
:107CCC0001201022C4F202029142009000F0EA80DE
:107CDC000898016801202822C4F202029142009007
:107CEC0000F0E0800898016801204022C4F20202F2
:107CFC009142009000F0D68008980168012058222B
:107D0C00C4F202029142009000F0CC800898016805
:107D1C0001207022C4F202029142009000F0C28055
:107D2C000898016801208822C4F202029142009056
:107D3C0000F0B880089801680120A022C4F2020269
:107D4C009142009000F0AE80089801680120B822A2
:107D5C00C4F202029142009000F0A48008980168DD
:107D6C00012040F21042C4F202029142009000F055
:107D7C00998008980168012040F22842C4F202025E
:107D8C009142009000F08E8008980168012040F22A
:107D9C004042C4F202029142009000F083800898A5
:107DAC000168012040F25842C4F202029142009054
:107DBC0078D008980168012040F27042C4F20202A7
:107DCC00914200906ED008980168012040F28842E0
:107DDC00C4F202029142009064D00898016801201C
:107DEC0040F2A042C4F20202914200905AD008988C
:107DFC000168012040F2B842C4F2020291420090A4
:107E0C0050D008980168012045F20842C5F60202DC
:107E1C009142009046D008980168012045F21C421E
:107E2C00C5F60202914200903CD0089801680120EE
:107E3C0045F23042C5F602029142009032D00898C9
:107E4C000168012045F24442C5F6020291420090BD
:107E5C0028D008980168012045F25842C5F6020264
:107E6C00914200901ED008980168012045F26C42A6
:107E7C00C5F602029142009014D0089801680120C6
:107E8C0045F28042C5F60202914200900AD0089851
:107E9C0000684AF66C31CAF2FD710844B0FA80F001
:107EAC00400900900098C00780B10898416E806E20
:107EBC0048600898C06E48B10898C16E086820F4F4
:107ECC00807008600898016F406F48600899012025
:107EDC0081F835000899002081F8340000208DF8D5
:0A7EEC0027009DF827000AB080BDB2
:107EF60080B590B00F900E9100200D908020C5F6B1
:107F060000000A900F980021C5F6020188423ED073
:107F16000F9840F20041C5F60201884237D00F980B
:107F260040F60001C5F60201884230D00F9840F6AF
:107F36000041C5F60201884229D00F9841F200019E
:107F4600C5F60201884222D00F9841F20041C5F6DB
:107F5600020188421BD00F9841F60001C5F60201C6
:107F6600884214D00F9841F60041C5F602018842B6
:107F76000DD00F9842F20041C5F60201884206D0A4
:107F86000F9842F60001C5F60201884200D106E0CC
:107F960042F27C10C0F60200B321FCF7FBFD0E98FE
:107FA600008818B10E98408800B906E042F27C10AD
:107FB600C0F60200B421FCF7EDFD0E98406888B3C8
:107FC6000E98406801282DD00E984068112829D0B7
:107FD6000E984068022825D00E984068122821D0B5
:107FE6000E984068B0F5881F1CD00E984068B0F512
:107FF600041F17D00E984068B0F5441F12D00E9893
:108006004068B0F5901F0DD00E984068B0F5081F77
:1080160008D00E984068B0F5481F03D00E98406807
:10802600032800D106E042F27C10C0F60200B5211A
:10803600FCF7B0FD0E9800680D99C840002800F0C6
:108046001E820E9800680D9A0121914008400C90FE
:108056000C98002800F00F820E98406800F003008C
:10806600012805D00E98406800F00300022844D18C
:108076000E98C06858B10E98C068012807D00E98AF
:10808600C068022803D00E98C068032800D106E015
:1080960042F27C10C0F60200C421FCF77BFD0F986B
:1080A60080680B900D984100032000FA01F10B98AF
:1080B60088430B900E98C0680D99490000FA01F1AB
:1080C6000B9808430B900B980F9988600F9840689F
:1080D6000B900D99012000FA01F10B9888430B9043
:1080E6000E984068C0F300100D9900FA01F10B9844
:1080F60008430B900B980F9948600E98406800F063
:108106000300032829D00E98806838B10E9880683D
:10811600012803D00E988068022800D106E042F2BA
:108126007C10C0F60200D621FCF734FD0F98C0681B
:108136000B900D984100032000FA01F10B9888433B
:108146000B900E9880680D99490000FA01F10B9882
:1081560008430B900B980F99C8600E98406800F082
:10816600030002287DD10F980021C5F6020188423E
:108176003ED00F9840F20041C5F60201884237D042
:108186000F9840F60001C5F60201884230D00F98DC
:1081960040F60041C5F60201884229D00F9841F207
:1081A6000001C5F60201884222D00F9841F2004133
:1081B600C5F6020188421BD00F9841F60001C5F6AC
:1081C6000201884214D00F9841F60041C5F602011B
:1081D60088420DD00F9842F20041C5F6020188424E
:1081E60006D00F9842F60001C5F60201884200D17A
:1081F60006E042F27C10C0F60200E321FCF7CAFC5E
:108206000E9800690F2800D806E042F27C10C0F6EE
:108216000200E421FCF7BEFC0F980D996FF00302F3
:1082260002EA51010844006A0B900D9800F007001D
:1082360081000F2000FA01F10B9888430B900E98ED
:1082460000690D9901F00701890000FA01F10B9808
:1082560008430B900B980F990D9B02EA53021144A9
:1082660008620F9800680B900D984100032000FAF1
:1082760001F10B9888430B900E98406800F00300BC
:108286000D99490000FA01F10B9808430B900B98E1
:108296000F9908600E9880798007002800F0EB801F
:1082A60044F2F440C5F60200016841F002010160A3
:1082B600006800F00200099009980D9820F003006C
:1082C60040F20841C5F6000140580B900D9800F0A9
:1082D600030081000F2000FA01F10B9888430B90F0
:1082E6000F980021C5F60201884202D100200890AD
:1082F6005DE00F9840F20041C5F60201884202D1C6
:108306000120079051E00F9840F60001C5F60201E2
:10831600884202D10220069045E00F9840F60041BF
:10832600C5F60201884202D10320059039E00F9874
:1083360041F20001C5F60201884202D104200490F0
:108346002DE00F9841F20041C5F60201884202D1A4
:108356000520039021E00F9841F60001C5F60201C1
:10836600884202D10620029015E00F9841F600419E
:10837600C5F60201884202D10720019009E00F9953
:1083860042F20042C5F602020A20914208BF0920C5
:108396000190019802900298039003980490049823
:1083A60005900598069006980790079808900898F3
:1083B6000D9901F00301890000FA01F10B980843B9
:1083C6000B900B980D9921F0030140F20842C5F677
:1083D600000288504FF0B04000680B900C990B9843
:1083E60088430B900E988079C006002803D50C9917
:1083F6000B9808430B900B984FF0B041086004208F
:10840600C5F6000000680B900C990B9888430B90FA
:108416000E9880798006002803D50C990B9808439E
:108426000B900B980421C5F6000108600A98406875
:108436000B900C990B9888430B900E9880798007C7
:10844600002803D50C990B9808430B900B980A99B2
:1084560048600A9800680B900C990B9888430B901B
:108466000E988079C00718B10C990B9808430B90A9
:108476000B980A9908600D9801300D90DAE510B056
:0284860080BDB7
:1084880080B584B002900EF028FB0190029818B9CC
:1084980001208DF80F005AE2029800684021C5F2C9
:1084A8000021884275D0029800688021C5F2002119
:1084B80088426ED002980068C021C5F20021884227
:1084C80067D00298006840F20011C5F20021884286
:1084D8005FD00298006840F24011C5F2002188423E
:1084E80057D00298006840F28011C5F200218842F6
:1084F8004FD00298006840F2C011C5F200218842AE
:1085080047D00298006840F20021C5F20021884255
:108518003FD00298006840F24021C5F2002188420D
:1085280037D00298006840F28021C5F200218842C5
:108538002FD00298006840F2C021C5F2002188427D
:1085480027D00298006840F20031C5F20021884225
:108558001FD00298006840F24031C5F200218842DD
:1085680017D00298006840F28031C5F20021884295
:108578000FD00298006840F2C031C5F2002188424D
:1085880007D00298006840F20041C5F200218842F5
:1085980000D106E042F2E410C0F60200E521FCF743
:1085A800F8FA0298C06858B10298C068402807D005
:1085B8000298C068802803D00298C068C02800D1FB
:1085C80006E042F2E410C0F60200E621FCF7E1FA08
:1085D8000298006970B102980069B0F5805F09D00F
:1085E80002980069B0F5005F04D002980069B0F500
:1085F800804F00D106E042F2E410C0F60200E72105
:10860800FCF7C7FA02984068B0F1804F03D002988F
:108618004068212800D806E042F2E410C0F60200C3
:10862800E821FCF7B6FA0298406950B3029840690D
:10863800022826D002984069B0F5817F21D002989F
:10864800406940F2022188421BD00298406940F2FA
:108658000231884215D002984069032811D0029847
:10866800406940F2031188420BD00298406940F2F9
:108678000321884205D00298406940F203318842BC
:1086880000D106E042F2E410C0F60200E921FCF74E
:1086980080FA0298806950B302988069082826D029
:1086A80002988069B0F5816F21D00298806940F600
:1086B800080188421BD00298806940F60841884228
:1086C80015D0029880690C2811D00298806940F270
:1086D8000C4188420BD00298806940F60C01884210
:1086E80005D00298806940F60C41884200D106E026
:1086F80042F2E410C0F60200EA21FCF74AFA0298B6
:10870800C06958B10298C069102807D00298C0699A
:10871800202803D00298C069302800D106E042F230
:10872800E410C0F60200EB21FCF733FA0298006A65
:1087380058B10298006A402807D00298006A802839
:1087480003D00298006AC02800D106E042F2E41083
:10875800C0F60200EC21FCF71CFA0298406AB0F15E
:10876800007F0CD00298406A48B10298406AB0F184
:10877800806F04D00298406AB0F1006F00D106E023
:1087880042F2E410C0F60200ED21FCF702FA02986A
:10879800C06A10B30298C06AB0F5805F1DD0029815
:1087A800C06AB0F5005F18D00298C06AB0F5405FA3
:1087B80013D00298C06AB0F5804F0ED00298C06AF4
:1087C800B0F5A04F09D00298C06AB0F5C04F04D0E8
:1087D8000298C06AB0F5E04F00D106E042F2E4101A
:1087E800C0F60200EE21FCF7D4F90298006B10B332
:1087F8000298006BB0F5004F1DD00298006BB0F5E1
:10880800803F18D00298006BB0F5C03F13D0029893
:10881800006BB0F5003F0ED00298006BB0F5203F1A
:1088280009D00298006BB0F5403F04D00298006B65
:10883800B0F5603F00D106E042F2E410C0F6020055
:10884800EF21FCF7A6F90298806A20B10298806AA5
:10885800FE2800D806E042F2E410C0F60200F0213B
:10886800FCF797F90298806870B102988068B0F1B7
:10887800805F09D002988068B0F1005F04D0029848
:108888008068B0F1405F00D106E042F2E410C0F623
:108898000200F121FCF77DF90298406B10F5803F4A
:1088A80005DD0298406BB0F5803F00DA06E042F241
:1088B800E410C0F60200F221FCF76BF90298806B15
:1088C80010F5803F05DD0298806BB0F5803F00DA37
:1088D80006E042F2E410C0F60200F321FCF759F971
:1088E8000299002081F83C000299022081F83D009D
:1088F80002980168C86820F00100C8600298006802
:10890800C068C00788B10EF0E8F80199401A062837
:108918000AD30299402088660299032081F83D0015
:1089280001208DF80F0012E0E8E7029800F013F834
:1089380002990020C865029908660299486602995A
:108948008866029A012182F83D108DF80F009DF883
:068958000F0004B080BD19
:10895E0083B00290029A1168D06812691043C86001
:10896E00029B009319689A685869D3F818C040EAB8
:10897E000C00D3F81CC040EA0C00D3F820C040EA2B
:10898E000C00D3F824C040EA0C00D3F82CC040EA07
:10899E000C00D3F830C040EA0C00D3F828C00023F6
:1089AE00CFF6FC7303EB8C43184310430861029817
:1089BE004068B0F1804F05D102980168086940F017
:1089CE004040086102980168002048610298406B9F
:1089DE00B0F1FF3F0FDC02980168486940F4802037
:1089EE0048610298406B40420190BDF80400029924
:1089FE000968086203E00299888E09680862029885
:108A0E00806BB0F1FF3F11DC02980168486940F4B9
:108A1E00002048610298806B40420190019A0298B2
:108A2E000168086A40EA0240086206E0029801689E
:108A3E00826B086A40EA0240086202984068B0F110
:108A4E00804F04D0029908790968886203E0029881
:108A5E00016800208862029801680020486203B015
:028A6E0070474F
:108A700044F60001C5F60201086840F48070086001
:028A800070473D
:108A820080B58CB00A900A9820B901208DF82F0089
:108A920000F0C1BD0A98006800B30A980078C007C8
:108AA200E0B90A98006800F00200022816D00A987D
:108AB200006800F01000102810D00A98006800F03A
:108AC200080008280AD00A98006800F00400042868
:108AD20004D00A9800788006002800D507E041F209
:108AE2003B70C0F6020040F2A111FCF755F80A985B
:108AF2000078C007002800F0AE800A98406848B1AC
:108B02000A984068B0F5803F04D00A984068B0F5F2
:108B1200A02F00D107E041F23B70C0F602004FF4F3
:108B2200D371FCF739F844F21040C5F60200006830
:108B320000F03800069044F22840C5F602000068B2
:108B420005900698102807D00698182815D1059880
:108B520000F00300022810D144F20040C5F60200E2
:108B62000068C0F3404038B10A98406820B901203B
:108B72008DF82F0000F04FBD6DE00A984068B0F507
:108B8200803F08D144F20041C5F60201086840F472
:108B9200803008602DE00A98406860B944F20041D4
:108BA200C5F60201086820F480300860086820F4E5
:108BB200802008601DE00A984068B0F5A02F0CD113
:108BC20044F20041C5F60201086840F480200860C2
:108BD200086840F4803008600BE044F20041C5F6BA
:108BE2000201086820F480300860086820F48020C0
:108BF20008600A984068B8B10DF072FF099044F21B
:108C02000040C5F602000068C0F3404058B90DF0BC
:108C120067FF0999401A652804D303208DF82F00B5
:108C220000F0F9BCEBE716E00DF05AFF099044F2B0
:108C32000040C5F602000068C0F3404058B10DF094
:108C42004FFF0999401A652804D303208DF82F009D
:108C520000F0E1BCEBE70A9800788007002840F1B9
:108C6200D5800A98C06898B10A98C06801280FD0C8
:108C72000A98C06801280BD00A98C068092807D052
:108C82000A98C068112803D00A98C068192800D130
:108C920007E041F23B70C0F602004FF4ED71FBF7C2
:108CA2007BFF0A9800697F2800D807E041F23B70F9
:108CB200C0F6020040F2DB11FBF76EFF44F21040F7
:108CC200C5F60200006800F03800049044F2284023
:108CD200C5F6020000680390049838B10498182879
:108CE20043D19DF80C00800700283ED144F2004099
:108CF200C5F602000068C0F3800038B10A98C06867
:108D020020B901208DF82F0000F085BC44F200410B
:108D1200C5F60201086820F019000A9AD2681043C9
:108D220008600DF0DDFE099044F20040C5F6020035
:108D32000068C0F3800058B90DF0D2FE0999401ABC
:108D4200032804D303208DF82F0000F064BCEBE766
:108D520044F20441C5F60201086820F0FE400A9A76
:108D6200126940EA0260086050E00A98C06870B375
:108D720044F20041C5F60201086820F019000A9A7F
:108D8200D268104308600DF0ABFE099044F2004037
:108D9200C5F602000068C0F3800058B90DF0A0FECD
:108DA2000999401A032804D303208DF82F0000F0FC
:108DB20032BCEBE744F20441C5F60201086820F038
:108DC200FE400A9A126940EA026008601EE044F21C
:108DD2000041C5F60201086820F0010008600DF0AC
:108DE2007FFE099044F20040C5F602000068C0F31D
:108DF200800058B10DF074FE0999401A032804D37B
:108E020003208DF82F0000F006BCEBE70A980078EB
:108E1200C006002840F19F800A98C06918B10A98DC
:108E2200C069802800D107E041F23B70C0F6020021
:108E320040F22B21FBF7B0FE0A98006A3F2800D8C7
:108E420007E041F23B70C0F602004FF40B71FBF7F2
:108E5200A3FE44F21040C5F60200006800F038009C
:108E6200029044F22840C5F6020000680190029880
:108E7200082807D00298182821D1019800F0030091
:108E820001281CD144F20040C5F602000068C0F37C
:108E9200002038B10A98C069802803D001208DF8DB
:108EA2002F00B8E344F20C41C5F60201086820F035
:108EB2007C500A9A126A40EA026008604BE00A9803
:108EC200C06950B344F20041C5F60201086840F09F
:108ED200800008600DF004FE099044F20040C5F6DF
:108EE20002000068C0F3002050B90DF0F9FD0999A5
:108EF200401A032803D303208DF82F008BE3ECE7FD
:108F020044F20C41C5F60201086820F07C500A9A2E
:108F1200126A40EA026008601DE044F20041C5F6B0
:108F22000201086820F0800008600DF0D9FD099068
:108F320044F20040C5F602000068C0F3002050B1C0
:108F42000DF0CEFD0999401A032803D303208DF8B2
:108F52002F0060E3ECE70A980078000700284FD55D
:108F62000A98406918B10A984069012800D107E0BF
:108F720041F23B70C0F6020040F26D21FBF70CFE9D
:108F82000A984069F0B144F27441C5F602010868DA
:108F920040F0010008600DF0A3FD099044F2744016
:108FA200C5F602000068C0F3400050B90DF098FD0C
:108FB2000999401A032803D303208DF82F002AE3CE
:108FC200ECE71DE044F27441C5F60201086820F0A6
:108FD200010008600DF084FD099044F27440C5F66A
:108FE20002000068C0F3400050B10DF079FD09990C
:108FF200401A032803D303208DF82F000BE3ECE77C
:109002000A980078800600284FD50A98806918B11E
:109012000A988069012800D107E041F23B70C0F64E
:1090220002004FF42671FBF7B7FD0A988069F0B190
:1090320044F20041C5F60201086840F4805008601D
:109042000DF04EFD099044F20040C5F602000068A2
:10905200C0F3403050B90DF043FD0999401A03287E
:1090620003D303208DF82F00D5E2ECE71DE044F294
:109072000041C5F60201086820F4805008600DF036
:109082002FFD099044F20040C5F602000068C0F3CB
:10909200403050B10DF024FD0999401A032803D342
:1090A20003208DF82F00B6E2ECE70A98007840071B
:1090B200002840F1A0800A98806838B10A98806838
:1090C200012803D00A988068052800D107E041F200
:1090D2003B70C0F6020040F2C221FBF75DFD44F690
:1090E2000001C5F60201086840F4807008600DF0C6
:1090F200F7FC099044F60000C5F602000068C005BE
:1091020000280AD40DF0ECFC0999401A652803D313
:1091120003208DF82F007EE2ECE70A988068012890
:1091220008D144F27041C5F60201086840F001001E
:1091320008602CE00A98806860B944F27041C5F674
:109142000201086820F001000860086820F00400AD
:1091520008601CE00A98806805280CD144F270412E
:10916200C5F60201086840F004000860086840F093
:10917200010008600BE044F27041C5F60201086884
:1091820020F001000860086820F0040008600A98D6
:109192008068C0B10DF0A4FC099044F27040C5F69D
:1091A20002000068C0F3400060B90DF099FC099913
:1091B200401A41F28931884203D303208DF82F00EF
:1091C20029E2EAE717E00DF08BFC099044F27040C7
:1091D200C5F602000068C0F3400060B10DF080FCEB
:1091E2000999401A41F28931884203D303208DF84C
:1091F2002F0010E2EAE70A98406A38B10A98406AFA
:10920200012803D00A98406A022800D107E041F2FF
:109212003B70C0F602004FF43D71FBF7BDFC0A98AB
:10922200406A002800F0F48144F21040C5F60200C2
:10923200006800F03800182800F068810A98406A37
:10924200022840F044810A98806A01280AD00A98CC
:10925200806A38B10A98806A032803D00A98806A23
:10926200022800D107E041F23B70C0F6020040F252
:10927200FD21FBF791FC0A98006C58B10A98006C2A
:10928200042807D00A98006C082803D00A98006CBA
:109292000C2800D107E041F23B70C0F6020040F218
:1092A200FE21FBF779FC0A98406C18B10A98406CD1
:1092B200022800D107E041F23B70C0F6020040F202
:1092C200FF21FBF769FC0A98C06A20B10A98C06ABC
:1092D2003F2800D807E041F23B70C0F602004FF48D
:1092E2004071FBF759FC0A98006B042805D30A98D1
:1092F200006BB0F5007F00D807E041F23B70C0F68A
:10930200020040F20131FBF747FC0A98406B20B1A2
:109312000A98406B802800D807E041F23B70C0F603
:10932200020040F20231FBF737FC0A98806B20B151
:109332000A98806B802800D807E041F23B70C0F6A3
:10934200020040F20331FBF727FC0A98C06B20B100
:109352000A98C06B802800D807E041F23B70C0F643
:1093620002004FF44171FBF717FC0A98806C400B26
:1093720000B907E041F23B70C0F6020040F205314D
:10938200FBF70AFC44F20041C5F60201086820F02E
:10939200807008600DF0A4FB099044F20040C5F60D
:1093A20002000068C0F3406050B10DF099FB0999CA
:1093B200401A032803D303208DF82F002BE1ECE79A
:1093C20044F22841C5F60201086840F2F3329043A4
:1093D2000A9B9A6ADB6A42EA0312104308600A99FE
:1093E200086BD1F834C08B6BCA6B01386FF35F2006
:1093F2004FF60061CFF6FF7101EB4C2189B20844B0
:109402000021CFF6FF7101EB034101F4FE01084494
:109412004FF07F4101EB026101F0FE41084444F24A
:109422003041C5F60201086044F22C41C5F6020142
:109432000091086820F00100086044F23442C5F649
:10944200020210684FF6F87398430A9B9B6C40EA3D
:10945200C3001060086820F00C000A9A126C1043D6
:109462000860086820F002000A9A526C10430860F3
:10947200086840F480300860086840F400300860F2
:10948200086840F480200860086840F00100086025
:1094920044F20041C5F60201086840F0807008609D
:1094A2000DF01EFB099044F20040C5F60200006870
:1094B200C0F3406050B90DF013FB0999401A03281C
:1094C20003D303208DF82F00A5E0ECE71DE044F262
:1094D2000041C5F60201086820F0807008600DF0B6
:1094E200FFFA099044F20040C5F602000068C0F39A
:1094F200406050B10DF0F4FA0999401A032803D3E1
:1095020003208DF82F0086E0ECE781E044F228404A
:10951200C5F602000068089044F23040C5F6020029
:10952200006807900A98406A01282DD0089800F038
:1095320003000A99896A884226D10898C0F3051166
:109542000A98C06A88421FD107986FF35F200A9970
:10955200096B0139884217D1BDF81C00410A0A98EB
:10956200406B013888420FD10798C0F306410A9830
:10957200806B0138884207D10798C0F306610A98C8
:10958200C06B0138884203D001208DF82F0042E0E1
:1095920044F23440C5F60200006880B2C008089068
:1095A2000A98806C0899884232D00A98806C400BE5
:1095B20000B907E041F23B70C0F602004FF45B7164
:1095C200FBF7EAFA44F22C41C5F60201086820F0E2
:1095D200010008600DF084FA09900DF081FA0999F2
:1095E200401A00B9F9E744F23441C5F602010868AD
:1095F2004FF6F87290430A9A926C40EAC2000860F1
:1096020044F22C41C5F60201086840F001000860EE
:0E96120000208DF82F009DF82F000CB080BDB9
:1096200080B586B004900391049818B901208DF894
:109630001700C6E30498006820B1049800683F282A
:1096400000D807E041F23B70C0F6020040F2A731BB
:10965000FBF7A3FA039860B30398012829D0039875
:10966000022826D00398032823D00398042820D06A
:10967000039805281DD0039806281AD003980728B8
:1096800017D00398082814D00398092811D00398FC
:109690000A280ED003980B280BD003980C2808D06A
:1096A00003980D2805D003980E2802D003980F28A0
:1096B00000D107E041F23B70C0F602004FF46A713E
:1096C000FBF76BFA039842F20001C5F2002109682A
:1096D00001F00F01884213D942F20000C5F20020C8
:1096E000016821F00F01039A11430160006800F046
:1096F0000F000399884203D001208DF8170060E322
:10970000049800784007002831D50498006944F295
:109710001841C5F60201096801F07001884226D996
:109720000498006978B10498006940280BD0049827
:109730000069502807D004980069602803D0049875
:109740000069702800D107E041F23B70C0F60200CA
:109750004FF47171FBF721FA44F21841C5F602018A
:10976000086820F07000049A126910430860049899
:1097700000780007002831D50498406944F21C4164
:10978000C5F60201096801F07001884226D90498E3
:10979000406978B10498406940280BD0049840692A
:1097A000502807D004984069602803D00498406985
:1097B000702800D107E041F23B70C0F6020040F291
:1097C000D631FBF7EAF944F21C41C5F602010868FC
:1097D00020F07000049A52691043086004980078E1
:1097E000C006002835D50498806944F21C41C5F6AE
:1097F0000201096801F4E06188422AD9049880696D
:1098000098B104988069B0F5806F0ED00498806993
:10981000B0F5A06F09D004988069B0F5C06F04D08E
:1098200004988069B0F5E06F00D107E041F23B7029
:10983000C0F6020040F2E731FBF7AFF944F21C41F9
:10984000C5F60201086820F4E060049A92691043AA
:109850000860049800788006002831D50498C06913
:1098600044F22041C5F60201096801F07001884206
:1098700026D90498C06978B10498C06940280BD0F3
:109880000498C069502807D00498C069602803D0A4
:109890000498C069702800D107E041F23B70C0F61F
:1098A000020040F2F931FBF778F944F22041C5F6A5
:1098B0000201086820F07000049AD2691043086021
:1098C000049800788007002841D50498C06844F2C5
:1098D0001841C5F60201096801F00F01884236D926
:1098E0000498C068F8B10498C06808281BD0049890
:1098F000C068092817D00498C0680A2813D00498B3
:10990000C0680B280FD00498C0680C280BD00498AE
:10991000C0680D2807D00498C0680E2803D00498AA
:10992000C0680F2800D107E041F23B70C0F602008A
:1099300040F20C41FBF731F944F21841C5F602013F
:10994000086820F00F00049AD26810430860049859
:109950000078C007002800F0BD800498806838B304
:1099600004988068B0F5006F22D004988068B0F544
:10997000106F1DD004988068B0F5206F18D004983F
:109980008068B0F5306F13D004988068B0F5406FF0
:109990000ED004988068B0F5506F09D004988068A4
:1099A000B0F5606F04D004988068B0F5706F00D196
:1099B00007E041F23B70C0F6020040F21C41FBF7A9
:1099C000ECF80498406801280AD00498406838B13F
:1099D00004984068022803D004984068032800D106
:1099E00007E041F23B70C0F6020040F21D41FBF778
:1099F000D4F844F21841C5F60201086820F47060FA
:109A0000049A9268104308600498406802280CD1B8
:109A100044F20040C5F602000068C0F3404018B9A7
:109A200001208DF81700CCE12DE004984068032850
:109A30000CD144F20040C5F602000068C0F340605B
:109A400018B901208DF81700BBE11CE004984068AC
:109A500001280CD144F20040C5F602000068C0F3B2
:109A6000002018B901208DF81700AAE10BE044F29C
:109A70000040C5F602000068C0F3800018B901205C
:109A80008DF817009DE144F21041C5F60201086807
:109A900020F00700049A5268104308600DF021F886
:109AA000019044F21040C5F60200006800F0380052
:109AB00004994968C90088420CD00DF012F8019948
:109AC000401A41F28931884203D303208DF81700F0
:109AD00077E1E6E7049800788007002841D50498EC
:109AE000C06844F21841C5F60201096801F00F018F
:109AF000884236D20498C068F8B10498C068082833
:109B00001BD00498C068092817D00498C0680A2898
:109B100013D00498C0680B280FD00498C0680C2894
:109B20000BD00498C0680D2807D00498C0680E2890
:109B300003D00498C0680F2800D107E041F23B70C1
:109B4000C0F6020040F25E41FBF727F844F21841EC
:109B5000C5F60201086820F00F00049AD26810438D
:109B60000860039842F20001C5F20021096801F083
:109B70000F01884213D242F20000C5F200200168B2
:109B800021F00F01039A11430160006800F00F00FB
:109B90000399884203D001208DF8170011E1049841
:109BA00000784007002831D50498006944F2184134
:109BB000C5F60201096801F07001884226D20498B6
:109BC000006978B10498006940280BD004980069B6
:109BD000502807D004980069602803D004980069D1
:109BE000702800D107E041F23B70C0F6020040F25D
:109BF0007F41FAF7D2FF44F21841C5F60201086826
:109C000020F07000049A12691043086004980078EC
:109C10000007002831D50498406944F21C41C5F67C
:109C20000201096801F07001884226D20498406957
:109C300078B10498406940280BD0049840695028B6
:109C400007D004984069602803D0049840697028C0
:109C500000D107E041F23B70C0F6020040F29141B2
:109C6000FAF79BFF44F21C41C5F60201086820F098
:109C70007000049A52691043086004980078C00686
:109C8000002835D50498806944F21C41C5F60201CC
:109C9000096801F4E06188422AD20498806998B189
:109CA00004988069B0F5806F0ED004988069B0F593
:109CB000A06F09D004988069B0F5C06F04D00498F3
:109CC0008069B0F5E06F00D107E041F23B70C0F66B
:109CD000020040F2A341FAF760FF44F21C41C5F6CE
:109CE0000201086820F4E060049A92691043086059
:109CF000049800788006002831D50498C06944F2A1
:109D00002041C5F60201096801F07001884226D29F
:109D10000498C06978B10498C06940280BD00498B1
:109D2000C069502807D00498C069602803D00498FF
:109D3000C069702800D107E041F23B70C0F6020014
:109D400040F2B541FAF729FF44F22041C5F602017D
:109D5000086820F07000049AD26910430860F7F791
:109D6000F9FA44F21842C5F602021168C1F303235E
:109D700042F24C21C0F60201CB5C03F01F03D84035
:109D800000900098126802F00F02895C01F01F0138
:109D9000C84046F64871C2F200410860009846F695
:109DA0004C71C2F20041086046F62470C2F20040D5
:109DB0000068FCF775F98DF80B009DF80B008DF825
:0A9DC00017009DF8170006B080BDE3
:109DCA0080B582B0F7F7C1FA44F21842C5F602022A
:109DDA001168C1F3032342F24C21C0F60201CB5CA5
:109DEA0003F01F03D84001900198126802F00F0295
:109DFA00895C01F01F0120FA01F146F64870C2F2AF
:109E0A0000400160019946F64C72C2F200421160AC
:069E1A00006802B080BDEB
:109E200080B5FFF7D2FF44F21C41C5F60201096874
:109E3000C1F3021242F24C21C0F60201895C01F02A
:069E40001F01C84080BDB7
:109E460080B5FFF7BFFF44F21C41C5F60201096861
:109E5600C1F3022242F24C21C0F60201895C01F0F4
:069E66001F01C84080BD91
:109E6C0080B586B00490039100208DF8070004980B
:109E7C00006820B1049800683F2800D807E041F63C
:109E8C007640C0F6020040F67261FAF780FE049844
:109E9C004068042805D304984068B0F5007F00D8CA
:109EAC0007E041F67640C0F6020040F67361FAF71F
:109EBC006EFE0498806820B104988068802800D8D1
:109ECC0007E041F67640C0F6020040F67461FAF7FE
:109EDC005EFE0498006920B104980069802800D8BF
:109EEC0007E041F67640C0F6020040F67561FAF7DD
:109EFC004EFE0498C06820B10498C068802800D831
:109F0C0007E041F67640C0F6020040F67661FAF7BB
:109F1C003EFE0498406958B104984069402807D027
:109F2C0004984069802803D004984069C02800D167
:109F3C0007E041F67640C0F6020040F67761FAF78A
:109F4C0026FE0498806918B104988069202800D1F5
:109F5C0007E041F67640C0F6020040F67861FAF769
:109F6C0016FE0498C069400B00B907E041F6764034
:109F7C00C0F6020040F67961FAF709FE44F2284077
:109F8C00C5F60200006800F00300032803D101208D
:109F9C008DF81700B7E044F20041C5F602010868DD
:109FAC0020F0806008600CF096FD029044F20040B6
:109FBC00C5F602000068C0F3C06050B10CF08BFD18
:109FCC000299401A032803D303208DF817009AE056
:109FDC00ECE744F22841C5F60201086820F47C3015
:109FEC00049A126840EA0230086004994868D1F873
:109FFC0008C0CB680A6901386FF35F204FF6006127
:10A00C00CFF6FF7101EB4C2189B208440021CFF649
:10A01C00FF7101EB034101F4FE0108444FF07F4155
:10A02C0001EB026101F0FE41084444F23841C5F6EF
:10A03C000201086044F22C41C5F602010091086847
:10A04C0020F0C000049A526910430860086820F0A0
:10A05C002000049A926910430860086820F01000F0
:10A06C00086044F23C42C5F6020210684FF6F873E1
:10A07C009843049BDB6940EAC3001060086840F019
:10A08C0010000860039840B944F22C41C5F6020157
:10A09C00086840F40020086013E00398012808D1F8
:10A0AC0044F22C41C5F60201086840F480100860A7
:10A0BC0007E044F22C41C5F60201086840F4001098
:10A0CC00086044F20041C5F60201086840F0806067
:10A0DC0008600CF000FD029044F20040C5F602004E
:10A0EC000068C0F3C06050B90CF0F5FC0299401A3E
:10A0FC00032803D303208DF8170004E0ECE79DF848
:0EA10C0007008DF817009DF8170006B080BD03
:10A11A0080B586B00490039100208DF8070004985A
:10A12A00006820B1049800683F2800D807E041F68B
:10A13A007640C0F6020040F6DA61FAF729FD049883
:10A14A004068042805D304984068B0F5007F00D819
:10A15A0007E041F67640C0F6020040F6DB61FAF706
:10A16A0017FD0498806820B104988068802800D878
:10A17A0007E041F67640C0F6020040F6DC61FAF7E5
:10A18A0007FD0498006920B104980069802800D866
:10A19A0007E041F67640C0F6020040F6DD61FAF7C4
:10A1AA00F7FC0498C06820B10498C068802800D8D9
:10A1BA0007E041F67640C0F6020040F6DE61FAF7A3
:10A1CA00E7FC0498406970B104984069B0F5806F63
:10A1DA0009D004984069B0F5006F04D0049840692A
:10A1EA00B0F5406F00D107E041F67640C0F60200B4
:10A1FA0040F6DF61FAF7CCFC0498806920B1049834
:10A20A008069B0F5007F00D107E041F67640C0F6DC
:10A21A0002004FF46E61FAF7BBFC0498C069400B68
:10A22A0000B907E041F67640C0F6020040F6E16167
:10A23A00FAF7AEFC44F22840C5F60200006800F0C6
:10A24A000300032803D101208DF81700B7E044F278
:10A25A000041C5F60201086820F0805008600CF041
:10A26A003BFC029044F20040C5F602000068C0F3CD
:10A27A00407050B10CF030FC0299401A032803D305
:10A28A0003208DF817009AE0ECE744F22841C5F65E
:10A29A000201086820F07C70049A126840EA0250B1
:10A2AA00086004994868D1F808C0CB680A6901387F
:10A2BA006FF35F204FF60061CFF6FF7101EB4C217F
:10A2CA0089B208440021CFF6FF7101EB034101F482
:10A2DA00FE0108444FF07F4101EB026101F0FE41AB
:10A2EA00084444F24041C5F60201086044F22C4198
:10A2FA00C5F602010091086820F44060049A526988
:10A30A0010430860086820F40070049A92691043A8
:10A31A000860086820F48070086044F24442C5F678
:10A32A00020210684FF6F8739843049BDB6940EA0F
:10A33A00C3001060086840F480700860039840B950
:10A34A0044F22C41C5F60201086840F48000086016
:10A35A0013E00398012808D144F22C41C5F6020102
:10A36A00086840F40000086007E044F22C41C5F692
:10A37A000201086840F08070086044F20041C5F6A6
:10A38A000201086840F0805008600CF0A5FB0290BA
:10A39A0044F20040C5F602000068C0F3407050B9AC
:10A3AA000CF09AFB0299401A032803D303208DF874
:10A3BA00170004E0ECE79DF807008DF817009DF8F8
:06A3CA00170006B080BD83
:10A3D00080B5FFF7FAFC44F22041C5F60201096896
:10A3E000C1F3021242F24C21C0F60201895C01F075
:06A3F0001F01C84080BD02
:10A3F60080B582B0019001208DF8030001980028F5
:10A4060000F0E9800198006844F20001C5F60001F9
:10A41600884200D106E041F2A270C0F60200FD219A
:10A42600FAF7B8FB01984068402802D001984068C6
:10A4360000B906E041F2A270C0F60200FE21FAF76A
:10A44600A9FB019880687F2800D806E041F2A27037
:10A45600C0F60200FF21FAF79DFB0198C068C00B09
:10A4660000B907E041F2A270C0F602004FF4807115
:10A47600FAF790FB0198006970B101980069B0F590
:10A48600001F09D001980069B0F5800F04D001982B
:10A496000069B0F5C00F00D107E041F2A270C0F626
:10A4A600020040F20111FAF775FB0198406918B1F4
:10A4B60001984069022800D107E041F2A270C0F677
:10A4C60002004FF48171FAF765FB0198806920B1AB
:10A4D60001988069B0F5801F00D107E041F2A270B3
:10A4E600C0F6020040F20311FAF754FB0198C06966
:10A4F60018B10198C069012800D107E041F2A270A5
:10A50600C0F602004FF48271FAF744FB019890F806
:10A51600210030B90199002081F820000198FBF74D
:10A52600B3FC0199022081F8210001980068C068F7
:10A53600C0F30010002844D101980168CA2048627F
:10A546000198016853204862019800F048F88DF898
:10A5560003009DF80300F0B90198016888684FF67A
:10A56600BF72CFF68F7210408860019A11685068EA
:10A5760013699269184302438868104388600198FA
:10A5860001688268C06840EA02400861019800F0EC
:10A596005DF88DF803009DF8030068B9019801681D
:10A5A600C86C20F00300C864019801684269C0695C
:10A5B6000243C86C1043C86401980168FF204862D2
:10A5C60002E000208DF803009DF8030018B90199F8
:0EA5D600012081F821009DF8030002B080BD35
:10A5E40080B584B0039000208DF8070003980068BC
:10A5F400C0684006002826D4039801684FF0FF3055
:10A60400C8600CF06CFA029003980068C1680020DE
:10A6140049060029009005D49DF80700033818BFA7
:10A62400012000900098C00768B10CF058FA029914
:10A63400401AB0F57A7F05D903208DF807000399F5
:0EA6440081F82100E0E79DF8070004B080BD1A
:10A6520080B582B0019000208DF8030044F20C0115
:10A66200C5F60001086820F08000086044F2080086
:10A67200C5F600000068800600280AD401980EF092
:10A6820031FA28B10199032081F821008DF80300E5
:10A6920019E044F20801C5F60001086820F0200024
:10A6A200086001980EF01EFA28B10199032081F882
:10A6B20021008DF8030044F20801C5F60001086884
:0EA6C20040F0200008609DF8030002B080BD4B
:10A6D00080B588B0069005910492049810B1049852
:10A6E000012800D107E041F2A270C0F6020040F25A
:10A6F0004F31FAF752FA0598C068B0F5003F07D01D
:10A700000598C068B0F5803F02D00598C06800B9D0
:10A7100007E041F2A270C0F602004FF45471FAF75C
:10A720003CFA0598006920B105980069B0F5802FC2
:10A7300000D107E041F2A270C0F6020040F25131B0
:10A74000FAF72BFA069890F82000012803D102208E
:10A750008DF81F0021E10699012081F8200006995B
:10A76000022081F8210006980168CA2048620698F4
:10A770000168532048620698FFF734FF8DF80B00FC
:10A780009DF80B00002840F0F580049800286CD15B
:10A790000698006880684006002820D50598007853
:10A7A00020B1059800780C2800D807E041F2A2708B
:10A7B000C0F6020040F26231FAF7EFF90598C0786E
:10A7C00018B10598C078012800D107E041F2A270C5
:10A7D000C0F6020040F26331FAF7DFF90FE00599A5
:10A7E0000020C87005980078172800D807E041F2CB
:10A7F000A270C0F602004FF45A71FAF7CEF905982C
:10A8000040783B2800D807E041F2A270C0F6020071
:10A8100040F26A31FAF7C1F9059880783B2800D8F0
:10A8200007E041F2A270C0F6020040F26B31FAF785
:10A83000B4F90598007800F0B4F800040090059889
:10A84000407800F0AEF80146009840EA01200190FF
:10A850000598807800F0A5F801460198084405990C
:10A86000C97840EA8150039066E0069800688068E5
:10A870004006002824D50598007800F0B1F830B1E2
:10A880000598007800F0ACF80C2800D807E041F2F9
:10A89000A270C0F6020040F27631FAF77EF9059810
:10A8A000C07818B10598C078012800D107E041F2BE
:10A8B000A270C0F6020040F27731FAF76EF911E0AB
:10A8C00005990020C8700598007800F089F81728CD
:10A8D00000D807E041F2A270C0F602004FF45F71A9
:10A8E000FAF75BF90598407800F07AF83B2800D831
:10A8F00007E041F2A270C0F6020040F27E31FAF7A2
:10A900004CF90598807800F06BF83B2800D807E0F8
:10A9100041F2A270C0F6020040F27F31FAF73DF931
:10A92000059908784B788A78C978000440EA0320B2
:10A93000104440EA81500390039847F67F71C0F2BB
:10A940007F010840069909680860069801688868D0
:10A9500020F4802088600599C868096940EA0102EE
:10A96000069801688868104388600698FFF771FEB2
:10A970008DF80B0006980168FF2048629DF80B00D7
:10A9800018B90699012081F821000699002081F864
:10A9900020009DF80B008DF81F009DF81F0008B0E7
:02A9A00080BD78
:10A9A20083B08DF80B00002001909DF80B008DF80C
:10A9B20003009DF803000A2808D301980130019092
:10A9C2009DF803000A388DF80300F2E7019800F0C1
:0EA9D2000F019DF8030040EA011003B070472A
:10A9E00081B08DF803009DF80300000900EB8000A2
:10A9F00040008DF802009DF802009DF8031001F060
:0AAA00000F010844C0B201B0704716
:10AA0A0080B58AB00890089818B901208DF82700F7
:10AA1A00DBE00898006847F20001C5F2002188428D
:10AA2A0007D00898006842F20041C4F60201884241
:10AA3A0000D107E041F6E040C0F602004FF4B071E1
:10AA4A00FAF7A6F80898406820B108984068B0F567
:10AA5A00803F00D107E041F6E040C0F6020040F234
:10AA6A006111FAF795F80898806820B1089880680B
:10AA7A00B0F5805F00D107E041F6E040C0F6020081
:10AA8A004FF4B171FAF784F80898C06848B1089889
:10AA9A00C068B0F5804F04D00898C068B0F5004F80
:10AAAA0000D107E041F6E040C0F6020040F263112F
:10AABA00FAF76EF80898006920B108980069B0F5AD
:10AACA00003F00D107E041F6E040C0F602004FF433
:10AADA00B271FAF75DF808984069800A00B907E090
:10AAEA0041F6E040C0F6020040F26511FAF750F86C
:10AAFA00089890F8300028B9089900200876089834
:10AB0A00FBF7FEF90899042081F8300008980EF046
:10AB1A0025F918B101208DF8270056E0089803A9F5
:10AB2A000EF0AEF918B101208DF827004DE09DF81E
:10AB3A001C0002909DF81D0001900898806B012866
:10AB4A0008D1029808B9019820B108994FF4007009
:10AB5A0088650BE00898806B012804D108994FF4A6
:10AB6A008070886502E00899002088650898C168A5
:10AB7A0000F02FF818B101208DF8270025E00BF01E
:10AB8A00ABFF009008980EF00FFA042812D00BF0D1
:10AB9A00A3FF0099401A013058B908994FF00040B4
:10ABAA0048630899012081F8300003208DF82700B6
:10ABBA000BE0E7E70899002048630899C862089AF9
:10ABCA00012182F830108DF827009DF827000AB07D
:02ABDA0080BD3C
:10ABDC0010B58CB00B900A9100208DF80B000A98E0
:10ABEC0038B10A98B0F5804F03D00A98B0F5004FF1
:10ABFC0000D107E041F6E040C0F6020040F66711D4
:10AC0C00F9F7C5FF0B99032081F830000B98806B86
:10AC1C00032829D00A98B0F5004F05D10B99486B41
:10AC2C0040F0805048631EE00A98B0F5804F09D17F
:10AC3C000B980EF0F4F90490049A0B99486B10439E
:10AC4C00486310E00A9848B90B9800F0EEF80490AD
:10AC5C00049A0B99486B1043486304E00B99486BBA
:10AC6C0040F00060486304E00B99486B40F0805062
:10AC7C0048630B98406B50B10B98016840F6FF701D
:10AC8C00C1F6E070886301208DF80B00ADE04FF445
:10AC9C0080300021F9F7B2FA03900398002800F0F5
:10ACAC009C800B98406805900B98806806900A98D9
:10ACBC0007900B98006908900B984069039943F62C
:10ACCC008932C5F2E652A1FB0221B0EB116F03D31E
:10ACDC000B984069099070E00B98806DB0F5007F7F
:10ACEC0003D10B984069099067E00B98806DB0F523
:10ACFC00807F31D10B984069A0B903984FF2810144
:10AD0C00C0F2FA21884209D3039843F68931C5F27F
:10AD1C00E651A0FB0110400E099002E00B9840692F
:10AD2C00099018E003980B9949694900B0FBF1F0C0
:10AD3C004FF28101C0F2FA21884209D3039843F6FD
:10AD4C008931C5F2E651A0FB0110400E099002E0DA
:10AD5C000B984069099030E00B984069A0B90398B2
:10AD6C0047F64101C0F27D11884209D3039843F69E
:10AD7C008931C5F2E651A0FB0110000E099002E0EA
:10AD8C000B984069099018E003980B9949694900A0
:10AD9C00B0FBF1F047F64101C0F27D11884209D3B6
:10ADAC00039843F68931C5F2E651A0FB0110000E61
:10ADBC00099002E00B98406909900B98006805997E
:10ADCC00069A079BDDF820C0099CEE46CEF804409D
:10ADDC00CEF800C005F0D2F807E00B99486B40F0B4
:10ADEC000060486301208DF80B000B9800684FF44D
:10ADFC00007105F09AFA0490049870B10B980168F0
:10AE0C0040F6FF70C1F6E0708863049A0B99486BAA
:10AE1C001043486301208DF80B000B99012081F839
:0AAE2C0030009DF80B000CB010BDC3
:10AE360080B586B0049000210391029104980068C1
:10AE460005F0ACF98001002803D54FF400600590A9
:10AE56002AE0049802A90EF025F90190019810B194
:10AE66000198059020E09DF80E00C007C8B104992E
:10AE76000868496C090405F037FC0190019810B187
:10AE86000198059010E004980068002105F066FC22
:10AE96000190019810B10198059005E000200590F9
:0EAEA60002E04FF080600590059806B080BD78
:10AEB40080B58EB00C900B910BF011FE03900B98A3
:10AEC40001900C980068002105F069F980010028C0
:10AED40003D54FF400600D90A2E00C980068402167
:10AEE40005F027FA0490049828B10C99486B48633C
:10AEF40004980D9094E00C990868496C090405F0D5
:10AF0400F4FB0490049828B10C99486B48630498A6
:10AF14000D9085E04FF0FF300590402006906020B2
:10AF24000790022008900020099001200A900C98B4
:10AF3400006805A905F054F90C98006805F083FD34
:10AF44000490049828B10C99486B486304980D90B8
:10AF540066E00C980068406B10F4957F22D10C9841
:10AF64000068406B0004002811D50020029002986C
:10AF740007280CD80C98006805F08BF80199086034
:10AF8400019804300190029801300290EFE70BF031
:10AF9400A6FD0399401A013018B94FF000400D90F6
:10AFA4003EE0D6E70C980068406B0007002802D505
:10AFB40008200D9034E00C980068406B800700284E
:10AFC40002D502200D902BE00C980068406B80069F
:10AFD400002802D520200D9022E00C980068406BD8
:10AFE400C004002813D50C98006805F052F80199A4
:10AFF40008600198043001900BF071FD0399401A28
:10B00400013018B94FF000400D9009E0E5E70C98C5
:10B01400016840F63A70C1F60000886300200D9084
:06B024000D980EB080BD86
:10B02A0080B588B006900020059004900390069899
:10B03A00006810F0ADFC0290029810B102980790D7
:10B04A007AE00698006805F032FB02900298B0F1A7
:10B05A00004F0DD106990020C8630698006810F0C9
:10B06A0097FC0290029810B10298079064E002E0FF
:10B07A0006990120C8630698C06B01280BD106986F
:10B08A000068002105F02EFB0290029818B14FF0DB
:10B09A008050079050E0059900204FF6FE729142C9
:10B0AA00019004D80398B0FA80F040090190019801
:10B0BA00C00758B306980068002105F013FB0290F8
:10B0CA00029810B10298079036E0069800680021AD
:10B0DA00CCF2101105F025FB0290029818B14FF03E
:10B0EA008050079028E006980068002105F054F87F
:10B0FA00049004994FF0FF3000EBD170B0FA80F061
:10B10A0040090390059801300590C4E705984FF669
:10B11A00FF71884203D34FF0807007900CE00699C4
:10B12A00002088639DF813004006002802D506997E
:0EB13A000120886300200790079808B080BDB0
:10B1480083B0019000910198C06D800F009908703C
:10B158000198C06DC0F38360009948700198C06D74
:10B16800C0F30160009988700198B0F85E000099FA
:10B17800C8700198C06D000A009908710198C06DE7
:10B18800009948710198006E000D0099C8800198D7
:10B19800006EC0F30340009908720198B0F860008F
:10B1A800C00B009948720198006EC0F38030009976
:10B1B80088720198006EC0F340300099C8720198F7
:10B1C800006EC0F30030009908730099002048739E
:10B1D8000198806B00284AD10199086E496E6FF377
:10B1E8009F20800040EA9170009908610198406EA4
:10B1F800C0F3C260009908750198406EC0F3026000
:10B20800009948750198406EC0F3425000998875BE
:10B218000198406EC0F382400099C8750198406E4D
:10B22800C0F3C2300099087600980069013001998E
:10B2380088640098007E00F00700811C012000FA55
:10B2480001F3019A916C594391640099097A01F0CC
:10B258000F0188400199C8640199886CCA6C520A28
:10B268005043086501994FF40070486533E0019830
:10B27800806B01281CD10198016E01F03F01B0F8E4
:10B28800660040EA014000990861009801694FF49E
:10B29800806000EB8120019988640199886C0865B9
:10B2A80001994FF40070C8640199C86C486512E0B0
:10B2B8000198016840F6FF70C1F6E0708863019953
:10B2C800486B40F0805048630199012081F83000B4
:10B2D8008DF80B0071E00198406EC0F38030009942
:10B2E80048760198406EC0F3C61000998876019898
:10B2F800406E00F07F000099C8760198806EC00FFC
:10B30800009908770198806EC0F3417000994877DA
:10B318000198806EC0F38260009988770198806EEA
:10B32800C0F383500099C8770198806EC0F34050ED
:10B33800009981F820000099002081F821000199E6
:10B34800896EC1F30041009A82F822100199B1F880
:10B358006810C90B009A82F823100199896EC1F30D
:10B368008031009A82F824100199896EC1F3403126
:10B37800009A82F825100199896EC1F30031009A6C
:10B3880082F826100199896EC1F38121009A82F80A
:10B3980027100199896EC1F30121009A82F82810BB
:10B3A800019991F868104908009A82F82910009AC2
:10B3B800012182F82A108DF80B009DF80B0003B0CC
:02B3C8007047CC
:10B3CA0080B58EB00C900B910A9209930A9801905D
:10B3DA000B9840B90C99486B40F000604863012013
:10B3EA008DF8370089E00C9890F83000012840F079
:10B3FA0081800C99002048630198099908440C99A6
:10B40A00096D884208D90C99486B40F0007048636E
:10B41A0001208DF8370070E00C99032081F8300084
:10B42A000C9801680020C8620B980C994862099828
:10B43A0040020C9988620C98806B012802D001980E
:10B44A00400201904FF0FF300390099840020490A7
:10B45A0090200590022006900020079008900C98F2
:10B46A00006803A904F0B9FE0C980168C86840F0A6
:10B47A004000C8600B980C99096888650C980168A7
:10B48A00012008650998022809D30C998220C8620C
:10B49A000C980068019905F08EF8029008E00C9962
:10B4AA008120C8620C980068019905F065F802903D
:10B4BA000298A8B10C98016840F6FF70C1F6E070D6
:10B4CA008863029A0C99486B104348630C990120CF
:10B4DA0081F830000C9A0021D1628DF837000CE017
:10B4EA000C980168C86B40F49570C86300208DF809
:10B4FA00370002E002208DF837009DF837000EB0C1
:02B50A0080BD02
:10B50C0080B584B003900398C06A019003980068DA
:10B51C00406B80B2C00B40B19DF8040000070028BE
:10B52C0003D503980DF0BFFF71E103980068406BE1
:10B53C00C0F30020002800F09F80039801684FF4AE
:10B54C008070886303980168C86B4CF23A12904380
:10B55C00C86303980168C86B20F08050C8630398D7
:10B56C000168C86820F04000C8609DF8040000071E
:10B57C00002837D59DF804008007002804D49DF8D6
:10B58C000400800600280ED50398006810F0CBF953
:10B59C000290029838B1029A0399486B10434863A1
:10B5AC0003980AF078FB0398016840F63A70C1F6EC
:10B5BC00000088630399012081F830000399002072
:10B5CC00C8629DF80400C00720B99DF804008007EC
:10B5DC00002803D5039806F017FD02E0039806F047
:10B5EC000CFD48E09DF804000006002843D50398A4
:10B5FC0001680020886203990968C8620399096888
:10B60C0008659DF804008007002804D49DF8040008
:10B61C00800600280ED50398006810F084F902907B
:10B62C00029838B1029A0399486B10434863039807
:10B63C000AF031FB0399012081F8300003990020B6
:10B64C00C8629DF80400C006002804D49DF80400CC
:10B65C008006002802D5039806F0CFFC9DF8040064
:10B66C00C00720B99DF804008007002802D5039874
:10B67C0006F0CAFCFFE7CAE003980068406BC0F311
:10B68C00803040B19DF804000007002803D50398D2
:10B69C000DF045FFBBE003980068406B10F03A0FCB
:10B6AC0000F08A8003980068406BC0F3400020B122
:10B6BC000399486B40F00200486303980068406BA4
:10B6CC00C0F3C00020B10399486B40F008004863F8
:10B6DC0003980068406BC0F3401020B10399486B8D
:10B6EC0040F02000486303980068406BC0F30010E2
:10B6FC0020B10399486B40F010004863039801682F
:10B70C0040F63A70C1F60000886303980168C86B74
:10B71C0020F49D70C86303980168C86820F040004D
:10B72C00C86003980168C86A40F40050C862039866
:10B73C000168C86840F08000C8600398006810F089
:10B74C00F2F802460399486B10434863039801686A
:10B75C00C86820F08000C860039801684FF400604E
:10B76C0088639DF80400000700280AD5039901207E
:10B77C0081F8300003990020C86203980AF08BFA14
:10B78C0019E09DF804000006002814D50398406BBE
:10B79C0080B103980168C86B20F08050C86303988F
:10B7AC000168002008650399012081F83000039896
:10B7BC000AF071FAFFE72AE003980068406BC0F3C7
:10B7CC00007020B3039801684FF080508863039891
:10B7DC000068006D400700280CD49DF8040080061A
:10B7EC00002803D503980AF056FA02E003980AF0F1
:10B7FC0052FA0BE09DF804008006002803D503984C
:10B80C000AF049FA02E003980AF045FAFFE704B09F
:02B81C0080BDED
:10B81E0080B586B00490049818B901208DF81700F1
:10B82E00EBE20498006843F20001C4F20101884281
:10B83E0027D00498006843F60001C4F20001884244
:10B84E001FD00498006843F60041C4F200018842FC
:10B85E0017D00498006843F20041C4F201018842F7
:10B86E000FD00498006845F20001C4F2010188422D
:10B87E0007D00498006841F20041C5F600018842E5
:10B88E0000D106E041F60900C0F60200FE21F9F7EC
:10B89E007DF90498406820B104984068B0F5800F97
:10B8AE0000D106E041F60900C0F60200FF21F9F7CB
:10B8BE006DF90498806870B104988068B0F5802F97
:10B8CE0009D004988068B0F5C02F04D00498806821
:10B8DE00B0F5003F00D107E041F60900C0F60200C6
:10B8EE004FF48071F9F752F90498C0681F2873D08D
:10B8FE000498C0681E286FD00498C0681D286BD0AD
:10B90E000498C0681C2867D00498C0681B2863D0B0
:10B91E000498C0681A285FD00498C06819285BD0B4
:10B92E000498C068182857D00498C068172853D0B8
:10B93E000498C06816284FD00498C06815284BD0BC
:10B94E000498C068142847D00498C068132843D0C0
:10B95E000498C06815283FD00498C06812283BD0C0
:10B96E000498C068112837D00498C068102833D0C6
:10B97E000498C0680F282FD00498C0680E282BD0CA
:10B98E000498C0680D2827D00498C0680C2823D0CE
:10B99E000498C0680B281FD00498C0680A281BD0D2
:10B9AE000498C068092817D00498C068082813D0D6
:10B9BE000498C06807280FD00498C06806280BD0DA
:10B9CE000498C068052807D00498C068042803D0DE
:10B9DE000498C068032800D107E041F60900C0F6BC
:10B9EE00020040F20111F9F7D1F80498C06B00285B
:10B9FE0043D00498C06B20283FD00498C06B4028D9
:10BA0E003BD00498C06B602837D00498C06B802858
:10BA1E0033D00498C06BA0282FD00498C06BC028D8
:10BA2E002BD00498C06BE02827D00498C06BB0F5DB
:10BA3E00807F22D00498C06BB0F5907F1DD0049803
:10BA4E00C06BB0F5A07F18D00498C06BB0F5B07F76
:10BA5E0013D00498C06BB0F5C07F0ED00498C06BA5
:10BA6E00B0F5D07F09D00498C06BB0F5E07F04D05C
:10BA7E000498C06BB0F5F07F00D107E041F60900E5
:10BA8E00C0F602004FF48171F9F780F804988069CE
:10BA9E00B0F1806F07D00498806920B10498806956
:10BAAE00B0F1005F00D107E041F60900C0F60200D8
:10BABE0040F20311F9F76AF80498406BB0F1804F29
:10BACE0002D00498406B00B907E041F60900C0F6B9
:10BADE0002004FF48271F9F759F80498C06910B357
:10BAEE000498C069B0F1805F1DD00498C069B0F1B0
:10BAFE00005F18D00498C069B0F1405F13D004986D
:10BB0E00C069B0F1804F0ED00498C069B0F1A04F5B
:10BB1E0009D00498C069B0F1C04F04D00498C06930
:10BB2E00B0F1E04F00D107E041F60900C0F6020087
:10BB3E0040F20511F9F72AF80498006A20B104982A
:10BB4E00006AB0F5000F00D107E041F60900C0F61B
:10BB5E0002004FF48371F9F719F80498406A20B186
:10BB6E000498406AB0F5002F00D107E041F60900B5
:10BB7E00C0F6020040F20711F9F708F80498406A7F
:10BB8E0008BB0498006920B104980069B0F1007FE9
:10BB9E0000D107E041F60900C0F602004FF48571AE
:10BBAE00F8F7F4FF0498406920B104984069B0F1A9
:10BBBE00807F00D107E041F60900C0F6020040F296
:10BBCE000B11F8F7E3FF04990020886204980068CF
:10BBDE0043F20001C4F20101884217D004980068B4
:10BBEE0043F60001C4F2000188420FD004980068A9
:10BBFE0043F60041C4F20001884207D00498C068A1
:10BC0E00102803D301208DF81700F6E0049800F0F9
:10BC1E00F8F802900498006843F20001C4F20101A2
:10BC2E00884212D00498006843F60001C4F2000165
:10BC3E0088420AD00498006843F60041C4F200011D
:10BC4E00884202D0029808281AD80498006843F255
:10BC5E000001C4F2010188420FD00498006843F637
:10BC6E000001C4F20001884207D00498006843F630
:10BC7E000041C4F20001884206D10298112803D374
:10BC8E0001208DF81700B8E0049890F8810030B9C3
:10BC9E000499002081F8800004980AF00BFB0499A7
:10BCAE00022081F8810004980168086820F00100E4
:10BCBE00086004980068806800F4F81003900498F7
:10BCCE008069B0F1806F15D104984068B0F5800F8F
:10BCDE0002D10498806B38B10498406850B904982A
:10BCEE00806BB0F1805F05D104980168086840F45C
:10BCFE008050086004988079400600280ED504987C
:10BD0E00C06807280AD304980068006820F4807081
:10BD1E00049A1168126D1043086005E004980168DA
:10BD2E00086820F480700860049B1968DA68D86986
:10BD3E00D3F828C040EA0C00DDF80CC040EA0C0035
:10BD4E00DB6B184310438860049A0192506B516A62
:10BD5E000843916B0843916908431168D2F804C0F7
:10BD6E009368D2F810E040EA0E00D2F814E040EAF0
:10BD7E000E00D2F820E040EA0E0040EA0C00D2F8A5
:10BD8E004CC040EA0C001843936C1843926D10435C
:10BD9E00C8600498406888B90498006880680121DA
:10BDAE0061F3CC2004990968886004980068806863
:10BDBE00022161F34A200499096888600498016899
:10BDCE00086D20F00100086504988079400600286F
:10BDDE0009D504980068C06820F00040049A1168E4
:10BDEE00526D1043C86004990020C1F88400049A73
:10BDFE00012182F881108DF817009DF8170006B00A
:02BE0E0080BDF5
:10BE100083B002900298C16B012000EB5110019099
:10BE20000298C0680130009000980730C008009068
:0ABE300000980199484303B07047E1
:10BE3A0082B00190019800684069009001980168F9
:10BE4A00886940F00800886101980168886940F0B3
:10BE5A001000886101980168086820F001000860F4
:10BE6A0001980168086940F26F32904308610198AD
:10BE7A000168886820F440408860019890F8810041
:10BE8A00042811D09DF80000800600280CD50199DD
:10BE9A00D1F8840040F08000C1F88400019801685C
:10BEAA00886940F020008861019890F88100032891
:10BEBA0011D09DF80000400600280CD50199D1F850
:10BECA00840040F00400C1F8840001980168886980
:10BEDA0040F0400088619DF80100800700280CD5D9
:10BEEA000199D1F8840040F00100C1F8840001985A
:10BEFA000168886940F4007088619DF80100C007F4
:10BF0A0060B10199D1F8840040F00800C1F88400BA
:10BF1A0001980168886940F480708861019900205D
:0EBF2A00A1F862000199A1F86A0002B0704708
:0EBF380081B00090009890F8810001B0704731
:10BF460080B584B00290029818B901208DF80F00D0
:10BF560043E1029800680021C4F20101884274D0CE
:10BF660002980068B0F1804F6FD00298006840F2E6
:10BF76000041C4F20001884267D00298006840F68A
:10BF86000001C4F2000188425FD00298006840F6C2
:10BF96000041C4F20001884257D00298006841F27D
:10BFA6000001C4F2000188424FD00298006841F2B5
:10BFB6000041C4F20001884247D00298006840F26E
:10BFC6000041C4F2010188423FD00298006841F660
:10BFD6000001C4F20001884237D00298006841F699
:10BFE6000041C4F2000188422FD00298006842F254
:10BFF6000001C4F20001884227D00298006844F28A
:10C006000001C4F2010188421FD00298006844F280
:10C016000041C4F20101884217D00298006844F634
:10C026000001C4F2010188420FD0029800684EF266
:10C036000001C4F20001884207D0029800684EF25F
:10C046000041C4F20001884200D107E041F67000C9
:10C05600C0F602004FF48B71F8F79CFD02988068D9
:10C0660078B10298806810280BD002988068202842
:10C0760007D002988068402803D00298806860281C
:10C0860000D107E041F67000C0F6020040F2171139
:10C09600F8F780FD0298006948B102980069B0F58A
:10C0A600807F04D002980069B0F5007F00D107E0D8
:10C0B60041F67000C0F602004FF48C71F8F76AFD85
:10C0C600029801680120B1F1804F01901ED00298BC
:10C0D6000168012040F60042C4F20002914201903C
:10C0E60014D00298016801204EF20002C4F2000248
:10C0F600914201900AD00298006841F60041CBF6C1
:10C10600FF710844B0FA80F0400901900198C00719
:10C1160040B90298C06848B10298C068B0F5803F3F
:10C1260003D303E00298C06800B107E041F670004F
:10C13600C0F6020040F21911F8F72CFD029880694A
:10C1460018B102988069802800D107E041F6700096
:10C15600C0F602004FF48D71F8F71CFD029890F8B6
:10C166003D0030B90299002081F83C0002980AF09F
:10C17600EFFA0299022081F83D00029951F8040B6A
:10C1860000F02FF80299012081F848000299012059
:10C1960081F83E00029981F83F00029981F840003B
:10C1A600029981F84100029981F84200029981F8CA
:10C1B60043000299012081F84400029981F8450064
:10C1C600029981F84600029981F8470002990120F8
:10C1D60081F83D0000208DF80F009DF80F0004B097
:02C1E60080BD1A
:10C1E80083B00290019102980068009002980021A3
:10C1F800C4F2010188421FD00298B0F1804F1BD0D1
:10C20800029840F20041C4F20001884214D002981A
:10C2180040F60001C4F2000188420DD0029840F6B1
:10C228000041C4F20001884206D0029840F2004161
:10C23800C4F20101884208D1009820F070000090F3
:10C248000198416800980843009002980021C4F2C0
:10C258000101884242D00298B0F1804F3ED0029846
:10C2680040F20041C4F20001884237D0029840F6FB
:10C278000001C4F20001884230D0029840F6004123
:10C28800C4F20001884229D0029840F20041C4F269
:10C298000101884222D0029844F20001C4F201014F
:10C2A80088421BD0029844F20041C4F2010188423E
:10C2B80014D0029844F60001C4F2010188420DD05E
:10C2C80002984EF20001C4F20001884206D002989A
:10C2D8004EF20041C4F20001884208D1009820F4CF
:10C2E800407000900198C168009808430090009839
:10C2F80020F08000019949690843009001988068FE
:10C308000299C8620198006802998862029800211F
:10C31800C4F2010188421BD0029840F20041C4F2E5
:10C328000101884214D0029844F20001C4F20101CC
:10C3380088420DD0029844F20041C4F201018842BB
:10C3480006D0029844F60001C4F20101884203D1E4
:10C3580001980069029908630299086840F004008E
:10C36800086002990120486100980299086003B0AA
:02C3780070470C
:10C37A0080B584B00290029818B901208DF80F0098
:10C38A0043E1029800680021C4F20101884274D096
:10C39A0002980068B0F1804F6FD00298006840F2AE
:10C3AA000041C4F20001884267D00298006840F652
:10C3BA000001C4F2000188425FD00298006840F68A
:10C3CA000041C4F20001884257D00298006841F245
:10C3DA000001C4F2000188424FD00298006841F27D
:10C3EA000041C4F20001884247D00298006840F236
:10C3FA000041C4F2010188423FD00298006841F628
:10C40A000001C4F20001884237D00298006841F660
:10C41A000041C4F2000188422FD00298006842F21B
:10C42A000001C4F20001884227D00298006844F251
:10C43A000001C4F2010188421FD00298006844F248
:10C44A000041C4F20101884217D00298006844F6FC
:10C45A000001C4F2010188420FD0029800684EF22E
:10C46A000001C4F20001884207D0029800684EF227
:10C47A000041C4F20001884200D107E041F6700091
:10C48A00C0F6020040F23351F8F782FB0298806846
:10C49A0078B10298806810280BD00298806820280A
:10C4AA0007D002988068402803D0029880686028E4
:10C4BA0000D107E041F67000C0F6020040F23451A4
:10C4CA00F8F766FB0298006948B102980069B0F56E
:10C4DA00807F04D002980069B0F5007F00D107E0A0
:10C4EA0041F67000C0F6020040F23551F8F750FBF1
:10C4FA00029801680120B1F1804F01901ED0029884
:10C50A000168012040F60042C4F200029142019003
:10C51A0014D00298016801204EF20002C4F200020F
:10C52A00914201900AD00298006841F60041CBF688
:10C53A00FF710844B0FA80F0400901900198C007E1
:10C54A0040B90298C06848B10298C068B0F5803F07
:10C55A0003D303E00298C06800B107E041F6700017
:10C56A00C0F6020040F23651F8F712FB02988069D1
:10C57A0018B102988069802800D107E041F670005E
:10C58A00C0F6020040F23751F8F702FB029890F821
:10C59A003D0030B90299002081F83C00029809F068
:10C5AA007BFB0299022081F83D00029951F8040BA5
:10C5BA00FFF715FE0299012081F84800029901202F
:10C5CA0081F83E00029981F83F00029981F8400003
:10C5DA00029981F84100029981F84200029981F892
:10C5EA0043000299012081F84400029981F845002C
:10C5FA00029981F84600029981F8470002990120C0
:10C60A0081F83D0000208DF80F009DF80F0004B05E
:02C61A0080BDE1
:10C61C0080B584B00290029818B901208DF80F00F3
:10C62C0043E1029800680021C4F20101884274D0F1
:10C63C0002980068B0F1804F6FD00298006840F209
:10C64C000041C4F20001884267D00298006840F6AD
:10C65C000001C4F2000188425FD00298006840F6E5
:10C66C000041C4F20001884257D00298006841F2A0
:10C67C000001C4F2000188424FD00298006841F2D8
:10C68C000041C4F20001884247D00298006840F291
:10C69C000041C4F2010188423FD00298006841F683
:10C6AC000001C4F20001884237D00298006841F6BC
:10C6BC000041C4F2000188422FD00298006842F277
:10C6CC000001C4F20001884227D00298006844F2AD
:10C6DC000001C4F2010188421FD00298006844F2A4
:10C6EC000041C4F20101884217D00298006844F658
:10C6FC000001C4F2010188420FD0029800684EF28A
:10C70C000001C4F20001884207D0029800684EF282
:10C71C000041C4F20001884200D107E041F67000EC
:10C72C00C0F6020040F2CF71F8F731FA0298806837
:10C73C0078B10298806810280BD002988068202865
:10C74C0007D002988068402803D00298806860283F
:10C75C0000D107E041F67000C0F602004FF4FA6118
:10C76C00F8F715FA0298006948B102980069B0F51B
:10C77C00807F04D002980069B0F5007F00D107E0FB
:10C78C0041F67000C0F6020040F2D171F8F7FFF9E3
:10C79C00029801680120B1F1804F01901ED00298DF
:10C7AC000168012040F60042C4F20002914201905F
:10C7BC0014D00298016801204EF20002C4F200026B
:10C7CC00914201900AD00298006841F60041CBF6E4
:10C7DC00FF710844B0FA80F0400901900198C0073D
:10C7EC0040B90298C06848B10298C068B0F5803F63
:10C7FC0003D303E00298C06800B107E041F6700073
:10C80C00C0F6020040F2D271F8F7C1F902988069C3
:10C81C0018B102988069802800D107E041F67000B9
:10C82C00C0F6020040F2D371F8F7B1F9029890F813
:10C83C003D0030B90299002081F83C00029809F0C3
:10C84C002AFA0299022081F83D00029951F8040B52
:10C85C00FFF7C4FC0299012081F8480002990120DD
:10C86C0081F83E00029981F83F00029981F840005E
:10C87C00029981F84100029981F84200029981F8ED
:10C88C0043000299012081F84400029981F8450087
:10C89C00029981F84600029981F84700029901201B
:10C8AC0081F83D0000208DF80F009DF80F0004B0BA
:02C8BC0080BD3D
:10C8BE0080B584B0039003980068C0680290039816
:10C8CE000068006901909DF80400800700281ED5BD
:10C8DE009DF808008007002819D5039801686FF0AD
:10C8EE0002000861039901200877039800688069A7
:10C8FE00800718B1039809F0CDF905E0039809F007
:10C90E00C9F9039809F0C6F90399002008779DF834
:10C91E000400400700281FD59DF808004007002896
:10C92E001AD5039801686FF004000861039902207C
:10C93E00087703980068806910F4407F03D003984D
:10C94E0009F0A8F905E0039809F0A4F9039809F095
:10C95E00A1F90399002008779DF80400000700282C
:10C96E001ED59DF808000007002819D50398016808
:10C97E006FF0080008610399042008770398006897
:10C98E00C069800718B1039809F084F905E003988F
:10C99E0009F080F9039809F07DF9039900200877D2
:10C9AE009DF80400C00600281FD59DF80800C0069B
:10C9BE0000281AD5039801686FF0100008610399DA
:10C9CE000820087703980068C06910F4407F03D0F0
:10C9DE00039809F05FF905E0039809F05BF90398F5
:10C9EE0009F058F90399002008779DF80400C00754
:10C9FE0058B19DF80800C00738B1039801686FF070
:10CA0E0001000861039809F0ABFB019800F080006B
:10CA1E00802804D09DF80500800600280CD59DF8CE
:10CA2E0008000006002807D5039801686FF402502D
:10CA3E000861039809F02EF99DF80500C00760B152
:10CA4E009DF808000006002807D5039801686FF4CA
:10CA5E0080700861039809F01DF99DF804004006E6
:10CA6E0000280CD59DF808004006002807D503982D
:10CA7E0001686FF040000861039809F00BF99DF80A
:10CA8E000400800600280CD59DF8080080060028BA
:10CA9E0007D5039801686FF020000861039809F02C
:06CAAE00F9F804B080BDA0
:10CAB40080B586B0059004910598006A02900599A6
:10CAC400086A20F001000862059840680190059802
:10CAD4008069039003984FF68F71CFF6FE7108407A
:10CAE4000390039820F003000390049801680398CE
:10CAF40008430390029820F0020002900498816891
:10CB040002980843029005980021C4F2010188426A
:10CB14001BD0059840F20041C4F20101884214D0B0
:10CB2400059844F20001C4F2010188420DD0059831
:10CB340044F20041C4F20101884206D0059844F64B
:10CB44000001C4F2010188421CD10498C06818B1E4
:10CB54000498C068082800D107E041F67000C0F6C8
:10CB6400020041F66B31F8F716F8029820F008003D
:10CB740002900498C168029808430290029820F039
:10CB84000400029005980021C4F2010188421BD0E0
:10CB9400059840F20041C4F20101884214D005987E
:10CBA40044F20001C4F2010188420DD0059844F218
:10CBB4000041C4F20101884206D0059844F6000100
:10CBC400C4F20101884233D104988069B0F5007F32
:10CBD40002D00498806900B907E041F67000C0F6FD
:10CBE400020041F67831F7F7D6FF04984069B0F5B2
:10CBF400807F02D00498406900B907E041F67000D4
:10CC0400C0F6020041F67931F7F7C5FF019820F428
:10CC140080700190019820F400700190049841699B
:10CC24000198084301900498816901980843019090
:10CC340001980599486003980599886104984068AB
:0ECC44000599486302980599086206B080BD04
:10CC520080B586B0059004910598006A0290059906
:10CC6200086A20F48070086205984068019005986F
:10CC7200C069039003984FF68F71CFF6FE7108409A
:10CC82000390039820F0030003900498016803982E
:10CC920008430390029820F400700290049881687F
:10CCA200029840EA0120029005980021C4F2010195
:10CCB200884221D0059840F20041C4F20101884225
:10CCC2001AD0059844F20001C4F20101884201D150
:10CCD200002088B9059844F20041C4F2010188425B
:10CCE20001D1002040B9059844F60001C4F20101C7
:10CCF20088421FD10120E8B90498C06818B104988D
:10CD0200C068082800D107E041F67000C0F60200B2
:10CD120041F60241F7F740FF029820F400600290CA
:10CD22000498C168029840EA01200290029820F417
:10CD32008060029005980021C4F2010188421BD054
:10CD4200059840F20041C4F20101884214D00598CE
:10CD520044F20001C4F2010188420DD0059844F268
:10CD62000041C4F20101884206D0059844F6000150
:10CD7200C4F20101884235D104988069B0F5007F80
:10CD820002D00498806900B907E041F67000C0F64D
:10CD9200020041F60F41F7F7FFFE04984069B0F533
:10CDA200807F02D00498406900B907E041F6700024
:10CDB200C0F6020041F61041F7F7EEFE019820F4AA
:10CDC20080500190019820F400500190049841692C
:10CDD200019840EA0110019004988169019840EAA3
:10CDE2000110019001980599486003980599C8615E
:10CDF200049840680599C86302980599086206B0CC
:02CE020080BDF1
:10CE040080B586B0059004910598006A0290059952
:10CE1400086A20F4805008620598406801900598DB
:10CE2400C0690390039848F6FF71CFF6FF6108408C
:10CE34000390039820F440700390049801680398C9
:10CE440040EA01200390029820F4005002900498D4
:10CE54008168029840EA0130029005980021C4F2EA
:10CE6400010188421BD0059840F20041C4F201013F
:10CE7400884214D0059844F20001C4F201018842AA
:10CE84000DD0059844F20041C4F20101884206D055
:10CE9400059844F60001C4F2010188421AD10498AD
:10CEA4004069B0F5807F02D00498406900B907E07A
:10CEB40041F67000C0F6020041F64F41F7F76BFEF1
:10CEC400019820F48040019004984169019840EA57
:10CED4008110019001980599486003980599C861EB
:10CEE400049840680599086402980599086206B098
:02CEF40080BDFF
:10CEF60085B0049003910498006A01900499086A29
:10CF060020F4801008620498406800900498406DF0
:10CF16000290029848F6FF71CFF6FF610840029032
:10CF260003980168029840EA01200290019820F4D3
:10CF36000010019003988168019840EA0150019021
:10CF460004980021C4F2010188421BD0049840F2E3
:10CF56000041C4F20101884214D0049844F2000151
:10CF6600C4F2010188420DD0049844F20041C4F293
:10CF76000101884206D0049844F60001C4F201017A
:10CF8600884209D1009820F48020009003984169D6
:10CF9600009840EA81200090009804994860029821
:10CFA60004994865039840680499C86501980499EE
:06CFB600086205B070479F
:10CFBC0080B586B004900391029200208DF8070092
:10CFCC00049800680021C4F20101884264D00498DE
:10CFDC000068B0F1804F5FD00498006840F20041C7
:10CFEC00C4F20001884257D00498006840F6000152
:10CFFC00C4F2000188424FD00498006840F600410A
:10D00C00C4F20001884247D00498006840F2004105
:10D01C00C4F2010188423FD00498006841F6000137
:10D02C00C4F20001884237D00498006841F60041F0
:10D03C00C4F2000188422FD00498006842F200012B
:10D04C00C4F20001884227D00498006844F2000121
:10D05C00C4F2010188421FD00498006844F20041D8
:10D06C00C4F20101884217D00498006844F600010C
:10D07C00C4F2010188420FD0049800684EF20001FE
:10D08C00C4F20001884207D0049800684EF20041B7
:10D09C00C4F20001884200D107E041F67000C0F6EE
:10D0AC00020041F24C01F7F772FD0398006838B1A9
:10D0BC0003980068022803D0039800680A2800D15E
:10D0CC0007E041F67000C0F6020041F24D01F7F79F
:10D0DC005EFD03984068012807D003984068022839
:10D0EC0003D003984068032800D107E041F6700094
:10D0FC00C0F6020041F24E01F7F749FD0398806833
:10D10C0058B103988068042807D0039880680828D1
:10D11C0003D0039880680C2800D107E041F670001A
:10D12C00C0F6020041F24F01F7F731FD0398C068D9
:10D13C000F2800D807E041F67000C0F6020041F25B
:10D14C005001F7F724FD049890F83C00012803D116
:10D15C0002208DF8170052E10499012081F83C005F
:10D16C000298A8B904980068039B19685A68DB6890
:10D17C0000F049F904980168886920F00C00886176
:10D18C0003988268049801688869104388612EE1CD
:10D19C00029804286BD1049800680021C4F20101A4
:10D1AC00884244D004980068B0F1804F3FD0049876
:10D1BC00006840F20041C4F20001884237D0049864
:10D1CC00006840F60001C4F2000188422FD0049898
:10D1DC00006840F60041C4F20001884227D0049850
:10D1EC00006840F20041C4F2010188421FD004984B
:10D1FC00006841F60001C4F20001884217D004987F
:10D20C00006844F20001C4F2010188420FD0049876
:10D21C0000684EF20001C4F20001884207D0049865
:10D22C0000684EF20041C4F20001884200D107E0D0
:10D23C0041F67000C0F6020041F26601F7F7A7FC58
:10D24C0004980068039B19685A68DB680DF0F9F9BB
:10D25C0004980168886920F44060886103988268AA
:10D26C0004980168886940EA02208861BFE002984E
:10D27C0008285AD1049800680021C4F201018842A0
:10D28C0034D004980068B0F1804F2FD00498006817
:10D29C0040F20041C4F20001884227D00498006893
:10D2AC0040F60001C4F2000188421FD004980068C7
:10D2BC0040F60041C4F20001884217D0049800687F
:10D2CC0040F20041C4F2010188420FD0049800687A
:10D2DC004EF20001C4F20001884207D004980068A5
:10D2EC004EF20041C4F20001884200D107E041F641
:10D2FC007000C0F6020041F27601F7F748FC049882
:10D30C000068039B19685A68DB6800F00FF90498F1
:10D31C000168C86920F00C00C86103988268049801
:10D32C000168C8691043C86161E002980C285BD1A0
:10D33C00049800680021C4F20101884234D004989A
:10D34C000068B0F1804F2FD00498006840F2004183
:10D35C00C4F20001884227D00498006840F600010E
:10D36C00C4F2000188421FD00498006840F60041C6
:10D37C00C4F20001884217D00498006840F20041C2
:10D38C00C4F2010188420FD0049800684EF20001EB
:10D39C00C4F20001884207D0049800684EF20041A4
:10D3AC00C4F20001884200D107E041F67000C0F6DB
:10D3BC00020041F28601F7F7EAFB04980068039B30
:10D3CC0019685A68DB680DF072F904980168C8692D
:10D3DC0020F44060C8610398826804980168C869A9
:10D3EC0040EA0220C86102E001208DF80700049990
:10D3FC00002081F83C009DF807008DF817009DF87F
:06D40C00170006B080BD10
:10D4120087B006900591049203930698006A0190E2
:10D422000699086A20F00100086206988069029055
:10D43200069901200022C4F20102914200904ED0CE
:10D4420006990120B1F1804F009048D00699012041
:10D4520040F20042C4F20002914200903FD006998D
:10D46200012040F60002C4F200029142009036D040
:10D472000699012040F60042C4F200029142009057
:10D482002DD00699012040F20042C4F201029142DD
:10D49200009024D00699012041F60002C4F2000255
:10D4A200914200901BD00699012044F20002C4F27E
:10D4B20001029142009012D0069901204EF2000220
:10D4C200C4F200029142009009D0069841F6004150
:10D4D200CBF6FF710844B0FA80F040090090009842
:10D4E200C00740B1029820F003000290049902980C
:10D4F2000843029003E0029840F001000290029873
:10D5020020F0F000029003980001C1B20298084393
:10D512000290019820F00A000190059800F00A019B
:10D52200019808430190029806998861019806992A
:06D53200086207B070471B
:10D5380086B005900491039202930598006A0090C2
:10D548000599086A20F4807008620598C0690190FE
:10D55800019820F003000190039901980843019075
:10D56800019820F0F000019002980001C1B20198E2
:10D5780008430190009820F420600090049800F07F
:10D588000A01009840EA0120009001980599C861B5
:0AD5980000980599086206B070477C
:10D5A20080B586B00490039100208DF80B0004989A
:10D5B20090F83C00012804D102208DF8170000F0F9
:10D5C20060BC0499012081F83C000499022081F892
:10D5D2003D0003980068B0F5805F23D0039800688F
:10D5E20070281FD003980068B0F5005F1AD0039826
:10D5F2000068402816D003980068502812D003987B
:10D60200006860280ED00398006858B1039800683B
:10D61200102807D003980068202803D003980068D8
:10D62200302800D107E041F67000C0F6020041F256
:10D632005151F7F7B1FA0498006880680190019897
:10D642004FF68871CFF6CE7108400190019820F410
:10D652007F400190019804990968886003980068E6
:10D662000090002800F0A2830098102800F09E830A
:10D672000098202800F09A830098302800F09683C2
:10D682000098402800F007830098502800F0ED81B0
:10D692000098602800F074820098702800F0AF8033
:10D6A2000098B0F5805F24D00098B0F5005F00F0DC
:10D6B20044810098B0F5801F00F078830098B0F1A3
:10D6C200101F00F0738300982021C0F210018842DD
:10D6D20000F06C8300983021C0F21001884200F003
:10D6E200658300984021C0F21001884200F05E83F9
:10D6F200B8E3049800680021C4F20101884274D0A2
:10D7020004980068B0F1804F6FD00498006840F22E
:10D712000041C4F20001884267D00498006840F6D4
:10D722000001C4F2000188425FD00498006840F60C
:10D732000041C4F20001884257D00498006841F2C7
:10D742000001C4F2000188424FD00498006841F2FF
:10D752000041C4F20001884247D00498006840F2B8
:10D762000041C4F2010188423FD00498006841F6AA
:10D772000001C4F20001884237D00498006841F6E3
:10D782000041C4F2000188422FD00498006842F29E
:10D792000001C4F20001884227D00498006844F2D4
:10D7A2000001C4F2010188421FD00498006844F2CB
:10D7B2000041C4F20101884217D00498006844F67F
:10D7C2000001C4F2010188420FD0049800684EF2B1
:10D7D2000001C4F20001884207D0049800684EF2AA
:10D7E2000041C4F20001884200D107E041F6700016
:10D7F200C0F6020041F25D51F7F7CEF935E3049825
:10D8020000680021C4F20101884234D00498006803
:10D81200B0F1804F2FD00498006840F20041C4F26A
:10D822000001884227D00498006840F60001C4F243
:10D83200000188421FD00498006840F60041C4F2FB
:10D842000001884217D00498006840F20041C4F2F7
:10D85200010188420FD0049800684EF20001C4F220
:10D862000001884207D0049800684EF20041C4F2D9
:10D872000001884200D107E041F67000C0F60200C4
:10D8820041F26451F7F788F90398806870B1039800
:10D892008068B0F5805F09D003988068B0F5005FBA
:10D8A20004D003988068B0F5405F00D107E041F6EC
:10D8B2007000C0F6020041F26751F7F76DF9039864
:10D8C2004068B0F5004F0DD00398406850B10398FE
:10D8D200406838B103984068022803D00398406832
:10D8E2000A2800D107E041F67000C0F6020041F2BA
:10D8F2006851F7F751F90398C0680F2800D807E07C
:10D9020041F67000C0F6020041F26951F7F744F99E
:10D9120004980068039B5A689968DB680CF002FF60
:10D922000498006880680190019840F077000190A7
:10D93200019804990968886097E2049800680021B8
:10D94200C4F20101884234D004980068B0F1804FDB
:10D952002FD00498006840F20041C4F200018842CE
:10D9620027D00498006840F60001C4F20001884202
:10D972001FD00498006840F60041C4F200018842BA
:10D9820017D00498006840F20041C4F201018842B5
:10D992000FD0049800684EF20001C4F200018842E0
:10D9A20007D0049800684EF20041C4F20001884298
:10D9B20000D107E041F67000C0F6020041F27C514E
:10D9C200F7F7EAF80398806870B103988068B0F5B9
:10D9D200805F09D003988068B0F5005F04D0039897
:10D9E2008068B0F5405F00D107E041F67000C0F6F4
:10D9F200020041F27F51F7F7CFF803984068B0F583
:10DA0200004F0DD00398406850B10398406838B178
:10DA120003984068022803D0039840680A2800D17E
:10DA220007E041F67000C0F602004FF4AC51F7F780
:10DA3200B3F80398C0680F2800D807E041F67000D9
:10DA4200C0F6020041F28151F7F7A6F80498006887
:10DA5200039B5A689968DB680CF064FE04980168BD
:10DA6200886840F480408860FFE1049800680021E3
:10DA7200C4F20101884244D004980068B0F1804F9A
:10DA82003FD00498006840F20041C4F2000188428D
:10DA920037D00498006840F60001C4F200018842C1
:10DAA2002FD00498006840F60041C4F20001884279
:10DAB20027D00498006840F20041C4F20101884274
:10DAC2001FD00498006841F60001C4F200018842A8
:10DAD20017D00498006844F20001C4F201018842A0
:10DAE2000FD0049800684EF20001C4F2000188428F
:10DAF20007D0049800684EF20041C4F20001884247
:10DB020000D107E041F67000C0F6020041F29051E8
:10DB1200F7F742F803984068B0F5004F0DD003982C
:10DB2200406850B10398406838B1039840680228B1
:10DB320003D0039840680A2800D107E041F670003C
:10DB4200C0F6020041F29351F7F726F80398C06835
:10DB52000F2800D807E041F67000C0F6020041F23B
:10DB62009451F7F719F804980068039A5168D2683B
:10DB72000CF0F2FD0498006850210CF015FE74E1DF
:10DB8200049800680021C4F20101884244D004983C
:10DB92000068B0F1804F3FD00498006840F2004125
:10DBA200C4F20001884237D00498006840F60001B0
:10DBB200C4F2000188422FD00498006840F6004168
:10DBC200C4F20001884227D00498006840F2004164
:10DBD200C4F2010188421FD00498006841F6000196
:10DBE200C4F20001884217D00498006844F2000190
:10DBF200C4F2010188420FD0049800684EF200017D
:10DC0200C4F20001884207D0049800684EF2004135
:10DC1200C4F20001884200D107E041F67000C0F66C
:10DC220002004FF4AD51F6F7B7FF03984068B0F524
:10DC3200004F0DD00398406850B10398406838B146
:10DC420003984068022803D0039840680A2800D14C
:10DC520007E041F67000C0F6020041F2A351F6F768
:10DC62009BFF0398C0680F2800D807E041F67000B8
:10DC7200C0F6020041F2A451F6F78EFF0498006844
:10DC8200039A5168D26800F000F904980068602194
:10DC92000CF08AFDE9E0049800680021C4F2010159
:10DCA200884244D004980068B0F1804F3FD0049875
:10DCB200006840F20041C4F20001884237D0049863
:10DCC200006840F60001C4F2000188422FD0049897
:10DCD200006840F60041C4F20001884227D004984F
:10DCE200006840F20041C4F2010188421FD004984A
:10DCF200006841F60001C4F20001884217D004987E
:10DD0200006844F20001C4F2010188420FD0049875
:10DD120000684EF20001C4F20001884207D0049864
:10DD220000684EF20041C4F20001884200D107E0CF
:10DD320041F67000C0F6020041F2B051F6F72CFF36
:10DD420003984068B0F5004F0DD00398406850B179
:10DD52000398406838B103984068022803D00398BA
:10DD620040680A2800D107E041F67000C0F60200C0
:10DD720041F2B351F6F710FF0398C0680F2800D89C
:10DD820007E041F67000C0F6020041F2B451F6F726
:10DD920003FF04980068039A5168D2680CF0DCFC17
:10DDA2000498006840210CF0FFFC5EE004980068D3
:10DDB2000021C4F20101884244D004980068B0F105
:10DDC200804F3FD00498006840F20041C4F2000145
:10DDD200884237D00498006840F60001C4F200017E
:10DDE20088422FD00498006840F60041C4F2000136
:10DDF200884227D00498006840F20041C4F2010131
:10DE020088421FD00498006841F60001C4F2000164
:10DE1200884217D00498006844F20001C4F201015C
:10DE220088420FD0049800684EF20001C4F200014B
:10DE3200884207D0049800684EF20041C4F2000103
:10DE4200884200D107E041F67000C0F6020041F2BC
:10DE5200C851F6F7A1FE04980068039909680CF00E
:10DE6200A3FC02E001208DF80B000499012081F847
:10DE72003D000499002081F83C009DF80B008DF8CC
:0ADE820017009DF8170006B080BDE0
:10DE8C0085B00490039102920498006A0090049962
:10DE9C00086A20F0100008620498806901900198CB
:10DEAC0020F4704001900299019840EA01300190F1
:10DEBC00009820F0A00000900399009840EA01100F
:10DECC00009001980499886100980499086205B043
:02DEDC0070478D
:10DEDE0080B584B002900191029800680021C4F2CE
:10DEEE000101884244D002980068B0F1804F3FD0C3
:10DEFE000298006840F20041C4F20001884237D017
:10DF0E000298006840F60001C4F2000188422FD04A
:10DF1E000298006840F60041C4F20001884227D002
:10DF2E000298006840F20041C4F2010188421FD0FD
:10DF3E000298006841F60001C4F20001884217D031
:10DF4E000298006844F20001C4F2010188420FD029
:10DF5E00029800684EF20001C4F20001884207D018
:10DF6E00029800684EF20041C4F20001884200D1CE
:10DF7E0007E041F67000C0F6020041F20861F6F7C4
:10DF8E0005FE01980068A0B101980068042810D021
:10DF9E000198006805280CD001980068062808D062
:10DFAE0001980068072804D001980068B0F5803FFA
:10DFBE0000D107E041F67000C0F6020041F209619F
:10DFCE00F6F7E4FD01984068002846D001984068B5
:10DFDE00102842D00198406820283ED00198406811
:10DFEE0030283AD001984068B0F5801F35D001989E
:10DFFE004068B0F1101F30D0019840682021C0F267
:10E00E001001884229D0019840683021C0F21001D9
:10E01E00884222D0019840684021C0F21001884207
:10E02E001BD001984068B0F5001F16D001984068CB
:10E03E001021C0F2200188420FD00198406840287C
:10E04E000BD001984068502807D00198406860288E
:10E05E0003D001984068702800D107E041F67000A7
:10E06E00C0F6020041F20A61F6F790FD029890F8B0
:10E07E003C00012803D102208DF80F002FE00299F9
:10E08E00012081F83C000299022081F83D0002989F
:10E09E00019900F028F858B10299012081F83D004D
:10E0AE000299002081F83C0001208DF80F0016E047
:10E0BE0002980168C86820F04000C86002980168A4
:10E0CE00C86820F48040C8600299012081F83D00A4
:10E0DE000299002081F83C0000208DF80F009DF879
:06E0EE000F0004B080BD2C
:10E0F40080B588B00690059100208DF8130006982D
:10E1040000688068039003984FF68F71CFF6CF7143
:10E1140008400390059841680398084303900398C6
:10E124004FF6F871CFF6FE71084003900598016828
:10E134000398084303900398069909688860059832
:10E1440040680090002800F0C5820098102800F074
:10E15400C1820098202800F0BD820098302800F089
:10E16400B9820098402800F0DE800098502800F022
:10E1740085810098602800F027820098702840D09C
:10E184000098B0F5801F00F0A5820098B0F1101F30
:10E1940000F0A08200982021C0F21001884200F013
:10E1A400998200983021C0F21001884200F09282D6
:10E1B40000984021C0F21001884200F08B82009840
:10E1C4005021C0F21001884200F08482009860213E
:10E1D400C0F21001884200F07D8200987021C0F2E4
:10E1E4001001884200F076820098B0F5001F00F01C
:10E1F400718200981021C0F22001884200F06A82E6
:10E20400BEE2069800680021C4F20101884234D0BD
:10E2140006980068B0F1804F2FD00698006840F24D
:10E224000041C4F20001884227D00698006840F6F5
:10E234000001C4F2000188421FD00698006840F62D
:10E244000041C4F20001884217D00698006840F2E9
:10E254000041C4F2010188420FD0069800684EF2D2
:10E264000001C4F20001884207D0069800684EF20B
:10E274000041C4F20001884200D107E041F6700079
:10E28400C0F6020041F6F641F6F785FC0598C06831
:10E2940070B10598C068B0F5805F09D00598C06872
:10E2A400B0F5005F04D00598C068B0F5405F00D1B8
:10E2B40007E041F67000C0F6020041F6F741F6F7B8
:10E2C4006AFC05988068B0F5004F0DD00598806809
:10E2D40050B10598806838B105988068022803D049
:10E2E400059880680A2800D107E041F67000C0F65E
:10E2F400020041F6F841F6F74EFC059800690F2834
:10E3040000D807E041F67000C0F6020041F6F9417A
:10E31400F6F741FC06980068059B9A68D9681B6962
:10E324000CF0FFF92FE2069800680021C4F2010105
:10E33400884264D006980068B0F1804F5FD0069898
:10E34400006840F20041C4F20001884257D00698A8
:10E35400006840F60001C4F2000188424FD00698DC
:10E36400006840F60041C4F20001884247D0069894
:10E37400006840F20041C4F2010188423FD006988F
:10E38400006841F60001C4F20001884237D00698C3
:10E39400006841F60041C4F2000188422FD006987B
:10E3A400006842F20001C4F20001884227D00698B6
:10E3B400006844F20001C4F2010188421FD00698AB
:10E3C400006844F20041C4F20101884217D0069863
:10E3D400006844F60001C4F2010188420FD0069897
:10E3E40000684EF20001C4F20001884207D006988A
:10E3F40000684EF20041C4F20001884200D107E0F7
:10E4040041F67000C0F6020041F60551F6F7C3FB71
:10E41400059800690F2800D807E041F67000C0F69F
:10E42400020041F60651F6F7B6FB05980068052888
:10E4340003D101208DF81F00A9E106980068006A45
:10E44400019006980168086A20F0010008620698A5
:10E45400006880690290029820F0F000029005980C
:10E464000169029840EA011002900298069909682D
:10E474008861019806990968086284E10698006831
:10E484000021C4F20101884264D006980068B0F10A
:10E49400804F5FD00698006840F20041C4F200014A
:10E4A400884257D00698006840F60001C4F2000183
:10E4B40088424FD00698006840F60041C4F200013B
:10E4C400884247D00698006840F20041C4F2010136
:10E4D40088423FD00698006841F60001C4F200016A
:10E4E400884237D00698006841F60041C4F2000122
:10E4F40088422FD00698006842F20001C4F200015D
:10E50400884227D00698006844F20001C4F2010151
:10E5140088421FD00698006844F20041C4F2010109
:10E52400884217D00698006844F60001C4F201013D
:10E5340088420FD0069800684EF20001C4F2000130
:10E54400884207D0069800684EF20041C4F20001E8
:10E55400884200D107E041F67000C0F6020041F69F
:10E564001F51F6F718FB05988068B0F5004F0DD0E1
:10E574000598806850B10598806838B1059880681E
:10E58400022803D0059880680A2800D107E041F6E4
:10E594007000C0F602004FF4E951F6F7FCFA059852
:10E5A40000690F2800D807E041F67000C0F60200A9
:10E5B40041F62151F6F7EFFA06980068059A91683A
:10E5C40012690CF0C8F8DEE0069800680021C4F275
:10E5D4000101884244D006980068B0F1804F3FD0D2
:10E5E4000698006840F20041C4F20001884237D026
:10E5F4000698006840F60001C4F2000188422FD05A
:10E604000698006840F60041C4F20001884227D011
:10E614000698006840F20041C4F2010188421FD00C
:10E624000698006841F60001C4F20001884217D040
:10E634000698006844F20001C4F2010188420FD038
:10E64400069800684EF20001C4F20001884207D027
:10E65400069800684EF20041C4F20001884200D1DD
:10E6640007E041F67000C0F6020041F62D51F6F7BE
:10E6740092FA05988068B0F5004F0DD0059880682F
:10E6840050B10598806838B105988068022803D095
:10E69400059880680A2800D107E041F67000C0F6AA
:10E6A400020041F62E51F6F776FA059800690F2814
:10E6B40000D807E041F67000C0F6020041F62F5181
:10E6C400F6F769FA06980068059A91681269FFF7E7
:10E6D400DBFB58E0069800680021C4F2010188427F
:10E6E40044D006980068B0F1804F3FD00698006887
:10E6F40040F20041C4F20001884237D00698006815
:10E7040040F60001C4F2000188422FD00698006848
:10E7140040F60041C4F20001884227D00698006800
:10E7240040F20041C4F2010188421FD006980068FB
:10E7340041F60001C4F20001884217D0069800682F
:10E7440044F20001C4F2010188420FD00698006827
:10E754004EF20001C4F20001884207D00698006816
:10E764004EF20041C4F20001884200D107E041F6B4
:10E774007000C0F6020041F64851F6F70CFA02E0C8
:10E7840001208DF813009DF813008DF81F009DF8EB
:06E794001F0008B080BD6B
:10E79A0080B582B00090009818B901208DF8070062
:10E7AA0001E100988069002861D00098006841F270
:10E7BA000001C4F2010188424FD00098006844F277
:10E7CA000041C4F20001884247D00098006844F62C
:10E7DA000001C4F2000188423FD00098006844F664
:10E7EA000041C4F20001884237D00098006845F21F
:10E7FA000001C4F2000188422FD00098006841F25B
:10E80A000041C4F20101884227D00098006847F607
:10E81A000001C4F2000188421FD00098006847F640
:10E82A000041C4F20001884217D00098006841F6FE
:10E83A000001C4F2010188420FD00098006841F635
:10E84A000041C4F20101884207D00098006840F6EE
:10E85A000041C5F60001884200D107E042F25C207F
:10E86A00C0F602004FF49F71F6F792F960E0009843
:10E87A00006841F20001C4F2010188424FD00098B9
:10E88A00006844F20041C4F20001884247D000986F
:10E89A00006844F60001C4F2000188423FD00098A3
:10E8AA00006844F60041C4F20001884237D000985B
:10E8BA00006845F20001C4F2000188422FD0009896
:10E8CA00006841F20041C4F20101884227D0009851
:10E8DA00006847F60001C4F2000188421FD0009880
:10E8EA00006847F60041C4F20001884217D0009838
:10E8FA00006841F60001C4F2010188420FD0009875
:10E90A00006841F60041C4F20101884207D000982C
:10E91A00006840F60041C5F60001884200D107E0D0
:10E92A0042F25C20C0F6020040F24311F6F730F9D9
:10E93A000098D0F8880030B90099002081F8840046
:10E94A00009807F08BFF00992420C1F888000098EE
:10E95A000168086820F0010008600098806A10B118
:10E96A00009800F024F80098F6F717F9012803D167
:10E97A0001208DF8070016E000980168486820F425
:10E98A009040486000980168886820F02A008860F2
:10E99A0000980168086840F00100086000980CF0CF
:0EE9AA00BBF88DF807009DF8070002B080BD95
:10E9B80080B582B001900198806AFF2800D807E0EE
:10E9C80042F25C20C0F602004FF44E61F6F7E1F81F
:10E9D800019890F82800000700281AD50198806B44
:10E9E80020B10198806BB0F5004F00D107E042F2EA
:10E9F8005C20C0F6020040F6E541F6F7CAF8019837
:10EA08000068406820F40040019A1168926B104336
:10EA18004860019890F82800C007D0B10198C06AF2
:10EA280020B10198C06AB0F5003F00D107E042F27A
:10EA38005C20C0F6020040F6EC41F6F7AAF801980F
:10EA48000068406820F40030019A1168D26A1043C7
:10EA58004860019890F82800800700281AD5019886
:10EA6800006B20B10198006BB0F5803F00D107E042
:10EA780042F25C20C0F6020040F6F341F6F789F84E
:10EA880001980068406820F48030019A1168126B80
:10EA980010434860019890F82800400700281AD5CC
:10EAA8000198406B20B10198406BB0F5802F00D1E0
:10EAB80007E042F25C20C0F6020040F6FA41F6F7A1
:10EAC80068F801980068406820F48020019A11686D
:10EAD800526B10434860019890F82800C00600283F
:10EAE8001AD50198C06B20B10198C06BB0F5805F52
:10EAF80000D107E042F25C20C0F6020040F6015166
:10EB0800F6F747F801980068806820F48050019A69
:10EB18001168D26B10438860019890F8280080062D
:10EB280000281AD50198006C20B10198006CB0F546
:10EB3800005F00D107E042F25C20C0F6020040F618
:10EB48000851F6F726F801980068806820F400500C
:10EB5800019A1168126C10438860019890F8280097
:10EB68004006002840F19E800198006841F20001AB
:10EB7800C4F20101884247D00198006844F200417C
:10EB8800C4F2000188423FD00198006844F60001B1
:10EB9800C4F20001884237D00198006844F6004169
:10EBA800C4F2000188422FD00198006845F20001A4
:10EBB800C4F20001884227D00198006841F2004160
:10EBC800C4F2010188421FD00198006847F600018D
:10EBD800C4F20001884217D00198006847F6004146
:10EBE800C4F2000188420FD00198006841F6000184
:10EBF800C4F20101884207D00198006841F600413B
:10EC0800C4F20101884200D107E042F25C20C0F65C
:10EC1800020040F60F51F5F7BCFF0198406C20B197
:10EC28000198406CB0F5801F00D107E042F25C20EB
:10EC3800C0F602004FF45161F5F7ABFF0198006888
:10EC4800406820F48010019A1168526C10434860A3
:10EC58000198406CB0F5801F24D10198806C70B188
:10EC68000198806CB0F5001F09D00198806CB0F550
:10EC7800800F04D00198806CB0F5C00F00D107E078
:10EC880042F25C20C0F6020040F61551F5F781FF0C
:10EC980001980068406820F4C000019A1168926CDD
:10ECA80010434860019890F82800000600281AD5FB
:10ECB8000198C06C20B10198C06CB0F5002F00D14C
:10ECC80007E042F25C20C0F6020040F61D51F5F75D
:10ECD80060FF01980068406820F40020019A1168DC
:0AECE800D26C1043486002B080BDFA
:10ECF20080B586B0DDF820C0049003918DF80B201A
:10ED0200019304980068C06903990840401AB0FA58
:10ED120080F040099DF80B10884253D108980130C9
:10ED220000284ED007F0DCFE0199401A089988426B
:10ED320001D8089818B903208DF8170045E0049807
:10ED420000680068400700283BD50398802838D027
:10ED52000398402835D004980068C069C0F3C00009
:10ED6200012813D1049801680820009008620498D1
:10ED72000BF07EFF00980499C1F8900004990020DE
:10ED820081F8840001208DF817001EE004980068C5
:10ED9200C069C0F3C020012813D1049801684FF460
:10EDA2000060086204980BF063FF04992020C1F808
:10EDB20090000499002081F8840003208DF8170048
:10EDC20003E09EE700208DF817009DF8170006B0BB
:02EDD20080BD02
:10EDD4008EB003900398D0F8880021285BD1039863
:10EDE400B0F86A00ADF80A00BDF80A00002852D055
:10EDF4000398B0F8560090BB039800680830079059
:10EE0400079850E8000F0690069820F4000001903F
:10EE140001990398006808300D910C900C990D9A93
:10EE240041E800200B900B980028E5D10398006876
:10EE34000590059850E8000F0490049840F04000B5
:10EE440000900099039800680A91099009990A9A18
:10EE540041E80020089008980028E7D11BE00398B7
:10EE64000068C069000600280FD503980168006D8A
:10EE7400007888620399086D013008650399B1F838
:10EE840056000138A1F85600FFE7BDF80A00013822
:0AEE9400ADF80A00A8E70EB07047C1
:10EE9E008DB002900298D0F88800212843D10298B4
:10EEAE00B0F8560080BB029800680690069850E8AD
:10EEBE00000F0590059820F08000019001990298AE
:10EECE0000680C910B900B990C9A41E800200A9067
:10EEDE000A980028E7D1029800680490049850E838
:10EEEE00000F0390039840F04000009000990298A4
:10EEFE000068099108900899099A41E80020079046
:10EF0E0007980028E7D10EE002980168006D00789E
:10EF1E0088620299086D013008650299B1F85600B1
:0AEF2E000138A1F856000DB070473D
:10EF380080B58AB003900291ADF806200398D0F806
:10EF48008C0020283AD1029810B1BDF8060018B9F3
:10EF580001208DF8130034E003990020C866039857
:10EF6800006840F60041C5F6000188421DD00398AC
:10EF7800006840680002002817D5039800680690CA
:10EF8800069850E8000F0590059840F080600090C2
:10EF9800009903980068099108900899099A41E82E
:10EFA8000020079007980028E7D103980299BDF838
:10EFB800062000F00AF88DF8130002E002208DF810
:0AEFC80013009DF813000AB080BD8D
:10EFD200A1B007900691ADF81620069807998865AA
:10EFE200BDF816000799A1F85C00BDF81600079954
:10EFF200A1F85E0007990020486707988068B0F57D
:10F00200805F0DD10798006928B9079940F2FF1077
:10F01200A1F8600003E00799FF20A1F8600025E055
:10F022000798806860B90798006920B90799FF209E
:10F03200A1F8600003E007997F20A1F8600015E0C5
:10F0420007988068B0F1805F0CD10798006920B9F9
:10F0520007997F20A1F8600003E007993F20A1F8FB
:10F06200600003E007990020A1F8600007990020E2
:10F07200C1F8900007992220C1F88C000798006817
:10F0820008301190119850E8000F1090109840F03D
:10F0920001000490049907980068083020911F909D
:10F0A2001F99209A41E800201E901E980028E5D161
:10F0B2000798406EB0F1005F51D1BDF81600079974
:10F0C200B1F8681088424ADB07988068B0F5805F23
:10F0D20009D10798006930B907994AF6D770C0F686
:10F0E2000100486705E007994BF2E320C0F60100F2
:10F0F200486707980069B8B1079800680F900F98A1
:10F1020050E8000F0E900E9840F48070039003991F
:10F11200079800681D911C901C991D9A41E80020D7
:10F122001B901B980028E7D10798006808300D90C3
:10F132000D9850E8000F0C900C9840F0805002900F
:10F1420002990798006808301A91199019991A9A29
:10F1520041E80020189018980028E5D148E0079867
:10F162008068B0F5805F09D10798006930B90799C6
:10F172004BF2EB50C0F60100486705E007994BF2ED
:10F182007F70C0F60100486707980069C0B1079810
:10F1920000680B900B9850E8000F0A900A9840F410
:10F1A200907001900199079800681791169016992E
:10F1B200179A41E80020159015980028E7D117E02A
:10F1C200079800680990099850E8000F089008987D
:10F1D20040F0200000900099079800681491139065
:10F1E2001399149A41E80020129012980028E7D14E
:06F1F200002021B070476F
:10F1F80080B5BAB0119011980068C0691090119844
:10F20800006800680F901198006880680E90109848
:10F2180040F60F0108400D900D98A8B99DF84000E0
:10F228008006002810D59DF83C008006002804D4EC
:10F238009DF83B00C006002806D51198406F10B114
:10F248001198416F884726E30D98002800F0EF8059
:10F258000E980121C1F20001084207D10F9840F22F
:10F268002011C0F20041084200F0E1809DF8400002
:10F27800C00770B19DF83D00C00750B111980168F2
:10F28800012008621199D1F8900040F00100C1F8FE
:10F2980090009DF84000800700280ED59DF83800A2
:10F2A800C00750B111980168022008621199D1F87D
:10F2B800900040F00400C1F890009DF8400040071D
:10F2C80000280ED59DF83800C00750B11198016884
:10F2D800042008621199D1F8900040F00200C1F8AA
:10F2E80090009DF840000007002815D59DF83C00C7
:10F2F8008006002805D40E980121C1F200010842B9
:10F308000AD011980168082008621199D1F8900074
:10F3180040F00800C1F890009DF84100000700285F
:10F3280010D59DF83F00400700280BD511980168BB
:10F338004FF4006008621199D1F8900040F0200065
:10F34800C1F890001198D0F8900000286ED09DF870
:10F358004000800600280FD59DF83C008006002854
:10F3680004D49DF83B00C006002805D51198406FCD
:10F3780010B11198416F88471198D0F890000C90FF
:10F3880011980068806800F04000402804D09DF87B
:10F39800300010F0280F42D011980BF066FC11983D
:10F3A800006880684006002835D511980068083044
:10F3B8002190219850E8000F2090209820F04000DC
:10F3C8000B900B991198006808303991389038994A
:10F3D800399A41E80020379037980028E5D11198EC
:10F3E800D0F8800098B11198D0F880104FF6A3009B
:10F3F800C0F6000008651198D0F8800007F027FED5
:10F4080020B11198D0F88000016D884702E011986A
:10F4180006F043FC02E0119806F03FFC06E0119864
:10F4280006F03BFC11990020C1F8900033E21198D6
:10F43800C06E012840F0DE819DF84000C00600281B
:10F4480040F1D8819DF83C00C006002840F1D281E7
:10F4580011980168102008621198006880684006B9
:10F46800002840F157811198D0F8800000681021D9
:10F47800C4F20201884200F090801198D0F8800010
:10F4880000682821C4F20201884200F086801198A1
:10F49800D0F8800000684021C4F2020188427CD084
:10F4A8001198D0F8800000685821C4F202018842FF
:10F4B80073D01198D0F8800000687021C4F202015E
:10F4C80088426AD01198D0F8800000688821C4F278
:10F4D8000201884261D01198D0F880000068A0210C
:10F4E800C4F20201884258D01198D0F88000006810
:10F4F800B821C4F2020188424FD01198D0F8800098
:10F50800006840F21041C4F20201884245D01198C7
:10F51800D0F88000006840F22841C4F20201884215
:10F528003BD01198D0F88000006840F24041C4F206
:10F538000201884231D01198D0F88000006840F26A
:10F548005841C4F20201884227D01198D0F88000AF
:10F55800006840F27041C4F2020188421DD011983F
:10F56800D0F88000006840F28841C4F20201884265
:10F5780013D01198D0F88000006840F2A041C4F27E
:10F588000201884209D01198D0F88000006840F242
:10F59800B841C4F20201884206D11198D0F880001F
:10F5A80000684068019005E01198D0F88000006874
:10F5B800406801900198ADF82A00BDF82A0000289B
:10F5C80000F09180BDF82A001199B1F85C108842CA
:10F5D80080F28980BDF82A001199A1F85E0011987F
:10F5E800D0F88000C069B0F5807F6FD011980068AE
:10F5F8001F901F9850E8000F1E901E9820F48070EE
:10F608000990099911980068369135903599369A7C
:10F6180041E80020349034980028E7D11198006818
:10F6280008301D901D9850E8000F1C901C9820F081
:10F6380001000890089911980068083033913290B9
:10F648003299339A41E80020319031980028E5D169
:10F658001198006808301B901B9850E8000F1A900A
:10F668001A9820F040000790079911980068083010
:10F6780030912F902F99309A41E800202E902E98A3
:10F688000028E5D111992020C1F88C00119900209B
:10F69800C866119800681990199850E8000F1890DA
:10F6A800189820F0100006900699119800682D917E
:10F6B8002C902C992D9A41E800202B902B9800280B
:10F6C800E7D11198D0F88000F7F7D4FF11990220FC
:10F6D80008671198B0F85C10B0F85E20891A89B2F2
:10F6E80006F093FF15E0BDF82A001199B1F85C10F7
:10F6F80088420ED11198D0F88000C069B0F5807F9B
:10F7080007D11199022008671198B0F85C1006F02B
:10F718007CFFC0E01199B1F85C00B1F85E10401AA6
:10F72800ADF816001198B0F85E00002861D0BDF859
:10F73800160000285DD0119800681790179850E8B7
:10F74800000F1690169820F4907004900499119860
:10F7580000682A91299029992A9A41E8002028903E
:10F7680028980028E7D11198006808301590159856
:10F7780050E8000F149014984FF6FE71CEF6FF7102
:10F788000840039003991198006808302791269043
:10F798002699279A41E80020259025980028E2D14B
:10F7A80011992020C1F88C0011990020C866119980
:10F7B8004867119800681390139850E8000F12904A
:10F7C800129820F010000290029911980068249174
:10F7D80023902399249A41E8002022902298002817
:10F7E800E7D11199022008671198BDF8161006F0A4
:10F7F8000CFF50E09DF84200C00600280DD59DF88A
:10F808003A004006002808D5119801684FF4801086
:10F818000862119806F041FA3DE09DF840000006A4
:10F82800002810D59DF83C000006002804D49DF857
:10F838003A000006002806D51198806F10B111987B
:10F84800816F884727E09DF840004006002808D5CA
:10F858009DF83C004006002803D5119800F02CF8CC
:10F8680019E09DF842000006002808D59DF83F00E1
:10F878004006002803D5119806F00FFA0BE09DF812
:10F888004300C00738B19DF83F000006002802D5A4
:0AF89800119806F002FA3AB080BDA4
:10F8A20080B582B001900198806B00900099002091
:0EF8B200A1F85E00009806F0F3F902B080BDE8
:10F8C00080B588B00290029800680490049850E8CF
:10F8D000000F0390039820F04000019001990298D6
:10F8E0000068079106900699079A41E80020059064
:10F8F00005980028E7D102992020C1F888000299D4
:0EF9000000208867029806F0CCF908B080BDA0
:10F90E0080B586B00490039102920193049818B9C1
:10F91E0001208DF81700D4E00498006841F2000130
:10F92E00C4F2010188424FD00498006844F20041AD
:10F93E00C4F20001884247D00498006844F60001E2
:10F94E00C4F2000188423FD00498006844F600419A
:10F95E00C4F20001884237D00498006845F20001D5
:10F96E00C4F2000188422FD00498006841F2004191
:10F97E00C4F20101884227D00498006847F60001BE
:10F98E00C4F2000188421FD00498006847F6004177
:10F99E00C4F20001884217D00498006841F60001B5
:10F9AE00C4F2010188420FD00498006841F600416C
:10F9BE00C4F20101884207D00498006840F6004165
:10F9CE00C5F60001884200D106E041F6D700C0F628
:10F9DE000200B121F5F7DAF8039818B10398B0F5E3
:10F9EE00004F00D106E041F6D700C0F60200B42168
:10F9FE00F5F7CCF802981F2800D806E041F6D7009C
:10FA0E00C0F60200B721F5F7C1F801981F2800D8FB
:10FA1E0006E041F6D700C0F60200BA21F5F7B6F8B7
:10FA2E000498D0F8880030B90499002081F8840039
:10FA3E00049806F011FF04992420C1F88800049858
:10FA4E000168086820F0010008600498806A10B10F
:10FA5E000498FEF7AAFF0498F5F79DF8012803D144
:10FA6E0001208DF817002CE004980168886840F496
:10FA7E008040886004980068806820F400400399F4
:10FA8E00084304990968886002984005009001991E
:10FA9E00009840EA014000900498006800686FF3F7
:10FAAE001940009908430499096808600498016890
:10FABE00086840F00100086004980BF02BF88DF8F0
:0AFACE0017009DF8170006B080BD78
:10FAD80082B001900198406E38B901990120A1F8CF
:10FAE8006A000199A1F8680031E010208DF8030040
:10FAF8008DF80200019800688068C0F342608DF8B4
:10FB08000100019800688068400F8DF800009DF89A
:10FB180002009DF8002042F2C423C0F60203995C5B
:10FB2800484342F2CC21C0F602018A5CB0FBF2F0F5
:10FB3800019AA2F86A009DF803009DF801209B5CD9
:10FB48005843895CB0FBF1F00199A1F8680002B054
:02FB58007047F4
:10FB5A0080B584B002900298006841F20001C4F2B4
:10FB6A00010188424FD00298006844F20041C4F271
:10FB7A000001884247D00298006844F60001C4F2A6
:10FB8A00000188423FD00298006844F60041C4F25E
:10FB9A000001884237D00298006845F20001C4F299
:10FBAA00000188422FD00298006841F20041C4F255
:10FBBA000101884227D00298006847F60001C4F282
:10FBCA00000188421FD00298006847F60041C4F23B
:10FBDA000001884217D00298006841F60001C4F279
:10FBEA00010188420FD00298006841F60041C4F230
:10FBFA000101884207D00298006840F60041C5F624
:10FC0A000001884200D107E041F6D700C0F60200A1
:10FC1A0040F23621F4F7BCFF029890F884000128DC
:10FC2A0003D102208DF80F0027E00299012081F804
:10FC3A00840002992420C1F88800029800680068AC
:10FC4A00019002980168086820F001000860019894
:10FC5A0020F000500190029900204866019802990C
:10FC6A000968086002992020C1F8880002990020DA
:10FC7A0081F8840000208DF80F009DF80F0004B071
:02FC8A0080BD3B
:10FC8C0080B584B0029001910298006841F20001A5
:10FC9C00C4F2010188424FD00298006844F200413E
:10FCAC00C4F20001884247D00298006844F6000173
:10FCBC00C4F2000188423FD00298006844F600412B
:10FCCC00C4F20001884237D00298006845F2000166
:10FCDC00C4F2000188422FD00298006841F2004122
:10FCEC00C4F20101884227D00298006847F600014F
:10FCFC00C4F2000188421FD00298006847F6004108
:10FD0C00C4F20001884217D00298006841F6000145
:10FD1C00C4F2010188420FD00298006841F60041FC
:10FD2C00C4F20101884207D00298006840F60041F5
:10FD3C00C5F60001884200D107E041F6D700C0F6B5
:10FD4C0002004FF41971F4F722FF019898B1019851
:10FD5C00B0F1005F0FD00198B0F1804F0BD001983B
:10FD6C00B0F1C04F07D00198B0F1004F03D001980B
:10FD7C00B0F1204F00D107E041F6D700C0F60200E9
:10FD8C0040F26521F4F703FF029890F884000128F3
:10FD9C0003D102208DF80F002DE00299012081F88B
:10FDAC00840002992420C1F8880002980068006839
:10FDBC00009002980168086820F001000860029821
:10FDCC000068806820F06040019908430299096836
:10FDDC0088600298FFF77AFE00980299096808601B
:10FDEC0002992020C1F888000299002081F8840033
:0EFDFC0000208DF80F009DF80F0004B080BDB0
:10FE0A0080B584B0029001910298006841F2000125
:10FE1A00C4F2010188424FD00298006844F20041BE
:10FE2A00C4F20001884247D00298006844F60001F3
:10FE3A00C4F2000188423FD00298006844F60041AB
:10FE4A00C4F20001884237D00298006845F20001E6
:10FE5A00C4F2000188422FD00298006841F20041A2
:10FE6A00C4F20101884227D00298006847F60001CF
:10FE7A00C4F2000188421FD00298006847F6004188
:10FE8A00C4F20001884217D00298006841F60001C6
:10FE9A00C4F2010188420FD00298006841F600417D
:10FEAA00C4F20101884207D00298006840F6004176
:10FEBA00C5F60001884200D107E041F6D700C0F636
:10FECA00020040F29521F4F763FE019898B1019877
:10FEDA00B0F1007F0FD00198B0F1806F0BD001987C
:10FEEA00B0F1C06F07D00198B0F1006F03D001984C
:10FEFA00B0F1206F00D107E041F6D700C0F602004A
:10FF0A0040F29621F4F744FE029890F88400012802
:10FF1A0003D102208DF80F002DE00299012081F80B
:10FF2A00840002992420C1F88800029800680068B9
:10FF3A00009002980168086820F0010008600298A1
:10FF4A000068806820F06060019908430299096896
:10FF5A0088600298FFF7BBFD00980299096808605B
:10FF6A0002992020C1F888000299002081F88400B3
:0EFF7A0000208DF80F009DF80F0004B080BD30
:10FF880010B588B0DDF82CE0DDF828C0CDF81CE00D
:10FF9800CDF818C0059304920391029000200190B7
:10FFA800029847F20001C5F20021884206D0029863
:10FFB80042F20041C4F60201884200D106E042F252
:10FFC800D420C0F60200CE21F4F7E3FD039818B15F
:10FFD8000398B0F5803F00D106E042F2D420C0F685
:10FFE8000200CF21F4F7D5FD049818B10498B0F5B4
:08FFF800805F00D106E042F237
:020000040801F1
:10000000D420C0F60200D021F4F7C7FD059838B11E
:100010000598B0F5804F03D00598B0F5004F00D19A
:1000200006E042F2D420C0F60200D121F4F7B5FD7B
:10003000069818B10698B0F5003F00D106E042F2EC
:10004000D420C0F60200D221F4F7A7FD0798800A59
:1000500000B906E042F2D420C0F60200D321F4F742
:100060009CFD0398049B059A069918431043084386
:10007000079901430198084301900298406842F6AD
:100080000041CFF6C07108400199084302994860C9
:06009000002008B010BDC5
:0E00960081B000900098D0F8800001B0704753
:1000A40082B001900091009800680199C1F8800025
:0600B400002002B07047BD
:1000BA0080B584B0039002910020019002984068B4
:1000CA003F2800D807E042F2D420C0F6020040F2EE
:1000DA006511F4F75DFD0298806848B1029880685E
:1000EA00B0F5807F04D002988068B0F5407F00D1D7
:1000FA0007E042F2D420C0F602004FF4B371F4F7DD
:10010A0047FD0298C06848B10298C068B0F5806F90
:10011A0004D00298C068B0F5006F00D107E042F23F
:10012A00D420C0F6020040F26711F4F731FD0298BC
:10013A00006920B102980069B0F5805F00D107E03C
:10014A0042F2D420C0F602004FF4B471F4F720FD55
:10015A000298006803998860029948688B68CA689F
:10016A000969184310430143019808430190039811
:10017A00C0684EF2C001CFF6FE71084001990843EB
:0A018A000399C860002004B080BD96
:0E01940081B0009000980069C0B201B07047C1
:1001A20080B584B003900291029840B1029804286D
:1001B20005D00298082802D002980C2800D107E046
:1001C20042F2D420C0F602004FF4CA71F4F7E4FC04
:1001D200039802990844143001900198006804B011
:0201E20080BDDE
:1001E40080B584B003900291002001900298406889
:1001F400400E00B907E042F2D420C0F6020040F2FB
:10020400A911F4F7C8FC02988068B8B30298806812
:10021400102833D00298806820282FD00298806854
:1002240030282BD002988068402827D00298806814
:10023400502823D00298806860281FD002988068D4
:1002440070281BD002988068802817D00298806894
:10025400902813D002988068A0280FD00298806854
:10026400B0280BD002988068C02807D00298806814
:10027400D02803D002988068E02800D107E042F239
:10028400D420C0F602004FF4D571F4F784FC029830
:10029400C06818B10298C068022800D107E042F291
:1002A400D420C0F6020040F2AB11F4F774FC0298BB
:1002B400006938B102980069042803D002980069E3
:1002C400082800D107E042F2D420C0F602004FF41F
:1002D400D671F4F760FC0298406918B1029840693D
:1002E400012800D107E042F2D420C0F6020040F217
:1002F400AD11F4F750FC0298006803994862029823
:1003040040680399886202998868CB680A694969D8
:100314001843104301430198084301900398C06AAD
:1003240020F0FF00019908430399C862002004B03B
:0203340080BD8A
:1003360080B58AB009900891089803901020019022
:1003460004904FF480700590002006904FF4805082
:100356000790099803A9FFF7ADFE0199099841F2A4
:0E036600883200F004F8029002980AB080BDC0
:1003740080B588B006908DF817100492049846F65C
:100384004C71C2F200410968C90844F6D352C1F263
:100394006202A1FB02218909484301900198411E90
:1003A400019118B94FF000400790E5E00698406BC2
:1003B4000290029901204522C0F2200211420090CD
:1003C40004D09DF80900C0F3401000900098C007C5
:1003D4000028E3D10698406B4007002804D506990D
:1003E400042088630790C7E00698406BC00720B1DB
:1003F4000699012088630790BEE00699C520C0F2E3
:10040400200088630698FFF7C3FE9DF81710884202
:1004140002D001200790AFE006980021FFF7BFFE4D
:10042400039003984EF20801CFF6FF51084202D11F
:1004340000200790A0E09DF80F000006002803D5D7
:100444004FF00070079097E09DF80F0040060028D9
:1004540002D5402007908FE09DF80F008006002809
:1004640002D58020079087E09DF80F00C006002881
:1004740003D54FF4807007907EE09DF80F000007CD
:10048400002803D54FF40070079075E09DF80F0025
:100494004007002803D54FF4806007906CE09DF876
:1004A4000F00C00718B14FF40060079064E09DF896
:1004B4000E000006002803D54FF4805007905BE03F
:1004C4009DF80E004006002803D54FF40050079015
:1004D40052E09DF80E008006002803D54FF48040BA
:1004E400079049E09DF80E00C006002803D54FF49C
:1004F4000040079040E09DF80E004007002803D517
:100504004FF40030079037E09DF80E008007002874
:1005140003D54FF4802007902EE09DF80E00C0070D
:1005240018B14FF40020079026E09DF80D00000656
:10053400002803D54FF4801007901DE09DF80D00AE
:100544004006002803D54FF40010079014E09DF8EE
:100554000D008006002803D54FF4800007900BE0BF
:100564009DF80C000007002803D54FF40000079005
:0E05740002E04FF480300790079808B080BD79
:1005820080B58AB0099008910898039011200190D3
:1005920004904FF480700590002006904FF4805034
:1005A2000790099803A9FFF787FD0199099841F27D
:0E05B2008832FFF7DEFE029002980AB080BD8C
:1005C00080B58AB009900891089803901220019094
:1005D00004904FF480700590002006904FF48050F6
:1005E0000790099803A9FFF768FD0199099841F25E
:0E05F0008832FFF7BFFE029002980AB080BD6D
:1005FE0080B58AB009900891089803901820019050
:10060E0004904FF480700590002006904FF48050B7
:10061E000790099803A9FFF749FD0199099841F23E
:0E062E008832FFF7A0FE029002980AB080BD4D
:10063C0080B58AB009900891089803901920019010
:10064C0004904FF480700590002006904FF4805079
:10065C000790099803A9FFF72AFD0199099841F21F
:0E066C008832FFF781FE029002980AB080BD2E
:10067A0080B58AB0099008910898039007200190E4
:10068A0004904FF480700590002006904FF480503B
:10069A000790099803A9FFF70BFD0199099841F200
:0E06AA008832FFF762FE029002980AB080BD0F
:1006B80080B588B007904FF4D57002900820039059
:1006C8004FF480700490002005904FF480500690FD
:1006D800079802A9FFF7EDFC07980BF09AF901902B
:0606E800019808B080BD7E
:1006EE0080B58AB009900891089803903720019040
:1006FE0004904FF480700590002006904FF48050C7
:10070E000790099803A9FFF7D1FC0199099841F2C6
:0E071E008832FFF728FE029002980AB080BDD4
:10072C0080B588B007900691069801902920029018
:10073C004FF480700390002004904FF4805005908B
:10074C00079801A9FFF7B3FC07980BF0AEF90090DE
:06075C00009808B080BD0A
:1007620080B58AB0099008910898039006200190FC
:1007720004904FF480700590002006904FF4805052
:100782000790099803A9FFF797FC0199099841F28C
:0E0792008832FFF7EEFD029002980AB080BD9B
:1007A00080B588B00790002002903321009103911A
:1007B0004FF48071049105904FF480500690079893
:1007C00002A9FFF77AFC0099079841F28832FFF7F7
:0A07D000D1FD0190019808B080BD32
:1007DA0080B588B0079000200290022103914FF45F
:1007EA004071049105904FF480500690079802A931
:1007FA00FFF75EFC079800F004F80190019808B032
:02080A0080BDAF
:10080C0085B0039046F64C70C2F200400068C008F8
:10081C0044F6D351C1F26201A0FB0110800941F2F0
:10082C008831484301900198411E019118B94FF04D
:10083C00004004902CE00398406B029001209DF83E
:10084C00081011F0450F009004D09DF80900C0F37A
:10085C00401000900098C0070028E4D10398406B2A
:10086C004007002804D503990420886304900FE006
:10087C000398406BC00720B1039901208863049052
:10088C0006E00399C520C0F2200088630020049084
:06089C00049805B070474E
:1008A20080B588B0079006910698019009200290C1
:1008B2004FF440700390002004904FF48050059054
:1008C200079801A9FFF7F8FB0798FFF79EFF009032
:0608D200009808B080BD93
:1008D80080B58AB009900891002003900321019106
:1008E80004914FF48071059106904FF48050079061
:1008F800099803A9FFF7DDFB01990998089A00F008
:0A09080004F8029002980AB080BDC6
:1009120080B588B006908DF81710049246F64C7098
:10092200C2F200400068C00844F6D351C1F262012D
:10093200A0FB0110800941F28831484301900198DF
:10094200411E019118B94FF0004007905AE00698F5
:10095200406B029001209DF8081011F0450F0090A5
:1009620004D09DF80900C0F3401000900098C00721
:100972000028E4D10698406B4007002804D5069968
:100982000420886307903DE00698406BC00720B1C1
:10099200069901208863079034E00698FFF7F9FB77
:1009A2009DF81710884202D0012007902AE006998C
:1009B200C520C0F22000886306980021FFF7F0FBF3
:1009C20003909DF80D0010F0E00F06D1BDF80E0067
:1009D200049908800020079014E09DF80D0040065D
:1009E200002803D54FF4005007900BE09DF80D004E
:1009F2000006002803D54FF48050079002E04FF420
:0A0A020080300790079808B080BD0F
:100A0C0080B58AB009900891089803900D20019048
:100A1C0004904FF480700590002006904FF48050A5
:100A2C000790099803A9FFF742FB0199099841F235
:0E0A3C008832FFF799FC029002980AB080BD44
:100A4A0080B588B00790002002900D210091039193
:100A5A004FF48071049105904FF4805006900798E6
:100A6A0002A9FFF725FB0099079841F28832FFF7A0
:0A0A7A007CFC0190019808B080BDDB
:100A840080B586B08DF816008DF81510ADF81220DB
:100A94008DF811309DF81600052803DBFF208DF832
:100AA4001700E0E09DF8150001460291012807D0E7
:100AB4000298023803280FD3029805280DD00DE0C0
:100AC4000F2003A9042200F0A8FF039818B9FD2001
:100AD4008DF81700C7E005E004E003E0FB208DF883
:100AE4001700C0E09DF811004007002803D5FA2044
:100AF4008DF81700B7E09DF8110010B39DF81500AC
:100B040001460191012803D0019802280AD018E077
:100B14009DF8110010F0210F03D1FA208DF8170071
:100B2400A1E00EE09DF811008006002808D59DF88C
:100B340011000006002803D4FA208DF8170092E073
:100B4400FFE79DF816000AF0F6FF9DF816104FF423
:100B5400806000EB01209DF815109DF8112002F033
:100B6400F002114300F048FEBDF81200A0B946F6A9
:100B74005070C2F2004001884A1C0280ADF8121085
:100B840000884FF6F071884206D146F65071C2F2E1
:100B940000414FF4404008809DF8161040F2044094
:100BA40000EB01209DF8131000F026FE9DF81610AE
:100BB40040F2054000EB01209DF8121000F01CFEED
:100BC4009DF8161040F2014000EB0120012100F0D5
:100BD40013FE9DF8161040F2014000EB012000F0D6
:100BE40058FE00B1F5E79DF81610012000FA01F354
:100BF40042F2F842C2F200421188994311809DF8F2
:100C0400111001F001019DF8163001FA03F3118867
:100C1400194311809DF8161000FA01F242F2F641D0
:100C2400C2F200410888904308809DF8162042F2E1
:100C3400E841C2F20041002021F812009DF816207C
:100C440046F6B261C2F2004188549DF8161040F293
:100C5400034000EB012000F01CFE00B9F5E79DF80D
:0E0C640016008DF817009DF9170006B080BD30
:100C720080B582B08DF806009DF80600052803DBDA
:100C8200FF208DF807005CE09DF806104FF48060AD
:100C920000EB012000F0FEFD00F00F00012803D060
:100CA200FB208DF807004CE09DF8061040F2014051
:100CB20000EB0120082100F0A0FD9DF8061040F293
:100CC200014000EB012000F0E5FD00B1F5E79DF8E1
:100CD2000610012000FA01F242F2F641C2F200418E
:100CE20008889043088042F2F840C2F2004000882F
:100CF2009DF80610C840C00718B100208DF8070003
:100D02001FE09DF8061040F2034000EB012000F0C6
:100D1200C1FD98B19DF8061040F2024000EB01209F
:100D220000F0B8FD0007002807D59DF806000AF07C
:100D320003FFF3208DF8070003E0E2E701208DF8BE
:0A0D420007009DF9070002B080BD14
:100D4C0080B586B08DF813000391ADF80A20002011
:100D5C008DF80900ADF806009DF81300052803DB9B
:100D6C004FF0FF300590E9E09DF813104FF48060D0
:100D7C0000EB012000F089FD00F00F00012803D0EA
:100D8C006FF004000590D9E0BDF80A0018B96FF0B7
:100D9C000D000590D2E09DF8131040F2034000EBDB
:100DAC00012000F072FD8DF809009DF8090017284C
:100DBC0007D09DF809001C2803D06FF006000590A1
:100DCC00BCE042F2F640C2F2004000889DF81310DD
:100DDC00C840C007A0B39DF8131040F2024000EBCE
:100DEC00012000F052FD8DF809009DF80900C006A5
:100DFC00002815D59DF8131040F2024000EB01209D
:100E0C00102100F0F5FC9DF81310012000FA01F2FE
:100E1C0042F2F641C2F200410888904308800FE08C
:100E2C009DF809000007002807D59DF813000AF06B
:100E3C007EFE6FF00C00059080E0002005907DE0B8
:100E4C001B2000F022FD9DF81310490003228A405C
:100E5C00104020FA01F1012088408002ADF8060014
:100E6C00BDF80A00BDF80610884203DDBDF8060087
:100E7C00ADF80A009DF813000AF00FFFADF806005C
:100E8C009DF8131040F2034000EB012000F0FDFC34
:100E9C008DF809009DF8090017280BD09DF8090062
:100EAC001C2807D09DF813000AF041FE6FF00600D5
:100EBC00059043E042F2F840C2F2004000889DF8F1
:100ECC001310C840C00740B1BDF80A00BDF80610A9
:100EDC00884202DD0020059030E0BDF80A00BDF824
:100EEC000610884200DC00E0C4E79DF8130003996B
:100EFC00BDF80A200AF065FF9DF8131040F201407E
:100F0C0000EB0120202100F073FC9DF8131040F23F
:100F1C00014000EB012000F0B8FC00B1F5E79DF8B2
:100F2C001310012000FA01F242F2F641C2F2004124
:100F3C00088810430880BDF80A000590059806B093
:020F4C0080BD66
:100F4E0080B586B08DF813000391ADF80A2000200D
:100F5E008DF80900ADF806009DF81300052803DB97
:100F6E004FF0FF300590B1E09DF813104FF4806004
:100F7E0000EB012000F088FC00F00F00012803D0E8
:100F8E006FF004000590A1E0BDF80A0018B96FF0EB
:100F9E000D0005909AE01A2000F076FC9DF81310D3
:100FAE00490003228A40104020FA01F101208840B6
:100FBE008002ADF80600BDF80600BDF80A108842A2
:100FCE0003DABDF80600ADF80A009DF813000AF02A
:100FDE00ADFEADF806009DF8131040F2034000EB95
:100FEE00012000F051FC8DF809009DF8090017282A
:100FFE0030D09DF809001C2824D1BDF8060000B1A0
:10100E003DE09DF813000AF047FE00901B2000F013
:10101E003BFC014600989DF8132052000323934099
:10102E00194021FA02F20121914089B289028842C7
:10103E0007D19DF813000AF079FD6FF006000590B8
:10104E0044E007E09DF813000AF070FD6FF0060013
:10105E0005903BE042F2F840C2F2004000889DF855
:10106E001310C840C00728B1BDF8060010B9002003
:10107E0005902BE0BDF8060000B100E0A5E7BDF835
:10108E000600BDF80A10884203DABDF80600ADF876
:10109E000A009DF813000399BDF80A200AF048FFD4
:1010AE009DF8131040F2014000EB0120402100F0AA
:1010BE009EFB9DF8131040F2014000EB012000F062
:1010CE00E3FB00B1F5E7BDF80A000590059806B000
:0210DE0080BDD3
:1010E00080B58AB084460C988DF823C00791ADF87E
:1010F0001A200593ADF8120000208DF81100ADF80C
:101100000E009DF82300052803DB4FF0FF30099007
:1011100042E19DF823104FF4806000EB012000F0C5
:10112000BAFB00F00F000238022800D803E06FF08D
:101130000400099030E1BDF81A0018B96FF00D00F5
:10114000099029E105980078029002990598407865
:1011500040EA0120029002990598807840EA012037
:10116000029002990598C07840EA01200290029806
:1011700078B99DF823104FF4806000EB012000F057
:101180008AFB00F00400042803D06FF00B000990E4
:1011900002E1BDF8120078B99DF823104FF4806089
:1011A00000EB012000F077FB00F00400042803D0DE
:1011B0006FF00A000990EFE09DF8231040F2034021
:1011C00000EB012000F067FB8DF811009DF8110085
:1011D00042280BD09DF81100222807D09DF811005D
:1011E000322803D06FF006000990D5E09DF8231057
:1011F00040F20C4000EB01200599042200F09AFB1C
:101200009DF823104FF4826000EB01209DF813102D
:1012100000F0F4FA9DF8231040F2114000EB012099
:101220009DF8121000F0EAFA1B2000F034FB9DF844
:101230002310490003228A40104020FA01F10120C6
:1012400088408002ADF80E00BDF81A00BDF80E10FF
:10125000884203DDBDF80E00ADF81A009DF82300AA
:101260000AF021FDADF80E009DF8231040F2034076
:1012700000EB012000F00FFB18B96FF0030009909C
:101280008AE042F2F840C2F2004000889DF8231044
:10129000C840C00740B1BDF81A00BDF80E10884222
:1012A00002DD0020099077E0BDF81A00BDF80E10AD
:1012B000884200DC00E0D1E79DF823000799BDF8E3
:1012C0001A200AF084FD0F2002A9042200F0A7FBD7
:1012D000029878B90520009002A90422019200F03A
:1012E0009EFB0098019A41F69A71C0F6020100F047
:1012F00021FB01E0002002909DF8231040F2014004
:1013000000EB0120202100F079FA9DF8231040F233
:10131000014000EB012000F0BEFA00B1F5E79DF8B6
:10132000231040F2024000EB012000F0B4FA8DF8E7
:1013300011009DF81100C006002809D59DF8231062
:1013400040F2024000EB0120102100F057FA19E0B2
:101350009DF811000007002813D59DF8231040F2D6
:10136000024000EB0120082100F048FA029820B169
:10137000052002A9042200F0DDFA6FF00C000990AC
:101380000AE0CCE7029820B1052002A9042200F06F
:0E139000D1FABDF81A00099009980AB080BD84
:10139E0080B58AB0DDF830C08DF823000791ADF826
:1013AE001A2005930020ADF808009DF823000528AB
:1013BE0003DB4FF0FF30099016E29DF823104FF437
:1013CE00806000EB012000F05FFA8DF8130000F052
:1013DE000F01881E0191032803D30198052801D01F
:1013EE0001E004E003E06FF004000990FCE1BDF8B9
:1013FE001A0018B96FF00D000990F5E19DF8231051
:10140E0042F2E840C2F2004030F8110038BB9DF8BD
:10141E0023000AF08BFCADF808009DF8231040F273
:10142E00034000EB012000F02FFA18B96FF0030013
:10143E000990D9E142F2F840C2F2004000889DF8CE
:10144E002310C840C00728B1BDF8080010B900200D
:10145E000990C9E1BDF8080000B100E0D7E79DF89A
:10146E00130000F0070001460091022808D00098F2
:10147E00032800F0FB800098042800F0838068E1C8
:10148E009DF8231042F2E840C2F2004030F81100FD
:10149E00002850D19DF823000DF10B0108220AF00F
:1014AE0047FD9DF8231040F2014000EB0120402142
:1014BE0000F09DF99DF8231040F2014000EB012051
:1014CE0000F0E2F900B1F5E79DF80B000599087000
:1014DE009DF80C00059948709DF80D0005998870CF
:1014EE009DF80E000599C8709DF80F000C990880A4
:1014FE000C990A889DF8100040EA022008809DF899
:10150E0011009DF8232042F2E841C2F2004121F879
:10151E0012009DF8232031F812309DF8120040EA97
:10152E00032021F812009DF8232046F6B261C2F284
:10153E00004180208854BDF81A009DF8232042F205
:10154E00E841C2F2004131F81210884204DABDF8C7
:10155E001A00ADF8080009E09DF8231042F2E840A9
:10156E00C2F2004030F81100ADF80800BDF80800D6
:10157E00ADF81A009DF823000799BDF808200AF06F
:10158E00D7FCF6E09DF8231042F2E840C2F200408C
:10159E0030F81100002846D19DF823000DF10B0103
:1015AE0002220AF0C5FC9DF8231040F2014000EB28
:1015BE000120402100F01BF99DF8231040F201405C
:1015CE0000EB012000F060F900B1F5E79DF80B107B
:1015DE009DF8232042F2E840C2F2004020F812109B
:1015EE009DF8232030F812309DF80C1041EA0321AB
:1015FE00023920F812109DF8231030F8110040F235
:10160E00EB51884207DB9DF823000AF08FFA6FF446
:10161E007A700990E8E09DF8232046F6B261C2F296
:10162E00004180208854BDF81A009DF8232042F214
:10163E00E841C2F2004131F81210884204DABDF8D6
:10164E001A00ADF8080009E09DF8231042F2E840B8
:10165E00C2F2004030F81100ADF808009DF82300EA
:10166E000799BDF808200AF063FC82E09DF823106C
:10167E0042F2E840C2F2004030F81100002845D195
:10168E009DF823000DF10B0106220AF051FC9DF886
:10169E00231040F2014000EB0120402100F0A7F89A
:1016AE009DF8231040F2014000EB012000F0ECF811
:1016BE0000B1F5E79DF80B00059908709DF80C0038
:1016CE00059948709DF80D00059988709DF80E00DB
:1016DE000599C8709DF80F009DF8232042F2E8414D
:1016EE00C2F2004121F812009DF8232031F8123089
:1016FE009DF8100040EA032021F812009DF82320E7
:10170E0046F6B261C2F2004180208854BDF81A003C
:10171E009DF8232042F2E841C2F2004131F8121046
:10172E00884204DABDF81A00ADF8080009E09DF809
:10173E00231042F2E840C2F2004030F81100ADF83A
:10174E0008009DF823000799BDF808200AF0F0FB69
:10175E000FE09DF82300BDF808100AF0A1FCBDF8BB
:10176E0008009DF8232042F2E841C2F2004121F820
:10177E0012009DF8231040F2014000EB01204021A1
:10178E0000F035F89DF8231040F2014000EB0120E7
:10179E0000F07AF800B1F5E7BDF808309DF8232087
:1017AE0042F2E840C2F2004030F81210C91A20F896
:1017BE0012109DF8231030F8110050B19DF823201F
:1017CE0046F6B261C2F20041885C40F001008854D6
:1017DE0007E09DF8232046F6B261C2F200410020D8
:0E17EE008854BDF80800099009980AB080BD23
:1017FC0080B586B005908DF8131046F6E060C2F205
:10180C0000400290C0688047029840698047029867
:10181C00806AB8B946F6E060C2F200400190016AF5
:10182C00F02088470198016A9DF8150088470198B7
:10183C00016A9DF8140088470198016A9DF813000D
:10184C00884716E0F0208DF80F000598000A8DF8F7
:10185C00100005988DF811009DF813008DF81200FA
:10186C0046F6E060C2F20040826A0DF10F000421DE
:10187C00904746F6E060C2F20040009080698047D5
:0A188C0000980069804706B080BD97
:1018960080B586B0059046F6E060C2F2004003903F
:1018A600C06880470398406980470398406A28B11A
:1018B60046F6E060C2F20040806A90B946F6E06003
:1018C600C2F200400290016A0F2088470298016A1E
:1018D6009DF8150088470298016A9DF8140088470C
:1018E60011E00F208DF810000598000A8DF8110000
:1018F60005988DF8120046F6E060C2F20040826A52
:1019060004A80321904746F6E060C2F20040019029
:10191600C0698047014601988DF813108069804799
:0E1926000198006980479DF8130006B080BD4F
:1019340080B588B007900691ADF816200020ADF868
:10194400100046F6E060C2F200400390C068804791
:101954000398406980470398806A90BB46F6E0602C
:10196400C2F200400290016AF02088470298016A9E
:101974000798BDF81020104480B2000A88470298E6
:10198400016A0798BDF810201044C0B288470020AF
:10199400ADF81000BDF81000BDF8161088420FDA3B
:1019A40046F6E060C2F20040016A0698BDF81020D5
:1019B400805C8847BDF810000130ADF81000E9E7FD
:1019C4001FE0F0208DF813000798BDF810100844AC
:1019D400000A8DF814000798BDF8101008448DF81B
:1019E400150046F6E060C2F200400190826A0DF1F3
:1019F4001300032190470198826A0698BDF81610D7
:101A0400904746F6E060C2F200400090806980474B
:0A1A140000980069804708B080BD0B
:101A1E0080B588B007900691ADF816200020ADF87D
:101A2E00100046F6E060C2F200400390C0688047A6
:101A3E000398406980470398406A28B146F6E060F3
:101A4E00C2F20040806A90BB46F6E060C2F20040EF
:101A5E000290016A0F2088470298016A0798BDF824
:101A6E001020104480B2000A88470298016A079835
:101A7E00BDF810201044C0B288470020ADF8100009
:101A8E00BDF81000BDF8161088420FDA46F6E06079
:101A9E00C2F20040C06980470699BDF810208854F4
:101AAE00BDF810000130ADF81000E9E71FE00F207F
